:020000040801F1
:100000005057002025020108A96F01085D6501080D
:10001000A56F01081B1A01081DAE010800000000B1
:100020000000000000000000000000008D9E01089C
:10003000EB300108000000004571010819A6010815
:10004000DDAE01083571010811A80108258B0108F2
:10005000F15D0108258901081D5C0108215C01088A
:100060006D5C0108B95C0108BD5C0108552F0108F1
:10007000572F0108592F01085B2F01085D2F010838
:100080005F2F0108612F0108731401082FAD0108CB
:1000900031AD0108251A0108271A0108095D010878
:1000A00013A8010819A8010817A8010815A8010834
:1000B0001BA801081DA801081FA801086365010805
:1000C000616501086765010865650108879E01088B
:1000D000899E0108BDAA0108C1AA010865AB0108F3
:1000E0001F5C0108F58901082DAD010827A801084A
:1000F0002DA801082BA8010829A8010875140108DA
:10010000255E0108859E010821A801088B9E010833
:10011000B9AA0108BBAA010823A8010825A801085B
:10012000632F0108652F0108672F0108692F010857
:1001300000F002F800F067F80AA090E8000C824492
:100140008344AAF10107DA4501D100F05CF8AFF26F
:10015000090EBAE80F0013F0010F18BFFB1A43F0A5
:100160000103184738750200587502000A444FF021
:10017000000C10F8013B13F0070408BF10F8014B06
:100180001D1108BF10F8015B641E05D010F8016B4B
:10019000641E01F8016BF9D113F0080F1EBF10F8AF
:1001A000014BAD1C0C1B09D16D1E58BF01F801CBD2
:1001B000FAD505E014F8016B01F8016B6D1EF9D555
:1001C0009142D6D37047000000230024002500266A
:1001D000103A28BF78C1FBD8520728BF30C148BFAA
:1001E0000B607047692900F06180002070471FB5DF
:1001F0009DE8030000F0F8FC00F082FE1FBD10B582
:1002000000F0E7FE10BD00F01BFF1146FFF7EFFF07
:100210000DF0E0F901F082F803B4FFF7F0FF03BC42
:100220000BF096FA0348004703480449044A054B7B
:100230007047000031010108504D00205057002048
:10024000505200205052002070470FB4014610B5A4
:1002500004AA039800F0A2FB10BC5DF814FB70B573
:10026000044685690068C10601D5302600E02026D5
:10027000C00707D070BDD4E9012130469047206AFD
:10028000401C20626D1EF6D570BD70B504468569B0
:100290000078C00707D170BDD4E901212020904724
:1002A000206A401C20626D1EF6D570BD2DE9F0411C
:1002B0000646002410687529314616A510D0AFF304
:1002C0000080002802DA404213A507E031688A075F
:1002D00001D512A502E0490704D511A5012401E0CA
:1002E000AFF3008000210A2206F1240709E0B0FBE9
:1002F000F2FCB0FBF2F302FB1C00303078541846DD
:10030000491C0028F3D123462A463046BDE8F04177
:1003100000F0EBBA000000002D0000002B000000F0
:10032000200000002DE9F05F894604464FF0000AE6
:10033000DFF824B1FB44C0F820A02046E1688847DC
:1003400000287DD0252806D0D4E901219047206AD5
:10035000401C2062F1E700255F462046E16888479F
:100360002028064607DB312E05D2B81910F8200CDC
:1003700008B10543F1E7A80701D525F00405C4F845
:100380001CA00027C4F818A02A2E09D030460BF074
:10039000CDF938B304EB8708303EC8F8186019E08F
:1003A00059F8041B204604EB87029161E1688847F5
:1003B000012F064618D1E069002820DA25F0200533
:1003C0001DE0D8F8180000EB800006EB4000303844
:1003D000C8F818002046E168884706460BF0A6F9E1
:1003E0000028EED1012F0AD02E2E08D12046E16838
:1003F00088477F1C0646022F45F02005C4DBA06914
:10040000002803DA404245F00105A061E80701D069
:1004100025F01005A6B1A6F14100192802D8203612
:1004200045F400654A463146204625604D46FFF7B3
:10043000D9FE60B1012807D0ED1D25F0070000E0CE
:1004400007E000F1080978E705F1040975E730468F
:100450007AE7206ABDE8F09F4B4B02002DE9F0419E
:1004600017460D4604460646012913DD38460CF0B2
:1004700025FB411C0CD0C0B20A2804F8010B02D0A5
:100480006D1E012DF2DC002020703046BDE8F081A9
:10049000B44201D10020F9E7384600F091FA002873
:1004A000F1D00026EFE700002DE9F0410C460746A9
:1004B0001646104600F06EF82078611C61280AD0BC
:1004C000722802D077283CD102E00125002405E003
:1004D0000225042402E0082448F2020511F8010B69
:1004E0002B2806D0622809D011F8010C74280AD0F4
:1004F0000BE045F0030544F00204EFE745F0040586
:1005000044F00104EAE744F01004384621460BF0B9
:1005100035F9411C15D00021316171604FF4007133
:10052000F560F1617061200704D530460222002198
:1005300000F04AFA306D40F0010030653046BDE809
:10054000F0810020FBE72DE9F0410D460646104CF6
:10055000206DC10704D0410804D020F00104F7E762
:1005600022460EE0542000F06AF907000ED0206DFC
:1005700047F00101084354212065384600F0F4F8A3
:100580003A4629463046BDE8F0418DE70020D6E7DF
:10059000F04B00202DE9F04704464FF000094FF0E2
:1005A000FF37C568D4E90486A80707D0204600F0C5
:1005B000BBFA30460BF0C1F8002802DA3846BDE835
:1005C000F087280502D5404600F068F94C21204606
:1005D00000F0CAF8206D20F0010020654846EEE7E3
:1005E00010B5431C02E010F8011B71B18107FAD16C
:1005F0004FF0013202C88C1A8C4314EAC211F9D0B0
:10060000C01A0A0603D0C01E10BDC01A10BD0A04CD
:1006100001D0801E10BD0902FCD0401E10BD421E3C
:1006200012F8013F002BFBD111F8013B002B02F81F
:10063000013BF9D17047032A40F2308010F0030CDF
:1006400000F0158011F8013BBCF1020F624498BF25
:1006500011F801CB00F8013B38BF11F8013BA2F1C2
:10066000040298BF00F801CB38BF00F8013B11F03D
:10067000030300F02580083AC0F0088051F8043BDD
:10068000083A51F804CBA0E80810F5E7121D5CBF4A
:1006900051F8043B40F8043BAFF30080D20724BF7D
:1006A00011F8013B11F801CB48BF11F8012B24BF11
:1006B00000F8013B00F801CB48BF00F8012B704760
:1006C00010B5203AC0F00B80B1E81850203AA0E8ED
:1006D0001850B1E81850A0E81850BFF4F5AF5FEA21
:1006E000027C24BFB1E81850A0E8185044BF18C9D4
:1006F00018C0BDE810405FEA827C24BF51F8043B7B
:1007000040F8043B08BF7047D20728BF31F8023BCE
:1007100048BF11F8012B28BF20F8023B48BF00F862
:10072000012B70474FF000020429C0F0128010F036
:10073000030C00F01B80CCF1040CBCF1020F18BFBD
:1007400000F8012BA8BF20F8022BA1EB0C0100F050
:100750000DB85FEAC17C24BF00F8012B00F8012B23
:1007600048BF00F8012B70474FF0000200B5134658
:1007700094469646203922BFA0E80C50A0E80C50C1
:10078000B1F12001BFF4F7AF090728BFA0E80C5072
:1007900048BF0CC05DF804EB890028BF40F8042B6B
:1007A00008BF704748BF20F8022B11F0804F18BFD8
:1007B00000F8012B704700004FF0013C50F8042B6B
:1007C00051F8043B9A4221D1A2EB0C03934313EA64
:1007D000CC1317D150F8042B51F8043B9A4215D191
:1007E000A2EB0C03934313EACC130BD150F8042B68
:1007F00051F8043B9A4209D1A2EB0C03934313EA4C
:10080000CC13DBD04FF00000704700BFD01A01BA04
:10081000B1FA81F101F0180122FA01F0CB40C1F1E7
:100820002001DBB2C0B2C01A2CFA01F3D11A9143F5
:1008300011EAC311E6D1704770477047704770B531
:10084000064600F0B5F9056806F10B0020F0070434
:10085000B4429CBF002070BD2B466A68BAB11068D4
:10086000A04210D304F1080188423CBF5068586090
:1008700007D35168101941601168091B0160586065
:100880001460101D70BD13465268002AE7D121463E
:10089000284600F095F90028DED170BD70B50446F9
:1008A000051F00F085F90068002C14BF446870BD76
:1008B000002C18BFAC423CBF20466468F8D30168E6
:1008C0000A18AA4218BF456003D12A680546114498
:1008D000016028684119A1421CBF6C6070BD61684D
:1008E000696021680844286070BD2DE9F0470D4615
:1008F00099469246044600F124080168880604D50A
:10090000E06921F01001216000E00120A84201DD32
:10091000471B00E00027A1697A1902EB0900081AB9
:10092000A0612078C00602D42046FFF798FC00267C
:1009300008E0D4E901211AF806009047206A401C1B
:10094000761C20624E45F4DB2078C0060AD520468E
:10095000FFF785FC06E0D4E9012130209047206AAA
:10096000401C2062381EA7F10107F4DC07E0D4E93F
:10097000012118F805009047206A401C2062281EBB
:10098000A5F10105F3DC2046FFF77FFC2078000687
:1009900002D50220BDE8F0870120FBE7074B70B5C8
:1009A0000D467B4400F05BF90446284600F008F849
:1009B00010B14FF0FF3070BD204670BDB3C10000D4
:1009C000007B00F0800070472DE9F0410446164698
:1009D0000D464769007B80072ED038460AF0C5FED9
:1009E00050BB3EB3012E02D0022E25D104E020469A
:1009F00000F065FA05441DE038460AF0ABFEE168F8
:100A0000002841F01001E16005DA204600F058F8B6
:100A10000120BDE8F081C9030BD56268E16A91420B
:100A200000D81146A26911442269891A814200DD69
:100A300008460544002D01DA0220EAE7E16A606811
:100A4000E268814206D29103E06203D522F40031CC
:100A500041F01002A6690027AE4213DCE16A814230
:100A600001D90B4600E0034603EB060C2369ACEB0F
:100A7000030CAC4506DD814201D98C4600E084467A
:100A80009C4505D1A760276042F02000A5620DE0DB
:100A9000AD1BE669AE1B8142A66000D90846C01AAC
:100AA000281A20605819606022F02000034908408D
:100AB000E060002084F84870ABE70000BFCFD7FFAC
:100AC000C16821F4001141F08001C1600021816002
:100AD000016070472DE9F047814614460E464FF0FD
:100AE000FF383248D5685769054209D03846A169B0
:100AF0000AF083FE002811DB2C48C0430540E56066
:100B00002B463246494638460AF085FEA16920F058
:100B10000042B21A11440028A16103D02046FFF719
:100B2000CFFF4046BDE8F08770B504460569C06A4E
:100B30006168884200D80846E16821F42011E1602C
:100B4000C90312D5A84208D02246411B2846FFF708
:100B5000C1FF10B14FF0FF3070BD0020E562C4E965
:100B60000150E06820F48030E060002070BD10B5D6
:100B70000446C06820F02000E060A16AA0698842B5
:100B80000DD02046FFF7D0FFE06820F4405040F041
:100B90001000E060A06AA0612069E062606044F239
:100BA0004001E0688843E06010BD000010000200D2
:100BB00000487047F44C00207047704770477047FA
:100BC00038B504460A4600206946AFF30080002885
:100BD00008BF38BD02460099204600F05BFA0120AC
:100BE00038BD012000F0AABBF8B5AFF30080054680
:100BF00000200C46102000BF0646A819A0420DD9BF
:100C0000324669460020AFF30080070008BF00F0BD
:100C100095FB0098A04218BF0546C419FFF7C8FF0E
:100C200005600746F01D20F007004619284600F031
:100C30000AF8B44208BFF8BDA21B31463868BDE8C7
:100C4000F84000F027BA00210160C0E901107047A8
:100C50001020704701694A1C02610878704700B58E
:100C60008FB0CDE901310021059105497944CDE9E5
:100C7000031011466846FFF755FB0FB000BD00009A
:100C8000E5FFFFFF70B50D4601461446D368506975
:100C90002A460AF09FFD002807DA411C07D0E168C8
:100CA00020F0004041F48041E160281A70BD2046E8
:100CB000FFF706FF4FF0FF3070BDC16800220260F1
:100CC00021F4805141F0400111F4C06FC16001D0A6
:100CD0008260704702694168891AC269891A816015
:100CE00070472DE9F0470446C06840F48000E0609A
:100CF000010312D520F40020E060810606D4E26AE8
:100D000061688A4200D80A46511A216040F40010F6
:100D1000E06094F82500BDE8F08720F40010E06062
:100D2000800602D52046FFF722FFE06842F28101EB
:100D30004FF0FF390140012903D02046FFF7C0FEE4
:100D4000B6E02168002600290ADAC94340F4805041
:100D50002160C4E902606068411C61600078DAE7E4
:100D600044F2400108420CD020F4A04040F0400082
:100D70002660E06021696068401AE169401AA0605D
:100D800096E0216991B9C00310D4E069FFF757FDDF
:100D90002061B0B1E06840F4006010F4407FE06092
:100DA00002D140F48070E06020696060E068D4F8AF
:100DB00014A0C1061AD5C0030ED52046FFF7B4FE15
:100DC00014E004F1240020610120E061E06820F4D7
:100DD000407040F48060E6E721696068401AA169CC
:100DE000014450460AF009FD0028A6DBE068C00374
:100DF0002AD56168E06A884200D808462169451A08
:100E0000E069471B1BD02046D4F81880FFF78CFE02
:100E100008EB05015046C4F818800AF0EEFC0028E3
:100E20008BDBE06840F40030E060000202D5A0698E
:100E30002844A061E1692069C91B45180DE02046DE
:100E4000FFF772FEE769F5E725696168D4E90607EF
:100E5000491BE56208446560A061E06820F010006D
:100E600010F4C06FE06002D0204600F03BFAE0686A
:100E700040F48050C4E90260000205D52069E062B8
:100E800060606FF0010046E7224639462846FFF7CA
:100E9000F9FE411C0CD02918E16258B1401E2060B7
:100EA000681C6060E06840F40030E060287832E759
:100EB000484630E765602046FFF7FFFEF8E710B5CB
:100EC0000146C268900703D0900607D5886A0AE0F9
:100ED00000F0DCF801210160881E10BD8B694868B4
:100EE00018440B69C01A91F848301BB191F84910A9
:100EF000401A10BD1103FCD50028FADD401E10BDBC
:100F000010B542485421FFF72FFC41485421FFF708
:100F10002BFC40485421FFF727FC3F493B483C4A03
:100F20003F4B08603D490A603A491960531C03650C
:100F3000481C1065012008653B48344A39A17844B3
:100F4000FFF7B2FA20B9384878440A3800F0EFF9D0
:100F500037482F4A35A17844FFF7A6FA20B934481C
:100F600078440A3800F0E3F932482A4A2FA178443D
:100F7000FFF79AFA20B92F4878440A3800F0D7F9D9
:100F800040232248DC000021224600F088F920B1ED
:100F900025487844543800F0CAF91D4822464023B9
:100FA000002100F07CF920B121487844543800F049
:100FB000BEF9184822461023002100F070F90028DD
:100FC00006D01C487844BDE81040563800F0AFB950
:100FD00010BD104870B5006D20F001040B48FFF7FC
:100FE000D9FA0B48FFF7D6FA0A48FFF7D3FA09E017
:100FF000206D20F001052046FFF7CCFA2046FFF7D0
:101000004DFC2C46002CF3D170BD0000F04B0020AD
:10101000444C0020984C0020C4030020C80300204A
:10102000CC030020720000007E3701007700000032
:101030006C3701005B37010000487047EC4C002022
:101040007546FFF7F9FFAE4605006946534620F0A6
:101050000700854618B020B5FFF7E6F8BDE8204048
:101060004FF000064FF000074FF000084FF0000B64
:1010700021F00701AC46ACE8C009ACE8C009ACE817
:10108000C009ACE8C0098D467047000000487047B1
:10109000EC4C0020034640688C46002818BF88426C
:1010A0003CBF03464068F8D318681844884207D00C
:1010B0000CF1030020F00700001D411A521A0146EE
:1010C000081D0A60FFF7EABB2DE9F04705460C460C
:1010D000C86820F4201040F48000C860800602D563
:1010E0000846FFF744FDE06841F282014FF0FF3906
:1010F0000140022903D02046FFF7E2FCB5E000F4EE
:101100002041B1F5004F0FD1C00306D56168E06AF8
:10111000884200D80846606006E02069E0626060AE
:1011200060690AF017FBA061A0680022EEB20028F7
:101130000DDAE1688B050AD4C043A06041F4903019
:101140002260E0606068411C61600670A5E0E068B4
:101150009046226040F40050E060206968BB6069FE
:101160000AF003FB012704F12405A0B1A08910F4C3
:10117000407F08D0E069FFF762FB206118B1E068AA
:1011800040F4006016E0E7612561E06820F44070FB
:1011900040F480600EE0E069FFF751FB0028206119
:1011A000F1D0E06840F4006010F4407FE06002D1CC
:1011B00040F48070E06020696060E06825696FF04D
:1011C000010AC1051FD56168E06A884200D8084657
:1011D000411B04D022462846FFF77CFCF0BBE068A8
:1011E000010203D5E562C4E9015854E0691CE162DB
:1011F0006160E16940F48030491EC4E90210304664
:101200002E70BDE8F087010202D500F480320AE0BA
:101210006068411C61600670E0680A2E40F480300E
:10122000E06006D00022E16A6068814203D90B4683
:1012300002E00122F7E70346A7895B1B7F0503D481
:10124000E7699F4200DDE2B1814200D80146E562D4
:101250000F1AC4E90158002B09DD00E005E0224621
:1012600019462846FFF736FC08B14846C9E747B19A
:10127000A069E5626560C01BA061E06840F01000F5
:10128000E060E068000208D56168A069E562491B7A
:1012900008446560A0615046B3E73046B1E770B5D9
:1012A000C468A50713D0650211D4B2F5807F09D0B8
:1012B000B2F5007F06D0B2F5806F08D1012300F1AE
:1012C000240106E05D1E6FF07F46B54201D3012088
:1012D00070BD0161C361416024F470611143C1605C
:1012E000002070BD70B5054640F202260A4C0FE0A2
:1012F00094F85000C00708D0AC4206D0E06836EA47
:10130000000002D1204600F021F8206D20F00104F9
:10131000002CEDD170BD0000F04B002010B504464C
:10132000AFF300802046BDE81040FEF775BF10B552
:1013300000F044F8BDE8104000F03AB810B500F0F5
:1013400057F8BDE8104000F033B8000070B504460F
:10135000C068810713D0800601D5A56A04E0A169A1
:10136000606808442169451A2046FFF7DDFB00222A
:10137000064629462046FFF727FB304670BD002071
:1013800070BD70B510B1BDE87040DFE70025074CB7
:101390006E1E07E02046FFF7D9FF00B13546206DED
:1013A00020F00104002CF5D1284670BDF04B002040
:1013B000002801D00AF0CCB97047000010B50146F2
:1013C00002A000F03DF8012010BD00005349475233
:1013D000545245443A2052656469726563743A20F8
:1013E00063616E2774206F70656E3A200000000004
:1013F00010B5012805D0002103A000F021F801203C
:1014000010BD09A1F8E7000053494752544D454D1E
:101410003A204F7574206F662068656170206D6595
:101420006D6F7279000000003A2048656170206D90
:10143000656D6F727920636F727275707465640088
:1014400070B505460C460A2000E06D1C0AF0F6F95E
:1014500035B128780028F8D102E0641C0AF0EEF9D2
:1014600014B120780028F8D1BDE870400A200AF0B5
:10147000E5B9704770470029816802D041F0010149
:1014800001E021F0010181607047000010B50020EB
:10149000214908600120087148714FF4602088607C
:1014A0000020C860032008741C4800F059F8072386
:1014B00001220F21194800F077F8072302220821A2
:1014C000164800F071F8072303220921134800F0A1
:1014D0006BF80121114800F02DF801210F4800F0B0
:1014E0001FF801210D48FFF7C6FF0C4800F096F8E1
:1014F00000BF0A4800F02DF80028FAD1074800F094
:101500009CF800BF054800F01DF80028FAD1012121
:10151000024800F088F810BDA40D0020002401400E
:101520000029816802D041F4807101E021F48071CA
:10153000816070474268491E22F4604242EA4131AC
:1015400041607047014600208968490700D50120A5
:101550007047014600208968090700D501207047BF
:1015600010B542680E4B0C791A400B6842EA04220F
:101570001343436082680B4B1A40D1E90243234373
:101580004C7942EA440213438360C26A097C22F424
:101590007002491EC9B242EA0151C16210BD000089
:1015A000FFFEF0FFFDF7F1FF70B5072509290AD905
:1015B000C468A1F10A0606EB4606B540AC43B34049
:1015C0001C43C46007E0046901EB4106B540AC432D
:1015D000B3401C4304611F23072A09D2446B521EE7
:1015E00002EB820293409C4391400C43446370BDE4
:1015F0000D2A09D2046BD21F02EB820293409C4356
:1016000091400C43046370BDC46A0D3A02EB820240
:1016100093409C4391400C43C46270BD816841F08B
:101620000801816070470029816802D041F4A0015F
:1016300001E021F4A00181607047816841F004015C
:101640008160704710B51848007858B301211748D9
:1016500004F07DFE30BB65211548006809F08EFD61
:1016600000241CE0002240F22551124809F0F7FA4C
:1016700066220F480168002001F038FC0C48006821
:1016800008F020FB01F052FC012240F225510948EC
:1016900009F0E5FA002004490870601CC4B2032C6C
:1016A000E0DB00BF10BD0000D800002000080140B2
:1016B000D400002000440040114800681149096826
:1016C0000844401C00EB40000F4901EB800080689B
:1016D000A8B10C480068042805DA0A480068401CD4
:1016E0000849086008E006480068182804DA044839
:1016F0000068401C024908600120044908707047D6
:101700000803002030010020100C00203F010020C1
:101710000C480068002808DD0A480068401E094996
:1017200008600120084908700BE00848006800289C
:1017300007DD06480068401E044908600120024990
:1017400008707047300100203F010020080300208E
:1017500000B502460B46184600F010F802EB820175
:1017600000EB410000BD0146092903DD01F137000E
:10177000C0B2704701F13000C0B2FAE7014630292B
:1017800001DB392901DD002001E001F00F00704785
:101790000149405A70470000006C0040014A8152E4
:1017A00070470000006C00402DE9F84300244EA172
:1017B0004E48FEF7C8FE4E490860084600680028FB
:1017C0007ED04FF480614B4804F0CFFD01204A49A0
:1017D00008704AA146480068FEF737FD642007F00C
:1017E00043FA642190FBF1F201FB1205084607F071
:1017F0003BFA642190FBF1F090FBF1F201FB120641
:10180000084607F031FA42F2107190FBF1F73346C7
:101810003A4641A1364800950068FEF716FD474854
:1018200000683C2190FBF1F201FB1205434800687F
:1018300090FBF1F62B46324641A12D480068FEF799
:1018400004FD692007F010FA0546682007F00CFA3D
:10185000642190FBF1F6682007F006FA642190FB02
:10186000F1F201FB120733463A463AA120480095AF
:101870000068FEF7EAFC00BF204604F00BFB804640
:10188000204605F01DFA50B1404604F0CBFD054658
:101890002B46424636A116480068FEF7D6FC04F0F7
:1018A00073FE00F05FFD611C0C46084605F022FA4D
:1018B0000028E1D030A10E480068FEF7C6FC00E029
:1018C00010E04FF4FA502E49086001E004F05CFE8D
:1018D0002B4800680028F9D10749087004480068BF
:1018E000FEF758FEBDE8F883770000009C4D030822
:1018F000AC030020000C0140D80000202A2A204D13
:1019000069737454696D65206261636B75702066DC
:10191000696C652E0A0000002A2A2050726F6772D7
:10192000616D2056657273696F6E3A2025692E25A8
:101930003032692E253032690A0000003000002064
:101940002A2A2054696D653A20253032693A2530BB
:1019500032690A002A2A20446174653A202530320F
:10196000692D253032692D253034690A00000000C8
:1019700025693D25690A00002A2A20456E640A006F
:1019800018000020F0B506460C461746BC420BD1A5
:10199000C4EBC400104951F82000B04201D12046E8
:1019A000F0BD4FF0FF30FBE7E01900EBD0714D10B8
:1019B000C5EBC500084951F82000B04205DA3A46A7
:1019C000691C3046FFF7DEFFEAE72A46214630462B
:1019D000FFF7D8FFE4E7000038E9010810B500245C
:1019E0000FE004F29310002109F0FCFA04F2C51094
:1019F000002109F0F7FA04F2F710002109F0F2FAD9
:101A0000641C322CEDD300214FF4C97009F0EAFABE
:101A10000021662009F0E6FA10BD00BFFEE701468E
:101A200001207047704770470120704710B50121B1
:101A3000224804F08CFC00283FD10BF04FF800281E
:101A40003BD11F49A1F804011E480AF05BFF10B901
:101A500007F084FC31E008F073FC00220421084602
:101A600008F08AFC01220621042008F085FCFFF71B
:101A70009BFE00201249A1F8040113A00AF042FFC6
:101A800090B901210A2009F0ADFA01210B2009F0DB
:101A9000A9FA01210C2009F0A5FA0222072104204D
:101AA00008F06AFC00BFFEE700210A2009F09AFA5C
:101AB00005F0E4F901200649087010BD0008014056
:101AC000C04A00209C4D03084D545F562A00000078
:101AD0003F0100202DE9FC5F4FF0000B3B48006800
:101AE000C0EBC0003A4951F82090484604F0F8F99C
:101AF0000090484604F096FC0546009804F0C0F9B2
:101B00000746009804F0B2F98046009804F0A4F962
:101B10000190009805F0E2F88246BAF5204F3DD1D9
:101B2000642095FBF0F695FBF0F100FB115465B3D2
:101B30000D2E26D2DFE806F0250714081B091C0A23
:101B40000B1D0C1E0D0000BF00BF00BF00BF00BF7B
:101B500000BF012C01DB1F2C01DD4FF0010B13E056
:101B6000012C01DB1D2C01DD4FF0010B0CE000BF4F
:101B700000BF00BF012C01DB1E2C01DD4FF0010B6B
:101B800002E04FF0010B00BF00BFBBF1010F0ED10F
:101B900001224846019909F039FA08E0BD4201DB0B
:101BA000454504DD01224846019909F02FFA07480E
:101BB0000068401C054908600846006805F09AF86E
:101BC00010B1002001490860BDE8FC9F2000002002
:101BD00038E9010810B50121294804F0B8FB90BB91
:101BE000682007F041F8044640F2E63225480168D3
:101BF000204609F03FFA00BF07F090FB04F0C4FC58
:101C0000214800680F2190FBF1F201FB120080B91E
:101C10004FF480611D4804F0A1FB28B14FF48061AE
:101C20001A4804F0A2FB04E04FF48061174804F066
:101C30009EFB154800680028DED142F6A201642010
:101C400009F0D0F91AE0FFE700BFFFF743FF04F007
:101C50009BFC4FF480610D4804F080FB28B14FF4E9
:101C600080610A4804F081FB04E04FF4806107487A
:101C700004F07DFB044800680028E6D110BD000098
:101C8000000801403000002020000020000C01402E
:101C90007047000010B503480078012801D107F013
:101CA000EFFA10BD3E0100202DE9F041064640F25A
:101CB000831006F0D9FF4FEA8008002422E0301993
:101CC00006F0D2FF07463119481C06F0CDFF054645
:101CD000AF420ADA0D480068B84206DB0B480068DC
:101CE000A84202DA3019BDE8F081AF4209DD0748A9
:101CF0000068A84203DB05480068B84201DB3019E0
:101D0000F1E7241D4445DADB0020ECE73000002039
:101D100010B50B2006F0A8FF012817D108F010FB22
:101D200003220421084608F027FB0422062110465E
:101D300008F022FB00201849086000BF07F0EEFA07
:101D400004F022FC144800680028F7D100210B2081
:101D500009F048F90C2006F087FF012812D1002075
:101D60000AF0BCFE70B900200C49A1F804010C482F
:101D70000AF0C8FD30B905220621042008F0FCFA5B
:101D800007F0ECFA00210C2009F02CF905F076F8A8
:101D900001200449087010BD20000020C04A002026
:101DA0009C4D03083F0100202DE9F0416B2006F017
:101DB0005BFF0746002482E004EBC40000EB400612
:101DC00006F16C0006F050FF0546062D75D2DFE8DF
:101DD00005F0030A131C252E204608F0D1F83C48D4
:101DE00040F8245069E000223146204608F0A2F86D
:101DF000374840F8245060E000223146204608F081
:101E000075F9334840F8245057E000223146204607
:101E100008F0BEF82E4840F824504EE0002231462B
:101E2000204608F009F92A4840F8245045E029489E
:101E300050F8240050B9601C06F010FC0020264920
:101E400041F824000120234941F82400601C04F0DB
:101E5000E9FE88BB1E4850F82400052820D2DFE8A0
:101E600000F003070D131900204608F089F817E069
:101E700001223146204608F05DF811E0012231468A
:101E8000204608F033F90BE001223146204608F0E5
:101E90007FF805E001223146204608F0CDF800BF6A
:101EA00000BF00200B4941F82400094A52F82410D1
:101EB00006F16C0009F096F800BF00BF641C4FF4F7
:101EC000BD7006F0D1FEA0423FF776AFBDE8F081CD
:101ED000D40E0020FC0E0020E80B002010B54FF4BB
:101EE000C27006F0C1FE04464FF4BF7006F0BCFE9F
:101EF0002049096888420BDD1E4801684FF4BF7015
:101F000009F070F81C48016840F27F1009F06AF887
:101F10004FF4C07006F0A8FE1649096888420BDA33
:101F2000144801684FF4C07009F05CF81248016869
:101F300040F2811009F056F8DCB10F480068844285
:101F400017D10C4801684FF4BF7009F04BF80A48EC
:101F5000016840F27F1009F045F8064801684FF427
:101F6000C07009F03FF80448016840F2811009F0A0
:101F700039F810BD340000203000002010B5614851
:101F8000046861480068844204D05F48046001200E
:101F90005E4908605B4844685D480068844204D03C
:101FA0005B480460012059490860564884685948D4
:101FB0000068844204D057480460012053490860F7
:101FC000012004F053FA044653480068844204D0C8
:101FD0005148046001204D490860022004F046FA8F
:101FE00004464E480068844204D04C4804600220F5
:101FF00046490860032004F039FA0446484800685E
:10200000844204D04648046001204049086004200E
:1020100004F02CFA044643480068844204D0414846
:1020200004600120394908603F4800680B2836D217
:10203000DFE800F0060A0E12161A1E22262B3000C8
:1020400000203A4908602EE00220384908602AE062
:1020500004203649086026E008203449086022E060
:102060001020324908601EE02020304908601AE044
:1020700040202E49086016E080202C49086012E0BC
:102080004FF48070294908600DE04FF40070274933
:10209000086008E04FF480602449086003E00020F5
:1020A0002249086000BF00BF21480068012805D10F
:1020B0001E48006880F001001C4908601D48006847
:1020C000012806D11948006840F4006017490860EB
:1020D00005E01648006820F40060144908601648BE
:1020E0000068012806D11148006840F480500F496B
:1020F000086005E00D48006820F480500B49086036
:1021000010BD0000B00B00205C000020E8020020A1
:10211000600000207C000020640000206800002097
:102120006C00002070000020740000204C00002093
:1021300078000020800000208400002010B5414875
:10214000006820B1012831D0022874D155E03E4802
:1021500000683E490968884224D04FF4BE7006F0FA
:1021600083FDB0B13A48006860B901203849086081
:1021700040F27D1006F078FD3649086001203149B3
:10218000086012E000203349086001202D490860F2
:102190000BE000202E4908602E49086001202949E3
:1021A000086002E000202A49086048E029480068E9
:1021B00010BB2548006800EB4000274951F820007B
:1021C000264908602048006800EB4000224901EBE6
:1021D00080004068224908600120224908601A48AE
:1021E000006800EB40001C4901EB80008068194941
:1021F000086002201349086021E016480068C0B951
:102200000020164908601649086001201549086039
:102210000D480068401C142190FBF1F201FB1200F4
:10222000094908600221012006F0BEFF002005498F
:10223000086004E0FFE700200249086000BF00BF1B
:1022400010BD0000D0000020C8000020CC000020FD
:102250008C00002088000020E40D002038000020C1
:102260003C000020E802002070B50025002414E0A6
:1022700004EB4400114901EB8000806801280BD178
:1022800004EB44010D4A52F8211001F2851006F0CA
:10229000EBFC012800D10125641C192CE8DB35B9C1
:1022A0000748006840F001000549086005E004485F
:1022B000006820F001000249086070BD100C002089
:1022C0004C00002010B50221234804F040F830B142
:1022D0002248006840F001002049086005E01F48DE
:1022E000006820F001001D49086004211A4804F02C
:1022F0002EF830B11948006840F002001749086014
:1023000005E01648006820F00200144908608021AA
:10231000114804F01CF830B11048006840F0040087
:102320000E49086005E00D48006820F004000B49E4
:10233000086010210A4804F00AF830B10748006824
:1023400040F008000549086005E00448006820F0F6
:1023500008000249086010BD000801405800002034
:10236000001001402DE9F84F0020009084E07148F2
:102370000068401E6F49086006F0BAFB6E490860AD
:10238000084600686D4988420EDB012000906A48CB
:102390000068401A6849086006F052FC6648006808
:1023A00006F02EFC06F04CFC6548006820B164483D
:1023B0000068401E624908606248006820B16148B8
:1023C0000068401E5F4908605F48006820B15E48B1
:1023D0000068401E5C4908605C48006820B15B48AA
:1023E0000068401E594908605948006820B15848A3
:1023F0000068401E564908605648006820B155489C
:102400000068401E534908604FF000080CE0524835
:1024100050F8280030B1504850F82800401E4E496E
:1024200041F8280008F10108B8F10A0FEFDB4B482A
:102430000068002805DD49480068401E47490860DB
:1024400005E00A20454908600120454908604548E3
:10245000D0F800B006F04CFB3C21B0FBF1F9B9F527
:10246000B46F01DB40F29F59CB4502D03D48C0F824
:10247000009001203C4908702E48006800287FF435
:1024800076AF0098002853D0692006F0EDFB054692
:10249000E91705EB91718910A5EB810141B9642120
:1024A00095FBF1F201FB125111B14FF01D0A01E051
:1024B0004FF01C0A682006F0D7FB0646642196FB05
:1024C000F1F496FBF1F201FB1260471C0D2C18D2BF
:1024D000DFE804F0170712081709170A0B170C1783
:1024E0000D0000BF00BF00BF00BF00BF00BF1F2F17
:1024F00001DD641C012709E0574501DD641C01274B
:1025000004E01E2F01DD641C012700BF00BF0C2C5E
:1025100004DD0124691C692008F064FD04EBC4009B
:1025200000EB041007EB80063146682008F05AFDE6
:10253000BDE8F88F04000020BC000020805101009D
:1025400028030020DC020020B0000020A4000020AE
:10255000F800002088000020E80B0020B8000020D0
:10256000E802002030000020AC00002010B5344804
:10257000046804F0010008B106F014FD04F0020044
:1025800010B106F047FD01E006F03CFD04F0040048
:1025900010B106F051FD01E006F044FD04F0080022
:1025A00010B106F05DFD01E006F050FD04F01000F2
:1025B00010B106F069FD01E006F05CFD04F02000BA
:1025C00010B106F075FD01E006F068FD04F0400072
:1025D00010B106F081FD01E006F074FD04F080000A
:1025E00010B106F08DFD01E006F080FD04F480706E
:1025F00010B106F099FD01E006F08CFD04F40070C6
:1026000010B106F0A5FD01E006F098FD04F480602D
:1026100010B106F0BFFC01E006F0B4FC04F4006069
:1026200010B106F0E5FC01E006F0D8FC04F480509F
:1026300010B106F0CBFC01E006F0C0FC10BD0000BC
:102640004C0000204A4800680B287ED2DFE800F0EA
:10265000060F1A25303B46515C67720045480068FA
:1026600020F4FF7020F4C060424908606DE04148EA
:10267000006820F4FF7020F4C06040F002003D4983
:10268000086062E03B48006820F4FF7020F4C060FE
:1026900040F004003749086057E03648006820F4ED
:1026A000FF7020F4C06040F00800324908604CE040
:1026B0003048006820F4FF7020F4C06040F0100043
:1026C0002C49086041E02B48006820F4FF7020F49A
:1026D000C06040F020002749086036E025480068C7
:1026E00020F4FF7020F4C06040F0400021490860F1
:1026F0002BE02048006820F4FF7020F4C06040F018
:1027000080001C49086020E01A48006820F4FF702F
:1027100020F4C06040F480701649086015E0154848
:10272000006820F4FF7020F4C06040F4007011498C
:1027300008600AE00F48006820F4FF7020F4C060D1
:1027400040F480600B49086000BF00BF0A48006881
:1027500030B10848006840F400600649086005E0B0
:102760000448006820F400600249086070470000D7
:10277000380000204C0000208C0000200146A1F110
:102780003000C1B2092901DDC81FC1B201F00F003C
:10279000704700000021002009E0084A525C00EB6D
:1027A000800302EB4302A2F130004A1CD1B2034A7B
:1027B000525C0AB10829F0DB70470000410100209B
:1027C0002DE9F05F4FF0000900240027A046002506
:1027D0000026F7480078002877D009F031F8F5494D
:1027E00001EB0010D0F800A0504603F079FBF2494D
:1027F000086009F025F8EF4901EB0010D0F800B0AF
:10280000584603F06DFB824604F068FAB0F5A04F1D
:1028100070D014DCB0F5605F6DD009DCB0F5005FFE
:102820001FD0B0F5205F38D0B0F5405F34D168E0FC
:10283000B0F5804F73D0B0F5904FF7D101E1B0F50E
:10284000304F6DD006DCB0F5084F6AD0B0F5204FA0
:10285000ECD130E2B0F5484F7ED0B0F5943FE5D1F1
:102860007EE114E0D248005D2C2803D0D048005D02
:102870002D2802D14FF0010907E0CD48005D05EB9E
:10288000850100EB4100A0F13005601CC4B2C848CE
:10289000005D08B1082CE5DB85E221E0C448005D5D
:1028A0002D2802D14FF0010918E0C148005D2C2805
:1028B00001D1012712E04FB1BD48005D06EB860152
:1028C00000EB4100A0F1300608E090E2B848005D5E
:1028D00005EB850100EB4100A0F13005601CC4B29E
:1028E000B348005D08B1082CD8DB092E04DD4FF099
:1028F000010905E0E4E03CE005EB850006EB40055E
:1029000051E223E0AA48005D2D2802D14FF00109D1
:102910001AE0A748005D2C2804D1012714E05CE0F0
:102920008CE14BE147B1A248005D06EB860100EB6C
:102930004100A0F1300607E09D48005D05EB8501F0
:1029400000EB4100A0F13005601CC4B29848005D66
:1029500008B1082CD6DB00E0FCE1632E02DD4FF06D
:10296000010905E005EBC50000EB051006EB80054D
:1029700019E220E08E48005D2D2802D14FF00109B8
:1029800017E08B48005D2C2801D1012711E047B1E9
:102990008748005D06EB860100EB4100A0F13006A0
:1029A00007E08348005D05EB850100EB4100A0F1E5
:1029B0003005601CC4B27E48005D08B1082CD9DB2C
:1029C000B6F57A7F02DB4FF0010905E005EB450023
:1029D000C0EBC51006EBC005E5E120E07448005DE2
:1029E0002D2802D14FF0010917E07148005D2C2815
:1029F00001D1012711E047B16D48005D06EB86016A
:102A000000EB4100A0F1300607E06948005D05EBEE
:102A1000850100EB4100A0F13005601CC4B26448A0
:102A2000005D08B1082CD9DB42F20F70864202DD4E
:102A30004FF0010904E040F27120684306EB0015F5
:102A4000B1E15B48007870B3594800782D282BD04D
:102A500057480078A0F130055548407800B35448F5
:102A6000407805EB850100EB4100A0F130055048AE
:102A7000807890B14E488078A0F130064C48C078FC
:102A800040B14B48C07806EB860100EB4100A0F155
:102A900030060BE04FF0010908E04FF0010905E0B6
:102AA0004FF0010902E0FFE74FF001093B2E02DD84
:102AB0004FF0010903E0C5EB051006EB800572E15C
:102AC0003B4800782D2802D14FF00108012419E07D
:102AD0003748005D2C2801D1012711E047B1344867
:102AE000005D06EB860100EB4100A0F1300607E037
:102AF0002F48005D05EB850100EB4100A0F130059A
:102B0000601CC4B22A48005D08B1082CE0DB092E25
:102B100002DD4FF0010922E0B8F1010F06D105EB0B
:102B2000850006EB4000C0F52F7505E005EB85003C
:102B300006EB400000F52F7540F27B1006F094F88C
:102B400068B1A5F57F7000EBC00101EB00102D21ED
:102B500001EB40005A2190FBF1F000F52F7522E1C6
:102B6000134800782D2802D14FF00108012410E00D
:102B70000F48005D2C2802D14FF0010909E00C48F4
:102B8000005D05EB850100EB4100A0F13005601C04
:102B9000C4B20748005D08B1082CE9DBB8F1010FA9
:102BA00002D1C5F52F7501E005F52F75FBE000009A
:102BB00041010020582C0020000300209948007893
:102BC0002D2802D14FF001091FE019E09548005D62
:102BD0002C2801D1012711E047B19248005D06EB96
:102BE000860100EB4100A0F1300607E08D48005D52
:102BF00005EB850100EB4100A0F13005601CC4B27B
:102C00008848005D08B1082CE0DB092E02DD4FF09A
:102C1000010912E005EB850006EB400540F27B1050
:102C200006F022F848B105EBC50000EB05102D2198
:102C300001EB40005A2190FBF1F5B4E079480078AF
:102C40002D2802D14FF00108012419E07548005DDC
:102C50002C2801D1012711E047B17248005D06EB35
:102C6000860100EB4100A0F1300607E06D48005DF1
:102C700005EB850100EB4100A0F13005601CC4B2FA
:102C80006848005D08B1082CE0DB092E02DD4FF03A
:102C900001090FE0B8F1010F06D105EB850006EB45
:102CA0004000C0F52F7505E005EB850006EB400000
:102CB00000F52F7577E05B4800782D2802D14FF0A2
:102CC000010946E0574841780078303800EB800031
:102CD00001EB4000A0F130055248C17880783038CF
:102CE00000EB800001EB4000A0F130060D2E26D253
:102CF000DFE806F0250714081B091C0A0B1D0C1E33
:102D00000D0000BF00BF00BF00BF00BF00BF012D0E
:102D100001DB1F2D01DD4FF0010913E0012D01DB67
:102D20001C2D01DD4FF001090CE000BF00BF00BF0A
:102D3000012D01DB1E2D01DD4FF0010902E04FF0F6
:102D4000010900BF00BF06EBC60000EB061005EB53
:102D5000800528E0334800782D2802D14FF0010982
:102D600020E0304800783038642148432D494978C4
:102D7000303901EB810100EB41002A498978084490
:102D8000A0F1300527480179C078303800EB800089
:102D900001EB4000A0F1300605EB4500C0EBC5108B
:102DA00006EBC00500BF00BFB9F1000F36D108F037
:102DB00047FD1D4901EB0010D0F800B0584603F064
:102DC0008FF8824603F05CF8A8420EDC08F038FD6C
:102DD000154901EB0010D0F800B0584603F080F818
:102DE000824603F043F8A84202DA4FF0010915E0E9
:102DF00008F026FD0C4901EB001001222946D0F80D
:102E000000A0504608F002F908F01AFD064901EB4F
:102E10000010006810B9284607F004FA4846BDE8DB
:102E2000F09F000041010020582C002030B5002404
:102E3000002351E0184603F015FF01284AD1284825
:102E40000068CD214843274901EB8000143000EB96
:102E500003100568244800EB041005602048006852
:102E6000CD2148431F4901EB8000143000EB0310D3
:102E700040681D4901EB0411486019480068CD21E4
:102E80004843184901EB8000143000EB03108068C0
:102E9000154901EB0411886011480068CD214843B1
:102EA000104901EB8000143000EB0310C0680E499C
:102EB00001EB0411C8600C4800EB04100068401CD2
:102EC00030B932230121601E074A02EB00108160F5
:102ED000601CC4B2581CC3B2322BABDB30BD000047
:102EE000B80200202C5A0208582C002070B5064663
:102EF0000C46154600200C490860012006F08AFEA9
:102F0000304606F0DFFE2C2006F084FE204606F058
:102F1000D9FE2C2006F07EFE284606F0D3FE0220C5
:102F200006F078FE70BD00000001002010B50320FF
:102F300006F070FE0548006806F050FF042006F019
:102F400069FE00200249087010BD00000001002049
:102F50000C010020704770477047704770477047FA
:102F6000704770477047704770470029016802D06A
:102F700041F0010101E021F0010101607047000012
:102F800010B5114800F028F81048114908601148A0
:102F90004860002088600320C8600020086180200D
:102FA0004861400088618000C861202008620002FA
:102FB000486200208862044800F07AF80121024843
:102FC000FFF7D3FF10BD0000080002404C24014071
:102FD000B80D00203C0D0020016821F001010160C6
:102FE0000021016041608160C1602D4B2C49C21AF3
:102FF0008039984243D018DC2A4BA0EB0302984258
:1030000035D00ADC284A801829D014282BD028284B
:1030100024D1486840F4706034E0142A2BD0282A68
:103020001CD1486840F470002CE02048B2F56C7F59
:103030002ED009DCB2F5627F26D0B2F5677F0DD1C4
:10304000016841F0F00108E0B2F5717F24D0B2F5DB
:10305000767F03D1016841F47021016070474868B0
:1030600040F00F000EE0486840F0F0000AE04868C9
:1030700040F4704006E0486840F4702002E0486880
:1030800040F0706048607047016841F00F01E4E76C
:10309000016841F47061E0E7016841F47041DCE7E8
:1030A0008000024044000240F8FFFDBF04040240DB
:1030B00030B5036847F6F07293430C6A8A6822437E
:1030C000D1E904452C4322438C692243CC69224335
:1030D0004C6A22438C6A22431A430260CA684260E7
:1030E0000A6882604968C16030BD7047002000E016
:1030F000401C41F288318842FADB7047002000E032
:10310000401CB0F57A7FFBDB70470000F8B5002467
:103110004748007850B104F065FA0021084603F0F2
:1031200013FA0122A521002004F0FEF900204149F4
:10313000086065E0404800683E490968084400EBC3
:1031400040003E4901EB8000806808B9012457E047
:1031500038480168891C052003F0F6F934480078E6
:1031600068B30120334D00902D68354E3668B54266
:1031700001D1012500E000252B462F4D2D682D4E55
:103180003668354405EB45052C4E06EB8505AA68E7
:10319000294D2D68274E3668354405EB4505274EE9
:1031A00006EB85056968244D2D68224E3668354446
:1031B00005EB4505214E56F8250007F0D3FE1D4AC4
:1031C00012681F4B1B689A4201D1012200E00022C5
:1031D0001146194A1268174B1B681A4402EB420247
:1031E000164B03EB8202906803F098FE11480068CA
:1031F000401C1049086008460068052800DB0124CF
:10320000002C97D00A48007868B10A48006850B985
:10321000012C08D104210F2003F096F90022A621E9
:10322000104607F0EFFF002001490870F8BD0000CC
:103230003F0100200C03002008030020100C002098
:103240003001002038B53E480078002877D00020B3
:103250003B49087001222C2104F05AFA0221002077
:1032600003F072F90020374B00901B68364C24683D
:10327000234403EB4303354C04EB83039A68314B3F
:103280001B68314C2468234403EB43032F4C04EBAD
:10329000830359682B4B1B682B4C2468234403EB96
:1032A00043032A4C54F82300002307F05BFE04215B
:1032B000084603F049F90022C221104607F0A2FF98
:1032C0000521042003F040F90022C121104607F037
:1032D00099FF0621022003F037F900228D210120F9
:1032E00005F0B4F80621122003F02EF900228E21F9
:1032F000012005F0ABF80621222003F025F9002279
:103300008F21012005F0A2F80621482003F01CF9C6
:1033100000228A21012005F099F80621582003F0A7
:1033200013F900228B21012005F090F80621682076
:1033300003F00AF900228C21012005F087F838BD3E
:103340003F0100200803002030010020100C002065
:103350002DE9F041FE48056840F2831005F084FC39
:1033600004464FF4C17005F07FFCFA490860022C56
:1033700015DB0120F8490860F8490860F849086041
:10338000F8490860F8490860F8490860F849086099
:10339000F8490860F8490860F849086014E000201E
:1033A000ED490860ED490860ED490860ED490860A5
:1033B000ED490860ED490860ED490860ED49086095
:1033C000ED490860ED490860032C15DB0120EC494C
:1033D0000860EC490860EC490860EC490860EC4979
:1033E0000860EC490860EC490860EC490860EC4969
:1033F0000860EC49086014E00020E1490860E149F8
:103400000860E1490860E1490860E1490860E14974
:103410000860E1490860E1490860E1490860E14964
:103420000860042C15DB0120DF490860DF490860D3
:10343000DF490860DF490860DF490860DF4908604C
:10344000DF490860DF490860DF490860DF4908603C
:1034500014E00020D4490860D4490860D4490860C9
:10346000D4490860D4490860D4490860D449086048
:10347000D4490860D4490860D4490860052C15DB9C
:103480000120D3490860D3490860D3490860D34973
:103490000860D3490860D3490860D3490860D3491C
:1034A0000860D3490860D349086014E00020C84987
:1034B0000860C8490860C8490860C8490860C84928
:1034C0000860C8490860C8490860C8490860C84918
:1034D0000860C8490860062C15DB0120C649086051
:1034E000C6490860C6490860C6490860C649086000
:1034F000C6490860C6490860C6490860C6490860F0
:10350000C649086014E00020BB490860BB49086058
:10351000BB490860BB490860BB490860BB490860FB
:10352000BB490860BB490860BB490860BB490860EB
:103530004FF4BD7005F098FB0446022C03DB01201C
:10354000B749086002E00020B5490860032C03DB9E
:103550000120B449086002E00020B2490860042C50
:1035600003DB0120B049086002E00020AE4908609A
:10357000052C03DB0120AD49086002E00020AB49C7
:103580000860062C03DB0120A949086002E0002046
:10359000A7490860072C03DB0120A649086002E068
:1035A0000020A4490860082C03DB0120A249086020
:1035B00002E00020A0490860092C03DB01209F499C
:1035C000086002E000209D4908600A2C03DB01200E
:1035D0009B49086002E00020994908606C2005F0D2
:1035E00043FB012806D0022817D003281ED0052847
:1035F00040D12FE00120934908600020564908601F
:103600005F49086068490860714908607A49086044
:103610008D4908608D49086034E0012089490860BF
:10362000894908600020894908602BE0012085490C
:103630000860002048490860514908605A490860FC
:10364000634908606C4908607F49086001207F4930
:10365000086017E000207B4908603F49086048493E
:103660000860514908605A49086063490860774911
:10367000086007E0012073490860744908607249D6
:10368000086000BF00BF872005F0EEFA012806D0D1
:10369000022817D003281ED0052840D12FE0012092
:1036A0006B49086000202D490860364908603F4991
:1036B00008604849086051490860664908606649E1
:1036C000086034E001206249086062490860002017
:1036D000614908602BE001205D49086000201E4917
:1036E0000860274908603049086039490860424944
:1036F00008605849086001205749086017E0002019
:1037000053490860154908601E4908602749086048
:1037100030490860394908604F49086007E00120D6
:103720004B4908604B4908604B49086000BF00BF27
:10373000A22005F099FA012806D0022805D0032816
:1037400004D0052803D1B9E088E09AE0A2E0C5E002
:10375000D00200204C010020540100206C01002008
:10376000840100209C010020B4010020CC01002035
:10377000E4010020FC010020140200202C020020A3
:10378000580100207001002088010020A0010020C5
:10379000B8010020D0010020E80100200002002034
:1037A00018020020300200205C010020740100207B
:1037B0008C010020A4010020BC010020D4010020C5
:1037C000EC010020040200201C0200203402002032
:1037D000600100207801002090010020A801002055
:1037E000C0010020D8010020F001002008020020C4
:1037F0002002002038020020640100207C0100200B
:1038000094010020AC010020C4010020DC01002054
:10381000F40100200C020020240200203C020020C1
:10382000680200206C020020700200207402002058
:10383000780200207C020020800200208402002008
:103840008802002050010020400200208C0200204D
:103850006801002044020020900200200120FB4962
:1038600008600020FA490860FA490860FA490860CF
:10387000FA490860FA490860FA490860FA4908609C
:1038800034E00120F1490860F64908600020F6495B
:1038900008602BE00120ED4908600020EC49086039
:1038A000EC490860EC490860EC490860EC490860A4
:1038B000EC4908600120EC49086017E00020E3496A
:1038C0000860E3490860E3490860E3490860E349A8
:1038D0000860E3490860E449086007E00120DB492B
:1038E0000860E0490860E049086000BF00BFBD20F3
:1038F00005F0BAF9012806D0022817D003281ED0F7
:10390000052840D12FE00120D84908600020D8497F
:103910000860D8490860D8490860D8490860D84983
:103920000860D8490860D849086034E00120CF49D0
:103930000860D44908600020D34908602BE00120CA
:10394000CA4908600020CA490860CA490860CA49D3
:103950000860CA490860CA490860CA49086001206D
:10396000C949086017E00020C0490860C0490860E4
:10397000C0490860C0490860C0490860C049086083
:10398000C149086007E00120B8490860BD490860E6
:10399000BD49086000BF00BFD82005F065F90128C7
:1039A00006D0022817D003281ED0052840D12FE0CA
:1039B0000120B64908600020B5490860B549086093
:1039C000B5490860B5490860B5490860B54908605F
:1039D000B549086034E00120AC490860B14908608D
:1039E0000020B14908602BE00120A84908600020B0
:1039F000A7490860A7490860A7490860A749086067
:103A0000A7490860A74908600120A749086017E096
:103A100000209E4908609E4908609E4908609E49B2
:103A200008609E4908609E4908609F49086007E059
:103A30000120964908609B4908609B49086000BFC7
:103A400000BFF32005F010F9012806D0022817D096
:103A500003281ED0052840D12FE00120934908609B
:103A6000002093490860934908609349086093498E
:103A7000086093490860934908609349086034E0FE
:103A800001208A4908608F49086000208E4908603B
:103A90002BE00120854908600020854908608549A0
:103AA000086085490860854908608549086085493E
:103AB000086001208449086017E000207B49086005
:103AC0007B4908607B4908607B4908607B49086046
:103AD0007B4908607C49086007E001207349086061
:103AE000784908607849086000BF00BF4FF48770CC
:103AF00005F0BAF8012806D002280DD0032814D00A
:103B0000052836D125E00120704908600020704961
:103B100008607049086034E001206C4908606C4915
:103B2000086000206B4908602BE0012067490860AD
:103B30000020694908606949086069490860694965
:103B400008606949086062490860012061490860AD
:103B500017E000205D4908605F4908605F49086020
:103B60005F4908605F4908605F490860594908601B
:103B700007E001205549086055490860554908602B
:103B800000BF00BF40F2291005F06EF8012806D0F2
:103B9000022817D003281ED0052840D12FE001208D
:103BA0005249086000205249086052490860524951
:103BB00008605249086052490860524908605249F9
:103BC000086034E00120494908604E49086000203F
:103BD0004D4908602BE00120444908600020444919
:103BE0000860444908604449086044490860444901
:103BF00008604449086001204349086017E000203C
:103C00003A4908603A4908603A4908603A49086008
:103C10003A4908603A4908603B49086007E00120DA
:103C200032490860374908603749086000BF00BF63
:103C30004FF4A27005F018F8012867D002287BD055
:103C4000032877D0052876D193E05FE0800100203B
:103C500084010020880100208C01002090010020B8
:103C600094010020480200209402002098010020C6
:103C70009C010020A0010020A4010020A801002038
:103C8000AC0100204C02002098020020B00100206E
:103C9000B4010020B8010020BC010020C0010020B8
:103CA000C4010020500200209C020020C801002016
:103CB000CC010020D0010020D4010020D801002038
:103CC000DC01002054020020A0020020E0010020BE
:103CD00058020020A4020020E4010020E801002096
:103CE000EC010020F0010020F4010020F801002088
:103CF000FC01002000020020040200200802002035
:103D00000C0200205C020020A80200200120F949DA
:103D100008600020F8490860F8490860F849086020
:103D2000F8490860F8490860F8490860F8490860EF
:103D300037E001E009E02CE00120EE490860F3499A
:103D400008600020F24908602BE00120E949086082
:103D50000020E9490860E9490860E9490860E94943
:103D60000860E9490860E94908600120E8490860FD
:103D700017E00020DF490860DF490860DF4908607C
:103D8000DF490860DF490860DF490860E0490860F2
:103D900007E00120D7490860DC490860DC49086079
:103DA00000BF00BF40F25F1004F05EFF012806D0A4
:103DB000022817D003281ED0052840D12FE001206B
:103DC000D44908600020D4490860D4490860D44927
:103DD0000860D4490860D4490860D4490860D449CF
:103DE000086034E00120CB490860D0490860002019
:103DF000CF4908602BE00120C64908600020C64971
:103E00000860C6490860C6490860C6490860C649D6
:103E10000860C64908600120C549086017E0002015
:103E2000BC490860BC490860BC490860BC490860DE
:103E3000BC490860BC490860BD49086007E0012032
:103E4000B4490860B9490860B949086000BF00BFBB
:103E5000B84800681D2872D2DFE810F01D00390252
:103E600043027100B70222035003C703F2031D048B
:103E70007100710071007100710071007100ED013D
:103E80001F02EC007100710071007100700281006E
:103E90008B0025039C034FF41670A749086000208F
:103EA000A6490870A649087003F030F9472847D0A2
:103EB00006DC1B2838D01E2848D02E284DD11AE009
:103EC0004D2807D0872825D08D2846D10120994933
:103ED000086042E0672004F0C7FE0446601C044608
:103EE000032800DD00242146672007F07BF801202D
:103EF0009449086031E040F27B1004F0B5FEC0F157
:103F00000106314640F27B1007F06CF801208D4924
:103F1000086022E000208C49086013208549086071
:103F200001208849086018E0002088490860884915
:103F300008608849086011207E4908600DE043E26E
:103F40000020854908604FF47A7506E01320814906
:103F5000086019207749086000BF00BFC6E301234D
:103F60000022AC21AB2000F0F5FB1A20714908605B
:103F7000BCE304F0C5FE0746172F08D0472F02D038
:103F8000872F50D100BF00206A49086050E0FEF73B
:103F900001FC0646012E42DB4FF4BD7004F064FEC6
:103FA000B0423CDB0B2E2FD2DFE806F02E060A0EC5
:103FB00012161A1E22262A0005206349086023E0F3
:103FC0000C20614908601FE013205F4908601BE076
:103FD0001A205D49086017E021205B49086013E062
:103FE0002820594908600FE02F20574908600BE04E
:103FF00036205549086007E03D205349086003E03A
:1040000044205149086000BF00BF002051490860AA
:1040100004204849086001204A49086002E019204C
:104020004449086004E00021384602F075FC00BFF6
:1040300000BF5BE3002000F0CDFD04F061FE074609
:10404000472F0AD004DC172F11D02D2F09D10AE0F9
:10405000872F03D08D2F04D104E000BF0020354905
:104060000860E6E000BF384606F066FEE1E03B4847
:104070000078374909780844C6B20C2E12D2DFE81E
:1040800006F006121F2C6F7B8895A2AFBCC90020DA
:104090002E4908602E49086013202E49086011201F
:1040A00024490860C3E003202749086013202949F8
:1040B000086004201F490860012022490860B6E01A
:1040C000052021490860132022490860042019496D
:1040D000086001201B490860A9E00C201A4908600B
:1040E00013201C490860042012490860012015496A
:1040F00008609CE01002002014020020180200203A
:104100001C02002020020020240200206002002067
:10411000AC020020280200202C02002030020020E7
:1041200034020020380200203C02002064020020FB
:10413000B0020020D0020020280300203E01002011
:104140003C010020E8020020B80200200803002003
:1041500030010020D8020020C0020020BC02002054
:104160001320F9490860F94908600420F8490860FB
:104170000120F84908605AE01A20F349086013202A
:10418000F24908600420F24908600120F149086002
:104190004DE02120EC4908601320EC490860042020
:1041A000EB4908600120EB49086040E02820E6491F
:1041B00008601320E54908600420E54908600120F3
:1041C000E449086033E02F20DF4908601320DF490D
:1041D00008600420DE4908600120DE49086026E00E
:1041E0003620D94908601320D84908600420D849EE
:1041F00008600120D749086019E03D20D2490860D5
:104200001320D24908600420D14908600120D14917
:1042100008600CE04420CC4908601320CB490860BA
:104220000420CB4908600120CA49086000BF00BFD4
:1042300000BF00BF5AE2FEF769FF04F061FD4728A6
:1042400010D004DC172816D02D2824D104E08728AC
:104250000DD08D281FD102E0FDF72EFA1BE0FDF7EF
:1042600057FA18E0B9480068B949086013E000201F
:10427000B74908600FE0B8480068B84909680844C1
:1042800000EB4000B64901EB8000806810B11220BD
:10429000AF49086000BF00BF28E2FEF7D3FF04F07B
:1042A0002FFD172807D047280BD087280DD10020D5
:1042B000A749086009E006F0EDFD1120A449086057
:1042C00003E01120A249086000BF00BF0EE20123F5
:1042D00000221C211D2000F03DFA02209C490860AC
:1042E00004E204F00DFD0746172F08D0472F02D037
:1042F000872F1CD100BF0020954908601CE0FEF705
:1043000049FA064640F60A30864202D0954886426F
:1043100009D101208C49086018208D4908600120CE
:104320009149087002E000208949086004E00121F9
:10433000384602F0F1FA00BF00BFD7E1012000F0DB
:1043400049FC04F0DDFC0746002088490870472F2F
:104350000AD004DC172F13D02D2F34D10CE0872F77
:1043600003D08D2F2FD106E000BF00207F490870B9
:104370007749086027E000BF384606F0DDFC22E000
:104380007B480078754909780844C6B216B1012EF9
:1043900017D109E002206C49086018206B490860B9
:1043A00004206B4908600CE04B2067490860182026
:1043B0006649086004206649086001206B4908705E
:1043C00000BF00BF00BF00BF90E15F48006800F081
:1043D00021FB04F095FC06464B2E4CD006DC172E34
:1043E00018D02D2E09D0472E58D10AE04E2E2ED0AF
:1043F000872E0BD08D2E51D100BF304606F09CFC8D
:104400004CE0524800685249086047E0002050499B
:10441000086043E007F014FA564901EB0010D0F8A9
:104420000080404601F05CFD074602F049FC68B19F
:104430000420514908600520454908604748006844
:104440004E4908604A4800684D49086026E000BFB0
:104450003D480068CD2148434A4901EB800040684F
:10446000394908600846006802F054FC0028EFD083
:104470004FF47A7512E000BF33480068CD214843FD
:10448000404951F82000304908600846006802F0B1
:1044900041FC0028F0D04FF47A7500BF00BF25E141
:1044A00002F09EF822E101F04FF9172804D04728C6
:1044B00003D0872820D11BE000BF2F480068244983
:1044C00008602D4805682D480068244908602C487C
:1044D0000068274908601C480068CD225043294ADB
:1044E00002EB800001228168002003F011F903E053
:1044F00000201749086000BF00BFF7E001F044F852
:10450000172804D0472803D0872841D13CE000BFBA
:10451000194800680E490860174805681748006880
:104520000E4908601648006811490860064800688E
:10453000CD225043134A02EB800001228168002003
:1045400003F0E6F824E00000B8020020D8020020C2
:10455000D0020020E80200200803002030010020E3
:10456000100C0020C6D53C003E0100203C0100207C
:10457000BC020020582C0020D40200203003002070
:10458000340300202C5A020800206649086000BF4E
:1045900000BFABE000F020F9172804D0472803D073
:1045A000872820D11BE000BF5F4800685D49086094
:1045B0005D4805685D4800685D4908605D480068C1
:1045C0005D4908605D480068CD2250435C4A02EBBB
:1045D000800001228168002003F09AF803E00020A7
:1045E0005049086000BF00BF80E000F0D9FD1728E7
:1045F00004D0472803D0872820D11BE000BF4A48B9
:1046000000684849086048480568484800684849C3
:104610000860484800684849086048480068CD225A
:104620005043474A02EB800001228168002003F0DA
:104630006FF803E000203B49086000BF00BF55E071
:1046400000F0AEFB172804D0472803D0872820D1DC
:104650001BE000BF344800683249086032480568F2
:1046600032480068324908603248006832490860C0
:1046700032480068CD225043314A02EB80000122CB
:104680008168002003F044F803E000202549086019
:1046900000BF00BF2AE001F04FF9172804D04728D7
:1046A00003D0872820D11BE000BF1F4800681D49A8
:1046B00008601D4805681D4800681D4908601D48C0
:1046C00000681D4908601D480068CD2250431C4AFF
:1046D00002EB800001228168002003F019F803E05A
:1046E00000201049086000BF00BF00BF00BF154890
:1046F000006858B900200B49086013490860012080
:10470000124908704FF416700E4908600548006899
:10471000854205D000200E49086001200B49087031
:10472000BDE8F081D0020020D40200203003002038
:104730003001002034030020BC020020B802002019
:104740002C5A020828030020C00200203F0100204C
:10475000DC020020F8B504460F4615461E4607F059
:1047600031FA01222146002002F0D2FF0321042069
:1047700001F0EAFE00223946104606F043FD3EB93C
:10478000062000231A4629460090184603F0E2FD51
:104790000421084601F0D8FE00220821022003F07F
:1047A00055FE00220921022003F050FE00220921BB
:1047B000022003F04BFE00220921022003F046FEF6
:1047C00000220B21022003F041FE04F071FD0521BF
:1047D000082001F0B9FEF8BD70B57F480078C1002F
:1047E0004FF07F40C8407D4908607B480078C10099
:1047F0004FF0807008417A49086077480078C1001E
:104800004FF0005008417749086073480078C100B4
:104810004FF0FE4008417449086004F071FA044604
:104820000020724908706C480078042874DA7048D7
:104830000068000E6F4908706D480068000C6E49F2
:1048400008706B480088000A6C4908706848007856
:104850006B49087060480078C0EB00100830694967
:10486000086008206849087068480068B0F5FA7F59
:1048700007DA0846007863490968884201D10120B7
:1048800000E0002002465B480178012003F0DEFDD5
:104890005D480078001D5C4908705C480068B0F510
:1048A000FA7F07DA0846007856490968884201D13C
:1048B000012000E0002002464F480178012003F06B
:1048C000C5FD51480078001D4F4908704F480068E9
:1048D000B0F5FA7F07DA084600784A490968884245
:1048E00001D1012000E00020024644480178012067
:1048F00003F0ACFD44480078001D4349087043486C
:104900000068B0F5FA7F08DA084600783D49096882
:10491000884202D1012001E00AE000200246384826
:104920000178012003F092FD36480078364908707E
:104930004B2C33D004DC172C07D02D2C49D137E079
:104940004E2C21D08D2C44D10DE0172406F078FF99
:104950002F4901EB0010012205682548016828460F
:1049600006F054FB35E0224800681C4909680840FD
:104970001D490968884206DA1D4800681849096817
:1049800008441B49086024E013480078002804DD2F
:1049900011480078401E104908701AE00E4800784F
:1049A000032804DA0C480078401C0B49087010E01A
:1049B0000F4800680949096808400A49096888429F
:1049C00006DD0B48006806490968401A0849086076
:1049D00000BF00BF204670BD3D0100201403002031
:1049E000180300201C030020200300203F010020AA
:1049F000F802002010030020110300201203002001
:104A0000130300202403002035010020140000209F
:104A1000582C00202DE9F041074600266448076025
:104A20006448007890B1FEF701FA61480068CD2231
:104A30005043614A02EB800001228168002002F0AD
:104A400067FE00205D4908605D4908600020594903
:104A500008705C480068002877D000205949086039
:104A600001213A2001F070FD5448006850B1002245
:104A70008721104603F0EAFC00228821104603F04B
:104A8000E5FC09E000222021104603F0DFFC0022B3
:104A90002021104603F0DAFC07213A2001F054FDF2
:104AA00000E0761C484800EB061080680028F8D02B
:104AB00042480068001DB0420CD0052E0ADB0022DF
:104AC0008521104603F0C2FC00228621104603F027
:104AD000BDFC09E000228921104603F0B7FC00224A
:104AE0008921104603F0B2FC02203849087033488F
:104AF0000578002457E0344800EB05100068401C9E
:104B000000284DD00120324908702D4800688442A9
:104B100001D1012000E0002002462021002003F006
:104B200095FC04202A49087025480068844201D178
:104B3000012000E000200146284602F0E1FC204868
:104B40000068844202D1012001E02EE000200346EB
:104B500001222946002002F017FF72201C4908702C
:104B600017480068844201D1012000E0002002467D
:104B70002021002003F06AFC11480068844201D122
:104B8000012000E0002002462946002002F01AFC25
:104B9000681CC5B20D480078401C0C49087000E044
:104BA0000524601CC4B2052CA5DBBDE8F081000023
:104BB000B80200203F0100202C5A0208BC0200204D
:104BC00030010020E8020020582C0020360100208F
:104BD0003501002070B50646002568480660684823
:104BE0000078A0B1FEF722F964480068CD22504356
:104BF000644A02EB800001228168002002F088FDF7
:104C000000205F490870604908606049086060489A
:104C10000068002879D000205D49086001213A2011
:104C200001F092FC5848006850B1002287211046DC
:104C300003F00CFC00228821104603F007FC09E079
:104C400000222021104603F001FC00222021104602
:104C500003F0FCFB07213A2001F076FC00E06D1C1C
:104C60004C4800EB051080680028F8D046480068E2
:104C7000001DA8420CD0052D0ADB0022852110461C
:104C800003F0E4FB00228621104603F0DFFB09E07D
:104C900000228921104603F0D9FB00228921104609
:104CA00003F0D4FB02203C490870002463E036483E
:104CB00000682044374901EB00100068401C0028C0
:104CC00056D001203549087030480068844201D12F
:104CD000012000E0002002462021002003F0B6FB66
:104CE0002A480068844201D1012000E000200246E9
:104CF0002021002003F0AAFB032028490870234844
:104D00000068844202D1012001E036E00020024622
:104D10001D48006820441F4B03EB00104168002031
:104D200006F070FA0BE019480068844201D10120B6
:104D300000E0002002462021002003F087FB1748F6
:104D400000787828EFDB7720144908700F48006856
:104D5000844201D1012000E00020024620210020F1
:104D600003F074FB0C480078401C0B49087000E00D
:104D70000524601CC4B2052C99DB70BDB80200206C
:104D80003F0100202C5A0208BC0200203001002004
:104D9000E8020020582C00203601002035010020B8
:104DA00070B503F0ADFF04460020F8490870F848DC
:104DB0000078052814DAF7480068B0F5FA7F05DABC
:104DC00000225F21012003F041FB04E000222021AA
:104DD000012003F03BFBF04800780B38EE490870E7
:104DE0004B2C7DD00EDC2B2C7BD006DC172C16D068
:104DF0001D2C19D0272C16D153E12D2C72D02E2C1E
:104E0000F9D1F0E08B2C72D004DC4D2C6CD04E2C00
:104E1000F1D18BE08D2C45D08E2CECD123E0FDF729
:104E2000CFFC00B10224ADE1D9480078052819DA99
:104E30003021D74802780078401CD54B1870D748ED
:104E400081540022012003F001FBD3480078001DAB
:104E5000D1490870CE480078032803D1084600786D
:104E60000F3008708EE1CA480078052819DA312120
:104E7000C74802780078401CC54B1870C748815459
:104E80000022012003F0E2FAC3480078001DC24965
:104E90000870BF480078032803D1084600780F3017
:104EA00008706FE1BA48007805281FDA3221B84847
:104EB00002780078401CB64B1870B8488154002224
:104EC000012003F0C3FAB4480078001DB24908700D
:104ED000AF480078032809D1084600780F3004E075
:104EE00062E0BEE09EE002E03FE008704AE1A848D0
:104EF0000078052819DA3321A54802780078401C8B
:104F0000A34B1870A54881540022012003F09EFA9B
:104F1000A1480078001DA04908709D48007803282A
:104F200003D1084600780F3008702BE198480078CC
:104F3000052819DA3421964802780078401C944BF1
:104F40001870964881540022012003F07FFA92489D
:104F50000078001D904908708D480078032803D11F
:104F6000084600780F3008700CE189480078052861
:104F700019DA3521864802780078401C844B187075
:104F8000864881540022012003F060FA82480078AC
:104F9000001D814908707E480078032803D1084627
:104FA00000780F300870EDE079480078052819DAAC
:104FB0003621774802780078401C754B1870774886
:104FC00081540022012003F041FA73480078001D4B
:104FD000714908706E480078032803D108460078AC
:104FE0000F300870CEE06A480078052819DA3721BA
:104FF000674802780078401C654B187067488154F8
:105000000022012003F022FA63480078001D624963
:1050100008705F480078032803D1084600780F30F5
:105020000870AFE05A480078052819DA3821584846
:1050300002780078401C564B187058488154002262
:10504000012003F003FA54480078001D524908700B
:105050004F480078032803D1084600780F300870C5
:1050600090E04B48007805281ADA39224848017840
:105070000078401C464B18704848425400223921A1
:10508000012003F0E3F944480078001D424908700C
:105090003F480078032803D1084600780F30087095
:1050A00070E03B480578062D6AD2DFE805F06953C9
:1050B0003D27110336480078401E3549087000200E
:1050C0003649334A1278885453203349087057E0E0
:1050D0002F480078401E2E49087000202F492C4A86
:1050E0001278885453202C4908700022892101200D
:1050F00003F0ACF944202849087041E024480078C6
:10510000401E2349087000202449214A12788854FF
:1051100044202149087000228921012003F096F9DA
:1051200026201D4908702BE019480078401E1849B8
:10513000087000211948164A127881542620164911
:10514000087000228921012003F080F917201249FC
:10515000087015E00E480078401E0D4908700020C8
:105160000E490B4A1278885417200B490870002208
:105170008921012003F06AF908200749087000BF5F
:1051800000BF00BF00BF204670BD00003F010020EF
:105190003D010020140000203501002041010020C5
:1051A00070B503F0ADFD04460020F2490870F248E6
:1051B0000078082814DAF1480068B0F5FA7F05DABB
:1051C00000225F21012003F041F904E000222021A8
:1051D000012003F03BF9EA4800780B38E8490870F1
:1051E0004B2C7DD00EDC2B2C7BD006DC172C16D064
:1051F0001D2C19D0272C16D155E12D2C72D02E2C18
:10520000F9D1F2E08B2C72D004DC4D2C6CD04E2CFA
:10521000F1D18CE08D2C45D08E2CECD123E0FDF724
:10522000CFFA00B10224A1E1D3480078042819DAAA
:105230003021D14802780078401CCF4B1870D148FB
:1052400081540022012003F001F9CD480078001DAF
:10525000CB490870C8480078022803D10846007876
:105260000F30087082E1C4480078042819DA31212F
:10527000C14802780078401CBF4B1870C148815467
:105280000022012003F0E2F8BD480078001DBC496F
:105290000870B9480078022803D1084600780F301A
:1052A000087063E1B448007804281FDA3221B2485C
:1052B00002780078401CB04B1870B248815400222C
:1052C000012003F0C3F8AE480078001DAC49087017
:1052D000A9480078022809D1084600780F3004E078
:1052E00064E0C1E0A0E002E040E008703EE1A248D6
:1052F000007804281ADA33229F4801780078401C8D
:105300009D4B18709F48425400223321012003F026
:105310009DF89B480078001D9949087096480078D0
:10532000022803D1084600780F3008701EE1924829
:105330000078042819DA34218F4802780078401C5C
:105340008D4B18708F4881540022012003F07EF8A5
:105350008B480078001D8A49087087480078022829
:1053600003D1084600780F300870FFE082480078CB
:1053700004281ADA3522804801780078401C7E4BD8
:1053800018708048425400223521012003F05EF855
:105390007B480078001D7A49087077480078022819
:1053A00003D1084600780F300870DFE072480078BB
:1053B000042819DA3621704802780078401C6E4BB8
:1053C0001870704881540022012003F03FF86C48A7
:1053D0000078001D6A49087067480078022803D1E8
:1053E000084600780F300870C0E063480078042851
:1053F00019DA3721604802780078401C5E4B18703B
:10540000604881540022012003F020F85C480078B5
:10541000001D5B49087058480078022803D10846EF
:1054200000780F300870A1E05348007804281ADA99
:105430003822514801780078401C4F4B1870514871
:10544000425400223821012003F000F84C48007833
:10545000001D4B49087048480078022803D10846CF
:1054600000780F30087081E043480078042819DA8A
:105470003921414802780078401C3F4B1870414860
:1054800081540022012002F0E1FF3D480078001D18
:105490003B49087038480078022803D10846007854
:1054A0000F30087062E034480578012D46D0022D97
:1054B0002ED0032D16D0042D56D10078401E2E4933
:1054C000087000202F492C4A1278885453202C4908
:1054D000087000222021012002F0B8FF4420284952
:1054E000087041E024480078401E234908700020DD
:1054F0002449214A12788854442021490870002206
:105500008921012002F0A2FF35201D4908702BE0FF
:1055100019480078401E1849087000201949164A99
:1055200012788854352016490870002289210120FC
:1055300002F08CFF17201249087015E00E48007821
:10554000401E0D49087000210E480B4A1278815404
:1055500017200B49087000228921012002F076FFF4
:1055600008200749087000BF00BF00BF00BF2046E9
:1055700070BD00003F0100203D010020140000200C
:1055800035010020410100202DE9F0416A480078F2
:1055900080B101206949087000206749087006F051
:1055A0004FF9674901EB00100668304600F03AFFFA
:1055B0006449086003F0A4FB044606F041F9604921
:1055C00001EB00100768384600F08AFC064601F03F
:1055D00085FB05460521082000F0B6FF57480078F6
:1055E00000285CD0002055490870B5F5F04F35D043
:1055F0000ADCDDB1B5F5C04F10D0B5F5D04F1DD0E8
:10560000B5F5E04F4AD121E0B5F5504F2ED0B5F5B4
:10561000604F33D0B5F5983F40D137E000231A46AC
:1056200048480168012001F08EFD37E000231A464A
:1056300044480168012002F07BF82FE000231A465D
:1056400040480168012002F06DF927E000231A4666
:105650003C480168012001F0A6FD1FE000231A4626
:1056600038480168012002F0FDF817E000231A46CF
:1056700034480168012002F085F90FE000231A4642
:1056800030480168012002F04EF907E000231A4675
:105690002C480168012001F085FD00BF00BF172CD8
:1056A00038D02D2C04D0472C41D08D2C40D118E07F
:1056B00006F0C6F8224901EB00100768384600F0F2
:1056C0000FFC064600F0DCFB1E490968884204DA3C
:1056D0001C480068401E1B490860012017490870DB
:1056E00026E006F0ADF8164901EB001007683846D1
:1056F00000F0F6FB064600F0B9FB12490968884243
:1057000004DD10480068401C0E49086001200B4968
:1057100008700DE006F094F8094901EB0010012231
:10572000066808480168304605F070FC00E000BFDC
:1057300000BF2046BDE8F0813F010020FC020020B0
:10574000582C0020F802002070B57648007880B10F
:1057500001207549087000207249087006F070F841
:10576000724901EB00100568284600F05BFE7049A5
:10577000086003F0C5FA04460521082000F0E4FEA5
:105780006948007810B1002067490870172C73D061
:105790002D2C04D0472C70D08D2C55D155E0654868
:1057A000006830B101280AD002281ED003284AD14F
:1057B00030E001205E4908605B49087043E05C48C6
:1057C0000068042802D005280DD106E005205849BC
:1057D000086001205449087005E001205449086020
:1057E0005149087000BF00BF2DE0514800680228F1
:1057F00008D003280CD102204D49086001204A49F5
:10580000087005E001204A4908604749087000BF58
:1058100000BF18E006F014F8444901EB00100668D8
:10582000304600F05DFB054600F02AFB4049096860
:10583000884204DA3E480068401E3D490860012065
:105840003949087000BF00BF68E03A48006830B1CD
:1058500001280AD0022821D003284FD135E00120A9
:10586000334908603049087048E031480068012831
:1058700004D0052810D108E042E04EE005202C4974
:10588000086001202849087006E0042028490860C3
:1058900001202549087000BF00BF2FE024480068A0
:1058A000012802D002280ED106E00220204908601B
:1058B00001201D49087006E003201D4908600120F1
:1058C0001949087000BF00BF18E005F0B9FF17497B
:1058D00001EB00100668304600F002FB054600F0C0
:1058E000C5FA13490968884204DD11480068401C64
:1058F0000F49086001200C49087000BF00BF0DE08F
:1059000005F09EFF094901EB0010012205680848D7
:105910000168284605F07AFB00E000BF00BF204682
:1059200070BD00003F010020FC020020582C002028
:10593000F8020020EC02002010B50020B1490870E8
:10594000B1480078082814DAB0480068B0F5FA7F4A
:1059500005DA00225F21012002F078FD04E0002238
:105960002021012002F072FDA94800780B38A849D7
:10597000087003F0C5F904462E2C6ED010DC1E2CE6
:105980006CD006DC172C1AD01B2C68D01D2C1AD119
:105990001AE0272C76D02B2C75D02D2CF7D1ADE02A
:1059A0008B2C47D006DC4B2C6ED04D2C6ED04E2C61
:1059B000EDD155E08D2C2BD08E2CE8D116E0FCF7E4
:1059C000FFFE00B102241AE18F48007808280CDAA3
:1059D00030218D4802780078401C8B4B18708D4820
:1059E00081540022012002F031FD08E18648007850
:1059F00008280CDA3121844802780078401C824B58
:105A00001870844881540022012002F01FFDF6E046
:105A10007D48007808280CDA32217B48027800782B
:105A2000401C794B18707B4881540022012002F001
:105A30000DFDE4E07448007808280DDA332272483E
:105A400001780078401C704B187072484254002254
:105A50003321012002F0FAFCD1E03CE08AE071E061
:105A60006948007808280CDA342167480278007801
:105A7000401C654B1870674881540022012002F0D9
:105A8000E5FCBCE087E04BE013E0FFE75E48007810
:105A900008280DDA35225C4801780078401C5A4B02
:105AA00018705C48425400223521012002F0CEFCDF
:105AB000A5E05548007808280CDA362152480278CB
:105AC0000078401C504B187052488154002201202D
:105AD00002F0BCFC93E04C48007808280DDA37222D
:105AE000494801780078401C474B18704948425497
:105AF00000223721012002F0A9FC80E04248007812
:105B000008280CDA3821404802780078401C3E4BC7
:105B10001870404881540022012002F097FC6EE08A
:105B20003948007808280CDA39213748027800789B
:105B3000401C354B1870374881540022012002F078
:105B400085FC5CE030480078082812DA324800789A
:105B500078B92C222C4801780078401C2A4B187008
:105B60002C48425401202C49087000222E2102F0BA
:105B70006DFC44E02448007860B92D212248027869
:105B80000078401C204B18702248815400220120CC
:105B900002F05CFC33E01C48007800282EDD1A4837
:105BA0000078401E184908701A480978405C2C2873
:105BB00002D100201849087000201649124A1278B4
:105BC000885411480078072809DA00222021012092
:105BD00002F03CFC0E4800780B380D4908700C4868
:105BE00000780B380A49087000222021012002F0B9
:105BF0002DFC074800780B380549087000BF00BF2E
:105C0000204610BD3F0100203D010020140000206F
:105C100035010020410100204001002070477047FD
:105C200010B5022000F09CF8B8B102210B4800F03A
:105C30008EFB60B90A4800680A49884207DA0A48B8
:105C4000007820B906480068401C054908600A2011
:105C500005490870022000F07DF810BD00080140E1
:105C6000D003002040420F000000002010B50420A7
:105C700000F076F8B8B104210B4800F068FB60B979
:105C80000A4840680A49884207DA0A48007820B979
:105C900006484068401C054948600A2005490870CC
:105CA000042000F057F810BD00080140D003002088
:105CB00040420F00010000207047000010B5102086
:105CC00000F04EF8B8B110210B4800F040FB60B96D
:105CD0000A48C0680A49884207DA0A48007820B9A9
:105CE0000648C068401C0549C8600A20054908707C
:105CF000102000F02FF810BD00140140D003002048
:105D000040420F000300002010B5802000F028F86A
:105D1000B8B180210B4800F01AFB60B90A488068CE
:105D20000A49884207DA0A48007820B9064880689C
:105D3000401C054988600A2005490870802000F051
:105D400009F810BD00080140D003002040420F00B8
:105D5000020000200149086070470000140401405F
:105D6000064A014600201268044B0A4014331B689F
:105D70000B4202D0002A00D00120704700040140ED
:105D800030B583791949026853B30B6893430B60AC
:105D90000A1D13680468A343136002790A44136858
:105DA000046823431360114A083213680468A3434C
:105DB0001360131D1C680568AC431C604479102CEB
:105DC00005D021440A68006802430A6030BD1168AA
:105DD000046821431160196800680143196030BDEF
:105DE0000079084401689143016030BD000401401E
:105DF0007047000004490A6822F010020A600A682D
:105E000002430A60704700000020024004490A680B
:105E100002F038020A600A6802430A607047000014
:105E200000200240704710B5044640F27B1002F09B
:105E30001BFF08B9204610BDA4F52F70C0EB001061
:105E400000EB4000192101EB4000322190FBF1F002
:105E500000F57F70EFE700000146C1EBC100024A88
:105E600002EB80004069704738E901080146C1EB48
:105E7000C100024A02EB80000069704738E901085E
:105E80000146C1EBC100024A02EB8000C0687047C6
:105E900038E901080146C1EBC100024A52F820006E
:105EA0007047000038E9010810B50446002300E0FF
:105EB0005B1CC3EBC300094901EB80008068A04272
:105EC00007D0C3EBC30051F820004FF6FF718842A2
:105ED000EED11846FFF7DEFF10BD000038E90108DB
:105EE00070B504464FF0FF3625460648854206DA6F
:105EF00040F2391200212846FBF744FD06463046A1
:105F000070BD000078D4030008B50121480202F0FA
:105F100019FC0121084602F0FDFB0121084602F0B0
:105F200011FC0121042002F00DFC0121082002F0E7
:105F300009FC0121102002F005FC0121202002F0C3
:105F400001FC0121402002F0FDFB0121480402F088
:105F5000EDFB0121880402F0E9FB0121082000F09B
:105F6000CFF90121AE4800F0CBF98620ADF8000052
:105F700004208DF8030003208DF802006946A9482B
:105F800000F070F94FF40070ADF8000003208DF8B8
:105F9000020018208DF803006946A24800F062F95B
:105FA0004FF48060ADF8000004208DF803006946CE
:105FB0009C4800F057F90120ADF8000003208DF84F
:105FC000020004208DF803006946964800F04AF963
:105FD0002020ADF8000003208DF8020010208DF87D
:105FE000030069468F4800F03DF94FF4D050ADF8FA
:105FF000000003208DF8020010208DF80300694690
:10600000884800F02FF94FF47050ADF800001020D0
:106010008DF8030003208DF802006946824800F0E5
:1060200021F94020ADF8000003208DF80200142073
:106030008DF8030069467C4800F014F98220ADF821
:10604000000003208DF8020004208DF8030069464B
:10605000754800F007F90320ADF8000000208DF826
:1060600003006946704800F0FDF82020ADF80000FC
:1060700000208DF8030069466C4800F0F3F84FF4F7
:106080007070ADF8000010208DF803006946674875
:1060900000F0E8F81020ADF8000004208DF80300AF
:1060A0006946624800F0DEF84FF20F00ADF80000DC
:1060B00003208DF8020048208DF8030069465C48F3
:1060C00000F0D0F82020ADF8000003208DF8020089
:1060D00018208DF803006946554800F0C3F84020A9
:1060E000ADF8000003208DF8020004208DF80300B5
:1060F00069464F4800F0B6F84FF48070ADF80000E4
:1061000003208DF8020018208DF8030069464848E6
:1061100000F0A8F84FF40070ADF8000003208DF8EF
:10612000020004208DF803006946414800F09AF807
:106130004FF44960ADF8000003208DF802001020F4
:106140008DF8030069463A4800F08CF80120ADF85C
:10615000000014208DF8030003208DF8020069462A
:10616000344800F07FF88020ADF8000010208DF852
:10617000030003208DF8020069462E4800F072F8F3
:106180004FF47F40ADF8000003208DF80200282076
:106190008DF803006946274800F064F801210020CB
:1061A00000F04CF8022024490860002008710C20FF
:1061B0004871012088710846FFF7E2FD02210020A6
:1061C00000F03CF804201C490860002008710C20F5
:1061D0004871012088710846FFF7D2FD0721002091
:1061E00000F02CF8802014490860002008710C2071
:1061F0004871012088710846FFF7C2FD0421022082
:1062000000F01CF810200C490860002008710C20D8
:106210004871012088710846FFF7B2FD08BD0000F3
:106220003000140000080140000C01400010014043
:1062300000140140001801409800002010B58A07A2
:1062400021F003040649130F21440F228C689A4061
:1062500094438C608A68984002438A6010BD0000B5
:1062600000000140F0B5CB78002503F00F02DB06FB
:1062700001D58B781A430B884FF00F0E13F0FF0FE8
:106280004FF0010C19D004680E880CFA05F31E407B
:106290009E420ED1AF000EFA07F6B44302FA07F79A
:1062A000CE783C43282E00D14361CE78482E00D1D1
:1062B00003616D1C082DE7D304600B88FF2B1DD9EB
:1062C0004468002505F108060CFA06F30E881E4006
:1062D0009E420FD1AF000EFA07F624EA060602FA34
:1062E00007F43443CE78282E00D14361CE78482E6F
:1062F00000D103616D1C082DE4D34460F0BD0000A3
:10630000F0B5104D6B68440D260184B2C0F30157FF
:10631000B440C0F30342032F05D0C0020AD50320C6
:106320009040834307E0686823F0706220F070605B
:10633000686002E0A34343F0706201B122436A60E7
:10634000F0BD000000000140806880B27047024646
:10635000002092680A4200D00120704702460020C7
:10636000D2680A4200D00120704741617047016144
:106370007047C1607047000070B506463546472D2E
:1063800000DA47251A48854200DD0546D222002161
:10639000284602F0E7FE441E012C00DA0124601CAE
:1063A00000EB4000134951F8200004EB4401114A6E
:1063B00052F82110401A04EB440102EB81014968B4
:1063C000691A4843611C01EB410102EB81014968F4
:1063D00004EB4402074B03EB82025268891A90FBDC
:1063E000F1F004EB44011A4652F82110084470BD44
:1063F00054220E00900B020810B504460748844250
:1064000009DA2046FFF76CFDC0EBC000044901EB40
:106410008000806810BD0020FCE7000078D40300F5
:1064200038E9010870B504460E48844218DA20465F
:10643000FFF756FD054600F037FC30B12046FFF768
:10644000DBFF054602F0E0FC70BD2046FFF748FD8B
:10645000C0EBC000044901EB800040680068F3E72E
:106460000020F1E778D4030038E901080146002054
:10647000002201291BDB062919DC072911D2DFE8DC
:1064800001F0100406080A0C0E00012209E00222A5
:1064900007E0042205E0082203E0102201E02022A8
:1064A00000BF00BF024B1B68134003B901207047B7
:1064B0005800002002461146002900DA0021B1F5FB
:1064C000805F01DB40F6FF714FF47A704843C1F5FD
:1064D000805390FBF3F0704710B54FF4C17002F099
:1064E000C3FBB8B110480468B4F5967F03DB40F2F3
:1064F0001450844207DD0D48006820B901210020B6
:1065000003F022FE0EE00A4804600121002002F0A0
:106510004BFE07E04FF42F70054908600121002071
:1065200002F042FE10BD0000B00B0020B0000020C1
:1065300034000020014601F114006422504340F66B
:10654000FF7290FBF2F07047024B1970024B18700B
:1065500070470000360100203501002000BFFEE733
:10656000704770477047704710B501210148FFF729
:10657000FEFE10BD0018014002494CF6CC400860F8
:10658000704700000030004002494AF6AA20086027
:10659000704700000030004001494860704700002B
:1065A0000030004001498860704700000030004022
:1065B00001490860704700000030004010B545F206
:1065C0005550FFF7F5FF0520FFF7E6FF40F6C41032
:1065D000FFF7E8FFFFF7D8FFFFF7CEFF10BD000081
:1065E00070B5C6480078002843D0C5480068CD2261
:1065F0005043C44A02EB800001228168002001F070
:1066000087F803210220FFF79FFF02F051FE05F0FB
:1066100017F90446002100F073FF05F011F9C4B228
:10662000002301222146184601F0AEF905F008F9D1
:10663000C4B200222146104600F0C4FE04210846E0
:10664000FFF782FF00220821022001F0FFFE002256
:106650000921022001F0FAFE00220921022001F0A6
:10666000F5FE00220921022001F0F0FE0020A349DE
:10667000087005F0E5F8A44901EB0010056828460C
:10668000FFF72EFC044600F029FBC0F30A010029A5
:106690007ED1C0122A287BD2DFE800F01517181926
:1066A0007A7A7A7A7A517A7A1A1B1C1D1E7A7A249F
:1066B00050167A7A259126271F202122237A7A7A6A
:1066C0003C7A287A7AD900BF00BF00BF00BF00BF64
:1066D00000BF00BF00BF00BF00BF00BF00BF00BFC2
:1066E00000BF00BF00BF00BF00BF00BF00220A21E3
:1066F000022001F0ABFE05F0A3F8834901EB001086
:1067000004682046FFF78EFE804908600620804915
:106710000860F1E000220A21022001F097FE05F056
:106720008FF8794901EB001004682046FFF77AFEE4
:10673000764908601B2076490860DDE000BF002232
:106740000B21022001F082FE05210820FFF7FCFE4C
:1067500000228921012001F079FE6E480078001D99
:106760006C49087000228921012001F06FFE694800
:106770000078001D6749087000223A21012001F0CD
:1067800065FE64480078001D62490870002200E040
:10679000A5E08921012001F059FE5E480078001D26
:1067A0005C49087000228921012001F04FFE05217B
:1067B0000820FFF7C9FE0720554908609CE0002229
:1067C0000B21022001F042FE05210820FFF7BCFE4C
:1067D00000228921012001F039FE4E480078001D79
:1067E0004C49087000228921012001F02FFE494800
:1067F0000078001D4749087000228921012001F01E
:1068000025FE44480078001D4249087000222D21D1
:10681000012001F01BFE3F480078001D3D49087033
:1068200000228921012001F011FE3A480078001D64
:106830003849087000228921012001F007FE052156
:106840000820FFF781FE08203149086054E004F079
:10685000F7FF2D4901EB001004682046FFF7E2FD29
:106860002A49086000220B21022001F0EFFD0521DA
:106870000820FFF769FE25480068010E002201206C
:1068800001F0E4FD23480078001D22490870002231
:106890001E480068C0F30741012001F0D7FD1D48E4
:1068A0000078001D1B490870002218480088C0F3BA
:1068B0000721012001F0CAFD16480078001D154986
:1068C0000870124801780022012001F0BFFD052167
:1068D0000820FFF739FE1C200D4908600CE000225B
:1068E0000B21022001F0B2FD05210820FFF72CFE4C
:1068F00009200749086000BF00BF70BD3F010020AC
:10690000B80200202C5A0208582C0020F80200205F
:10691000D00200203501002070B505460C46B54870
:10692000007808287BDCB3480078082814DAB248DD
:106930000068B0F5FA7F05DA00225F21012001F03E
:1069400085FD04E000222021012001F07FFDAB48FD
:1069500000780B38A94908704B2D7BD00CDC2B2D0F
:1069600079D004DC1D2D14D0272D2AD114E12D2D32
:1069700072D02E2DF9D1C3E08B2D57D004DC4D2DD4
:106980006BD04E2DF1D16FE08D2D34D08E2DECD10A
:1069900018E098480078082813DA302195480278E2
:1069A0000078401C934B18709548815424B90022FC
:1069B000012001F04BFD04E000222A21012001F01A
:1069C00045FD15E18B480078082813DA3121894804
:1069D00002780078401C874B18708948815424B98C
:1069E0000022012001F032FD04E000222A210120D2
:1069F00001F02CFDFCE07F480078082815DA3222EF
:106A00007C4801780078401C7A4B18707C484254CE
:106A100034B900223221012001F018FD05E0E8E040
:106A200000222A21012001F011FDE1E071480078E7
:106A3000082818DA33226F4801780078401C6D4B23
:106A400018706F4842544CB900223321012001F0E4
:106A5000FDFC08E03BE085E06BE01FE000222A211E
:106A6000012001F0F3FCC3E062480078082814DA42
:106A70003422604801780078401C5E4B18706048F2
:106A800042542CB900223421012001F0DFFC04E043
:106A900000222A21012001F0D9FCA9E05548007804
:106AA000082813DA3521534802780078401C514BEE
:106AB00018705348815424B90022012001F0C6FC0B
:106AC00004E000222A21012001F0C0FC90E04948A6
:106AD0000078082813DA3621464802780078401CEE
:106AE000444B18704648815424B90022012001F01B
:106AF000ADFC04E000222A21012001F0A7FC77E090
:106B00003C480078082813DA37213A4802780078A0
:106B1000401C384B18703A48815424B90022012097
:106B200001F094FC04E000222A21012001F08EFCF7
:106B30005EE030480078082813DA38212D480278C2
:106B40000078401C2B4B18702D48815424B900222A
:106B5000012001F07BFC04E000222A21012001F049
:106B600075FC45E023480078082814DA39222148CA
:106B700001780078401C1F4B1870214842542CB9F2
:106B800000223921012001F061FC04E000222A21C9
:106B9000012001F05BFC2BE016480078002826DD80
:106BA00014480078401E1349087000201449114A07
:106BB000127888540F480078072809DA002220212B
:106BC000012001F043FC0D4800780B380B49087098
:106BD0000A4800780B38094908700022202101205A
:106BE00001F034FC054800780B380449087000BFF8
:106BF00000BF70BD3D0100201400002035010020C1
:106C00004101002010B510210448FFF7B0FB4FF4FC
:106C100080610348FFF7A9FB012010BD0008014077
:106C20000010014030B502460B4801680B4803686C
:106C30000EE001EB41000A4C54F82000904201D1D3
:106C4000012030BD481C142490FBF4F504FB150111
:106C50009942EED10020F4E7C8000020CC000020CB
:106C6000E40D0020014608480068CD225043074A41
:106C700002EB8000143000EB0110C068006808B11E
:106C8000012070470020FCE7B80200202C5A0208BF
:106C90000146C1EBC100034A02EB8000008B00F407
:106CA000FE60704738E901080146C1EBC100034AA4
:106CB00002EB8000007EC0F34000704738E9010815
:106CC0000146C1EBC100044A02EB8000007E00F0E7
:106CD000010080F00100704738E901080146C1EB6E
:106CE000C100034A02EB8000806900F4FF20704776
:106CF00038E901080146C1EBC100054A52F82000FD
:106D00004FF6FF72904201D1012070470020FCE74E
:106D100038E901080146CD204843054A02EB8000CE
:106D2000C068006808B1012070470020FCE700003F
:106D30002C5A020838B500250820ADF800001020B4
:106D40008DF8030003208DF8020069464A48FFF7DA
:106D500089FA08214848FFF708FBFCF7CFF94648B5
:106D6000FFF7F2FA04130820ADF8000048208DF870
:106D7000030069464048FFF775FA0F2C76D10420CE
:106D8000ADF8000010208DF8030003208DF80200FC
:106D900069463948FFF766FA04213748FFF7E5FAF4
:106DA000FCF7ACF93448FFF7CFFA04130420ADF830
:106DB000000048208DF8030069462F48FFF752FA7B
:106DC0000F2C4FD10220ADF8000010208DF80300E9
:106DD00003208DF8020069462748FFF743FA022195
:106DE0002548FFF7C2FAFCF789F92348FFF7ACFA08
:106DF00004130220ADF8000048208DF80300694616
:106E00001D48FFF72FFA0F2C27D10120ADF8000005
:106E100010208DF8030003208DF802006946164803
:106E2000FFF720FA01211448FFF79FFAFCF766F9F3
:106E30001148FFF789FA04130120ADF8000048203B
:106E40008DF8030069460C48FFF70CFA0F2C00D1AF
:106E50000FE0E0B240F010050BE0E0B240F020059A
:106E600007E003E0E0B240F0400502E0E0B240F0AD
:106E70008005284638BD00000014014070B500F0C0
:106E800035F8002417E0002511E0A107080E294677
:106E900003F0E4F9002606E000222146012004F078
:106EA00013F9701CC6B2402EF6DB681CC5B2082D63
:106EB000EBDB601CC4B2022CE5DB00F023F870BDF4
:106EC00010B548F220010748FFF74FFA4FF4804110
:106ED0000448FFF74CFA40210348FFF746FAFFF752
:106EE000CDFF10BD000C01400008014010B53E224E
:106EF0000021084604F0E8F83E220121002004F0B9
:106F0000E3F810BD10B53F220021084604F0DCF87C
:106F10003F220121002004F0D7F810BD70B50546CE
:106F20000C466E201C490870012D28D11B480068B2
:106F3000C8280CDA00201A490870E2B2FE2101F0DC
:106F400085FAE2B22021002001F080FA23E0134804
:106F50000068B0F5FA7F1EDD10480068B0F52F7F9D
:106F600019DA01200E490870E2B2F821002001F080
:106F70006DFAE2B22021002001F068FA0BE0022D48
:106F800009D1E2B2F721002001F060FAE2B2FD215E
:106F9000002001F05BFA70BD3501002014000020D4
:106FA0000403002000BFFEE77047000010B54FF457
:106FB0008031C80200F0A0F84FF4E06000F092F8D1
:106FC000284800F051F82620264908700020487013
:106FD00001208870C870084600F046F82720214933
:106FE00008700020487001208870C870084600F0C2
:106FF0003BF803201B49087000204870022088706D
:107000000120C870084600F02FF8072015490870C5
:107010000020487088700120C870084600F024F8ED
:107020000820104908700020487088700120C8703E
:10703000084600F019F80A200A4908700020487034
:1070400088700120C870084600F00EF81720054926
:1070500008700020487088700120C870084600F051
:1070600003F810BD91000020F0B50F22C37801781D
:1070700001244FF0E0263BB3184B1B6803F4E06398
:10708000C3F5E0631D0AC5F10403EA4045789D405D
:10709000837813402B431A018B07DF0E21F0030383
:1070A0000F49BA405D182968FF23BB4099431A4035
:1070B00011432960007800F01F018C40400906EB65
:1070C0008000C0F80041F0BD01F01F008440480975
:1070D00006EB8000C0F88041F0BD00000CED00E040
:1070E00000E400E0024908430249086070470000DC
:1070F0000000FA050CED00E0024A1140014302488D
:107100000160704780FFFF1F08ED00E010B50848E0
:10711000006820B901200649086003F089FB03F0EC
:10712000BFF803F03DF901F0EBFD0446204610BD29
:10713000DC0200207047000001490862704700002F
:1071400000000E4270472DE9F04180460C4615467E
:107150001E4604F1920003F011FA074685B104E0DF
:1071600032462021404601F071F938467F1C06283E
:10717000F6DB324604F19201404604F043F80FE09A
:10718000324604F19201404604F03CF804E03246F5
:107190002021404601F05AF938467F1C0628F6DBCC
:1071A000BDE8F081704770472DE9F04107460D4674
:1071B00090461E4680240C4800780C380A49087016
:1071C0000EE005EA040028B132463021384601F0CD
:1071D0003DF904E032463121384601F037F96410B8
:1071E000002CEED1BDE8F081350100202DE9F04101
:1071F00006460C4690461D460020244908702A4643
:107200002021304601F022F90A2094FBF0F00A21F7
:1072100090FBF1F201FB12003030C7B22A4639462A
:10722000304601F013F90A2094FBF0F100FB114005
:107230003030C7B22A463946304601F007F92A46AF
:107240002D21304601F002F94FF47A7094FBF0F0F2
:107250000A2190FBF1F201FB12003030C7B22A463E
:107260003946304601F0F2F8642094FBF0F00A2130
:1072700090FBF1F201FB12003030C7B22A463946CA
:10728000304601F0E3F8BDE8F08100003401002051
:107290002DE9F0470746884691461E464748007844
:1072A000303846490870464D2C6804F00F00FAF754
:1072B0005AFA824632465146384601F0C7F8C4F3BE
:1072C0000320FAF750FA824632465146384601F01A
:1072D000BDF8C4F30340FAF746FA824632465146F7
:1072E000384601F0B3F8C4F30360FAF73CFA82467B
:1072F00032465146384601F0A9F832462D2138462B
:1073000001F0A4F82D1D2C6804F00F00FAF72BFAF9
:10731000824632465146384601F098F8C4F30320BD
:10732000FAF721FA824632465146384601F08EF885
:10733000C4F30340FAF717FA8246324651463846FC
:1073400001F084F8C4F30360FAF70DFA824632467E
:107350005146384601F07AF832462D21384601F080
:1073600075F82D1D2C6804F00F00FAF7FCF9824621
:1073700032465146384601F069F8C4F30320FAF763
:10738000F2F9824632465146384601F05FF8C4F3BE
:107390000340FAF7E8F9824632465146384601F092
:1073A00055F8C4F30360FAF7DEF9824632465146D7
:1073B000384601F04BF8BDE8F087000035010020A9
:1073C000E8F7FF1F2DE9F04105460C4616467120EF
:1073D00049490870494901EB04110868FEF780FD2E
:1073E0008046FFF755FC074607F00F0000287AD1CA
:1073F0003811152877D2DFE800F0760B1C222876AA
:10740000762E343A40464C52585E767664766B005F
:1074100040F27B1001F028FC28B9324600212846B2
:1074200003F0F0FE04E032460F21284603F0EAFEA6
:107430005FE032460121284603F0E4FE59E032467F
:107440000221284603F0DEFE53E03246032128469F
:1074500003F0D8FE4DE032460421284603F0D2FE68
:1074600047E032460521284603F0CCFE41E0324693
:107470000621284603F0C6FE3BE032460721284697
:1074800003F0C0FE35E032460821284603F0BAFE7C
:107490002FE032460921284603F0B4FE29E03246A7
:1074A0000A21284603F0AEFE23E032460B2128468F
:1074B00003F0A8FE1DE032460C21284603F0A2FE90
:1074C00017E032460D21284603F09CFE11E00AE049
:1074D0003246F021284600F0B9FF3246F521284611
:1074E00000F0B4FF05E032460E21284603F08AFE84
:1074F00000BF00BFBDE8F08135010020582C0020FE
:1075000070B504460D46074800EB04102A46416852
:10751000002003F077FE2A460E21002003F072FEC1
:1075200070BD0000582C00202DE9F04105460C46A6
:1075300016460027672001F097FB06283FD2DFE8B8
:1075400000F0030C16202A3404EB4401234A52F8BD
:107550003100F9F745F8074631E004EB44011F4AD2
:1075600002EBC1014868F9F73BF8074627E004EB56
:1075700044011A4A02EBC1018868F9F731F807465D
:107580001DE004EB4401154A02EBC101C868F9F79C
:1075900027F8074613E004EB4401104A02EBC1014F
:1075A0000869F9F71DF8074609E004EB44010B4AA6
:1075B00002EBC1014869F9F713F8074600BF00BFA5
:1075C00007EB4700C0F140000549087032462146EC
:1075D000284603F017FEBDE8F0810000F4460208DB
:1075E0003501002010B500210846FEF7ADFF00224E
:1075F0000221084600F02AFF00212020FEF7A4FF08
:1076000000220321022000F021FF00214020FEF78C
:107610009BFF00220321022000F018FF00216020C0
:10762000FEF792FF00220421022000F00FFF042148
:107630000020FEF789FF00220521022000F006FF4E
:1076400004212020FEF780FF00220621022000F006
:10765000FDFE04214020FEF777FF002206210220D4
:1076600000F0F4FE04216020FEF76EFF00220721E7
:10767000022000F0EBFE10BD10B50020224908707A
:107680002249087000220D21022000F0DFFE202098
:107690001D49087000220E21022000F0D7FE402074
:1076A0001949087000220E21022000F0CFFE602050
:1076B0001549087000220F21022000F0C7FE0020AB
:1076C000114908700420114908700022102102207D
:1076D00000F0BCFE20200C4908700022112102207D
:1076E00000F0B4FE40200849087000221121022059
:1076F00000F0ACFE60200449087000221221022034
:1077000000F0A4FE10BD000035010020360100206D
:1077100070B504460D461646FFF764FF0021084683
:10772000FEF712FF324629462046FFF7FDFE70BDE8
:107730002DE9F04180460C4615461E4604F1160020
:1077400002F01CFF074685B104E032462021404686
:1077500000F07CFE38467F1C0628F6DB324604F13A
:107760001601404603F04EFD0FE0324604F11601CB
:10777000404603F047FD04E032462021404600F039
:1077800065FE38467F1C0628F6DBBDE8F0812DE952
:10779000F04106460D461746284601F065FA0446B4
:1077A000210E3A46304600F051FE3A46C4F30741F6
:1077B000304600F04BFE3A46C4F30721304600F055
:1077C00045FEE1B23A46304600F040FEBDE8F081A9
:1077D0002DE9F04107460C4615461E4605B33246D4
:1077E0002021384600F032FE32462021384600F093
:1077F0002DFE210E3246384600F028FE3246C4F3F4
:107800000741384600F022FE3246C4F307213846CD
:1078100000F01CFEE1B23246384600F017FE1FE0D1
:10782000210E3246384600F011FE3246C4F30741BD
:10783000384600F00BFE3246C4F30721384600F00C
:1078400005FEE1B23246384600F000FE3246202105
:10785000384600F0FBFD32462021384600F0F6FDA8
:10786000BDE8F081704700002DE9F04106460C4666
:1078700090461D46002029490870294894FBF0F0E5
:107880000A2190FBF1F201FB12003030C7B22A4608
:107890003946304600F0DAFD42F2107094FBF0F009
:1078A0000A2190FBF1F201FB12003030C7B22A46E8
:1078B0003946304600F0CAFD4FF47A7094FBF0F080
:1078C0000A2190FBF1F201FB12003030C7B22A46C8
:1078D0003946304600F0BAFD2A462D21304600F0E8
:1078E000B5FD0A2094FBF0F00A2190FBF1F201FBB8
:1078F00012003030C7B22A463946304600F0A6FDA5
:107900000A2094FBF0F100FB11403030C7B22A4648
:107910003946304600F09AFDBDE8F0813401002080
:10792000A086010070472DE9F04180460C461546BF
:107930001E4604F1100002F021FE074685B104E066
:1079400032462021404600F081FD38467F1C062843
:10795000F6DB324604F11001404603F053FC0FE021
:10796000324604F11001404603F04CFC04E032467C
:107970002021404600F06AFD38467F1C0628F6DBD1
:10798000BDE8F081704700002DE9F84F06460D462E
:1079900017469846A34901EB05110868FEF7A0FABF
:1079A0008246FFF79BF981469E4901EB0511086865
:1079B000FEF738FD04464C209B490870C9F30A00C5
:1079C000002822D14FEAE9202A281ED2DFE800F061
:1079D000A11D1D1D151E2F363D44521D97ABB5BF71
:1079E0001D73251D901DDD1D1DFEC91DD31D1D1DF3
:1079F0001DFDFC1D1D4BFB1D1DFA062043463A468E
:107A000021460090304600F0A5FC08E143463A4686
:107A10002146304600F03CFC01E1402082490870DC
:107A200043463A462146304600F05CF9F7E04346CB
:107A30003A462146304600F0C9FBF0E043463A465C
:107A40002146304600F018FAE9E043463A4621461E
:107A5000304600F0EBF8E2E043463A462146304635
:107A600000F0B4F9DBE043463A462146304600F0E8
:107A700065FAD4E040F27B1001F0F6F830B94346E5
:107A80003A462146304600F0D1FA13E0A4F52F70B3
:107A9000C0EB001000EB4000192101EB4000322147
:107AA00090FBF1F000F57F7A43463A465146304666
:107AB00000F0BCFAB3E040F27B1001F0D5F830B929
:107AC00043463A462146304600F0E2FB0FE0C4EB65
:107AD000041000EB4000192101EB4000322190FB23
:107AE000F1FA43463A465146304600F0D1FB96E063
:107AF00043463A4621463046FFF778FB8FE04C205C
:107B00004949087043463A4621463046FFF71BFB79
:107B100085E04C204449087043463A4621463046A9
:107B2000FFF706FE7BE04C203F49087043463A468B
:107B300021463046FFF7F6FE71E04C203A490870C6
:107B400043463A4621463046FFF72DFB67E04C207E
:107B50003549087043463A4621463046FFF782FED3
:107B60005DE04C203049087043463A462146304695
:107B7000FFF708FF53E04C202B49087043463A4674
:107B800021463046FFF7CFFE49E040F27B1001F07E
:107B90006BF830B943463A462146304600F0AEFA1B
:107BA00019E0A4F52F70C0EB001000EB4000192184
:107BB00001EB4000322190FBF1F000F52F7A4346B3
:107BC0003A4604E024E01CE00DE005E012E05146F6
:107BD000304600F093FA22E043463A4621463046CA
:107BE000FFF7E2FA1BE043463A4621463046FFF7EC
:107BF0004FFB14E043463A4621463046FFF734FE39
:107C00000DE043463A4621463046FFF7CBFA06E000
:107C100043463A4621463046FFF7DAFD00BF00BF33
:107C2000BDE8F88F582C0020350100202DE9F041E7
:107C300006460C4690461D4600202949087042F22F
:107C4000107094FBF0F00A2190FBF1F201FB12009E
:107C50003030C7B22A463946304600F0F7FB2A4694
:107C60002E21304600F0F2FB4FF47A7094FBF0F0D6
:107C70000A2190FBF1F201FB12003030C7B22A4614
:107C80003946304600F0E2FB642094FBF0F00A2114
:107C900090FBF1F201FB12003030C7B22A463946A0
:107CA000304600F0D3FB0A2094FBF0F00A2190FB51
:107CB000F1F201FB12003030C7B22A463946304695
:107CC00000F0C4FB0A2094FBF0F100FB11403030BF
:107CD000C7B22A463946304600F0B8FBBDE8F0810D
:107CE000340100202DE9F04106460C4617461D469A
:107CF000002034490870344894FBF0F000F0FF088D
:107D00002B463A464146002000F088FC42F21070B3
:107D100094FBF0F00A2190FBF1F201FB12003030ED
:107D200000F0FF082A464146304600F08FFB2A4605
:107D30002E21304600F08AFB4FF47A7094FBF0F06D
:107D40000A2190FBF1F201FB1200303000F0FF0835
:107D50002A464146304600F079FB642094FBF0F05F
:107D60000A2190FBF1F201FB1200303000F0FF0815
:107D70002A464146304600F069FB2A462E2130460D
:107D800000F064FB0A2094FBF0F00A2190FBF1F272
:107D900001FB1200303000F0FF082A464146304611
:107DA00000F054FB0A2094FBF0F100FB114030304E
:107DB00000F0FF082A464146304600F047FBBDE888
:107DC000F081000034010020A08601002DE9F0417F
:107DD00007460C4615461E4625B132462021384638
:107DE00000F034FB4FF4167094FBF0F00A2190FB86
:107DF000F1F201FB1200303000F0FF08324641463C
:107E0000384600F023FB3C2094FBF0F00A2190FB65
:107E1000F1F201FB1200303000F0FF08324641461B
:107E2000384600F013FB32463A21384600F00EFB8C
:107E30003C2094FBF0F100FB11400A2190FBF1F093
:107E4000303000F0FF0832464146384600F0FEFA76
:107E50003C2094FBF0F100FB11400A2190FBF1F271
:107E600001FB1200303000F0FF0832464146384630
:107E700000F0ECFABDE8F0812DE9F04106460C4631
:107E800017461D4600202C49087042F2107094FBE2
:107E9000F0F0642190FBF1F201FB120000F0FF080A
:107EA0002B463A464146304600F0B8FB4FF47A7014
:107EB00094FBF0F00A2190FBF1F201FB120030304C
:107EC00000F0FF082A464146304600F0BFFA2A4635
:107ED0002E21304600F0BAFA642094FBF0F00A211B
:107EE00090FBF1F201FB1200303000F0FF082A464F
:107EF0004146304600F0AAFA0A2094FBF0F00A212D
:107F000090FBF1F201FB1200303000F0FF082A462E
:107F10004146304600F09AFA0A2094FBF0F100FB4B
:107F20001140303000F0FF082A464146304600F04C
:107F30008DFABDE8F0810000340100202DE9F843FE
:107F400007460D4690461E460020374908702C46CD
:107F5000B4F52F7F0ADBA4F52F7406203346424682
:107F600021460090384600F0F5F95BE000202E49EC
:107F70000870C4F52F7442F2107094FBF0F00A21DF
:107F800090FBF1F201FB120000F0FF09334642467C
:107F90004946384603F0FCF94FF47A7094FBF0F050
:107FA0000A2190FBF1F201FB120000F0FF093346B9
:107FB00042464946384603F0EBF9642094FBF0F062
:107FC0000A2190FBF1F201FB120000F0FF09334699
:107FD00042464946384603F0DBF90A2094FBF0F0AC
:107FE0000A2190FBF1F201FB120000F0FF09334679
:107FF00042464946384603F0CBF90B48007820B991
:1080000032462D21384600F021FA0A2094FBF0F187
:1080100000FB1140303000F0FF0932464946384637
:1080200000F014FABDE8F883340100202DE9F04790
:1080300007460D4690461E462C46B4F52F7F08DBBA
:10804000A4F52F74334642462146384600F020F905
:108050004FE0002028490870C4F52F744FF47A705F
:1080600094FBF0F00A2190FBF1F201FB120000F00A
:10807000FF09334642464946384603F089F96420F1
:1080800094FBF0F00A2190FBF1F201FB120000F0EA
:10809000FF09334642464946384603F079F9164807
:1080A000007820B932462D21384600F0CFF90A2059
:1080B00094FBF0F00A2190FBF1F201FB120030304A
:1080C00000F0FF0932464946384600F0BFF9324613
:1080D0002E21384600F0BAF90A2094FBF0F100FB9B
:1080E0001140303000F0FF0932464946384600F072
:1080F000ADF9BDE8F0870000340100202DE9F0471C
:1081000007460D4690461E462C46B4F52F7F08DBE9
:10811000A4F52F74334642462146384600F0B8F89D
:108120004FE0002028490870C4F52F744FF47A708E
:1081300094FBF0F00A2190FBF1F201FB120000F039
:10814000FF09334642464946384603F021F9642088
:1081500094FBF0F00A2190FBF1F201FB120000F019
:10816000FF09334642464946384603F011F916489E
:10817000007820B932462D21384600F067F90A20F0
:1081800094FBF0F00A2190FBF1F201FB1200303079
:1081900000F0FF0932464946384600F057F93246AA
:1081A0002E21384600F052F90A2094FBF0F100FB32
:1081B0001140303000F0FF0932464946384600F0A1
:1081C00045F9BDE8F0870000340100202DE9F041B9
:1081D00006460C4617461D4600202C49087042F200
:1081E000107094FBF0F00A2190FBF1F201FB1200F9
:1081F00000F0FF082B463A464146304600F00EFAA2
:108200004FF47A7094FBF0F00A2190FBF1F201FB3D
:10821000120000F0FF082B463A464146304600F077
:10822000FDF9642094FBF0F00A2190FBF1F201FBD0
:108230001200303000F0FF082A464146304600F078
:1082400005F92A462E21304600F000F90A2094FB59
:10825000F0F00A2190FBF1F201FB1200303000F047
:10826000FF082A464146304600F0F0F80A2094FB09
:10827000F0F100FB1140303000F0FF082A46414683
:10828000304600F0E3F8BDE8F08100003401002042
:108290002DE9F04106460C4617461D4600202C49A4
:1082A000087042F2107094FBF0F00A2190FBF1F29A
:1082B00001FB120000F0FF082B463A4641463046CB
:1082C00000F0ACF94FF47A7094FBF0F00A2190FBC7
:1082D000F1F201FB120000F0FF082B463A4641463E
:1082E000304600F09BF9642094FBF0F00A2190FBEB
:1082F000F1F201FB120000F0FF082B463A4641461E
:10830000304600F08BF90A2094FBF0F00A2190FB34
:10831000F1F201FB1200303000F0FF082A4641461E
:10832000304600F093F82A462E21304600F08EF8B1
:108330000A2094FBF0F100FB1140303000F0FF0800
:108340002A464146304600F081F8BDE8F081000041
:10835000340100202DE9F04707460C4690461E46A2
:10836000089D002037490870062D0FDB364894FB26
:10837000F0F00A2190FBF1F201FB120000F0FF097E
:10838000334642464946384600F048F9052D10DB91
:1083900042F2107094FBF0F00A2190FBF1F201FB25
:1083A000120000F0FF09334642464946384600F0C5
:1083B00035F9042D10DB4FF47A7094FBF0F00A21AC
:1083C00090FBF1F201FB120000F0FF093346424638
:1083D0004946384600F022F9032D0FDB642094FB58
:1083E000F0F00A2190FBF1F201FB120000F0FF090E
:1083F000334642464946384600F010F9022D0FDB5D
:108400000A2094FBF0F00A2190FBF1F201FB12002C
:1084100000F0FF09334642464946384600F0FEF870
:10842000012D0CDB0A2094FBF0F100FB11403030F1
:1084300000F0FF0932464946384600F007F8BDE82B
:10844000F087000034010020A086010070B50646C8
:108450000C46154626B1012E07D0022E0FD109E099
:108460002946204600F00EF809E02946204600F093
:1084700043F804E02946204600F08AF800BF00BF18
:1084800070BD00002DE9F04105460E46002706B1FB
:10849000FF27202D00DA202500241EE01348007855
:1084A000802818DA124801781048007801F0D6FECA
:1084B000A5F120000F4B03EBC000005D80EA07022E
:1084C0000A4800788111012002F0FEFD074800787B
:1084D000401C06490870601CC4B2082CDEDB03484F
:1084E0000078801E01490870BDE8F0813501002048
:1084F00036010020741902082DE9F04105460F46A7
:108500004FF000080FB14FF0FF08202D00DA2025B2
:1085100000242DE0002622E01A48007880281CDA8A
:10852000194800782044C1B21648007801F096FE40
:10853000A5F12000154B03EB401006EB0413C05CC3
:1085400080EA08020F4800788111012002F0BCFD8A
:108550000C480078401C0B490870701CC6B2102EE5
:10856000DADB08480078103806490870601CC4B28D
:10857000022CCFDB034800780B3002490870BDE8BD
:10858000F081000035010020360100207C20020827
:108590002DE9F04106460F464FF000080FB14FF0AD
:1085A000FF0800242BE0002520E0194800788028EF
:1085B0001ADA184800782044C1B21548007801F052
:1085C0004DFE154800EBC61005EB4413C05C80EA75
:1085D00008020F4800788111012002F075FD0C4857
:1085E0000078401C0A490870681CC5B2202DDCDBED
:1085F00007480078203806490870601CC4B2042C73
:10860000D1DB03480078163001490870BDE8F081DD
:1086100035010020360100209C3C02082DE9F04184
:1086200007460C4615461E4614B90B48007850B153
:1086300001200949087004F13000C1B232463846C1
:10864000FFF704FF05E025B1324620213846FFF749
:10865000FDFEBDE8F08100003401002010B50446A5
:108660002448006800EB4000234941F82040611E87
:1086700001EBC10101EB410101F16C0000F0F4FAE2
:108680001C49096801EB41011B4A02EB810148606A
:10869000611E01EBC10101EB410101F1860000F017
:1086A000E3FA1449096801EB4101134A02EB810125
:1086B000886010480068401C142190FBF1F201FB17
:1086C00012000C490860084600680C490968884295
:1086D0000ED10221012001F037FD06480068401E3E
:1086E0000449086008460068002801DA1320086081
:1086F00010BD0000CC000020E40D0020C8000020C8
:10870000034A516821F44041014351607047000021
:1087100000100240044A0029516901D0014300E0E1
:10872000814351617047000000100240044A002953
:10873000D16901D0014300E08143D161704700005D
:1087400000100240044A0029916901D0014300E071
:1087500081439161704700000010024010B500F0A5
:1087600035F84FF4803000F0C3F800F029F91649CD
:10877000087008460078012824D11020FDF73AFB44
:108780000220FDF743FB002000F0A8F8002000F0D5
:10879000E5F84FF4806000F0D7F84FF44040FFF761
:1087A000AFFF00214FF4803000F0E8F8012000F026
:1087B000DFF800BF392000F079F80028FAD0022055
:1087C00000F0F4F810BD0000900000200B48016894
:1087D00041F0010101604168094A114041600168AE
:1087E000084A11400160016821F48021016041685C
:1087F00021F4FE01416000218160704700100240B9
:108800000000FFF8FFFFF6FE224A10B55168224B28
:1088100011F00C0103D0042903D0082903D0036010
:1088200015E01E4912E05168022301F4701103EBB8
:108830009141536813F4803F04D053689B0303D5E0
:10884000174B02E0174B00E0144B5943016051688D
:10885000154B01F0F00109095C5C0168E1404160E1
:10886000546804F4E064240A1C5D21FA04F4846072
:10887000546804F46054E40A1B5DD940C160526836
:10888000094B02F44042920B1B1F9A5CB1FBF2F1C0
:10889000016110BD0010024000127A0040787D0195
:1088A00020BCBE0000093D00CA4D0308024600205E
:1088B00053090949012B0BD0022B0BD0D1F82410FE
:1088C00002F01F02012393400B4200D001207047A9
:1088D0000968F5E7096AF3E700100240034A5168A6
:1088E00021F0F00101435160704700000010024088
:1088F0000B490A6822F480320A600A6822F4802256
:108900000A60B0F5803F07D0B0F5802F03D108682A
:1089100040F4A02008607047086840F48030F9E710
:108920000010024070470000064900220A7001F85A
:108930002029012802D0042802D1052081F8200036
:108940007047000020100240034A516821F4E061A2
:1089500001435160704700000010024003494A681B
:1089600022F4605242EAC0004860704700100240A2
:10897000014908667047000000004242034A5368FC
:10898000084323F47C1318435060704700100240E2
:1089900001490860704700003C04424202490A6AEB
:1089A00002430A627047000000100240034A516807
:1089B00021F00301014351607047000000100240A4
:1089C00030B50B4C40F2FF153120FFF76FFF2070E0
:1089D0006068401C6060207810B96068A842F3D1DC
:1089E0003120FFF763FF002800D0012030BD0000D8
:1089F000B80300207047000002490A8882430A80B9
:108A0000704700000428004010B54FF47A7400BF8E
:108A100001214FF0C050FFF789FE0120FEF78CFBCB
:108A20000120FFF781FF2848046042F21070844261
:108A300001DA04F5FA7400BF4120FFF737FF18B9D7
:108A4000214800680028F7D14120FFF72FFFE8B93F
:108A50000020FFF769FF0020FEF76EFB00214FF0BA
:108A6000C050FFF763FE4FF480611848FDF77FFCAC
:108A70004FF4FA701449086000BF134800680028DA
:108A8000FBD14FF480611148FDF76FFC4120FFF7E7
:108A90000DFF0028BCD04FF48070FFF77FFF01204E
:108AA000FFF776FF00F0D4F800F0CAF8012108467D
:108AB00000F04AF800F0C4F847F6FF7000F0B0F894
:108AC00000F0BEF810BD000018000020000C0140AE
:108AD0000248018841F010010180704704280040DD
:108AE0000248018821F010010180704704280040ED
:108AF000034800880249091F098840EA014070477D
:108B00001C28004006490988054A0140121FC9B2C5
:108B10001288024202D009B101207047002070473C
:108B20000428004010B50120FFF7ECFF48B100F029
:108B300087F80120FFF760FF02480068401C0149E8
:108B4000086010BD04000020044A0029118801D0EB
:108B5000014300E08143118070470000002800407D
:108B600010B501214FF0C050FFF7E0FD0120FEF7E6
:108B7000E3FA0420F8F70CFE4AF2A55188422FD000
:108B8000FFF742FF00F05CF84AF6C00000F038F84A
:108B900000F056F84AF2A5510420F8F7FFFD002135
:108BA0000820F8F7FBFD00210C20F8F7F7FD002165
:108BB0001020F8F7F3FD00211420F8F7EFFD002155
:108BC0001820F8F7EBFD00211C20F8F7E7FD002145
:108BD0002020F8F7E3FD00212420F8F7DFFD0DE069
:108BE0004120FFF763FE08B9FFF70EFF00F030F8F1
:108BF00001210846FFF7A8FF00F022F810BD000091
:108C000000B50246FFF764FF0449100C0880081DF8
:108C100002805DF804EBFFF763BF000018280040F6
:108C200000B50246FFF754FF0449C2F30340088031
:108C3000081D02805DF804EBFFF752BF08280040D2
:108C4000024801888906FCD57047000004280040CE
:108C50000448018821F00801018001880907FCD53A
:108C6000704700000428004010B50446204600F07C
:108C7000CBF810BD70B54FF4C970FFF7F5FF05468E
:108C8000002D01DB322D00DB0025681E051E00DAF9
:108C900031252C4602221848016818480068FAF766
:108CA00025F900BF04F29310FFF7DEFF064601F03E
:108CB00009F82C2000F0AEFF04F2C510FFF7D4FF36
:108CC000064600F0FFFF2C2000F0A4FF04F2F7108E
:108CD000FFF7CAFF064600F0F5FF641E002C00DA1D
:108CE0003124AC4202D02C2000F094FFAC42D9D108
:108CF000FAF71CF970BD0000E0000020E40000203D
:108D000070B520480078D0B100BFFEF713F80446D4
:108D1000FAF7ECF9FEF70EF80546FAF7E7F9FEF771
:108D200009F80646FAF7E2F9AC42EED1B442ECD1CA
:108D30000CB1002070BD002012490870FAE700BF96
:108D4000FDF7F8FF04460CB90020F3E7FAF7CEF977
:108D5000FDF7F0FF0546FAF7C9F9FDF7EBFF064608
:108D6000FAF7C4F9AC42EBD1B442E9D1054804703A
:108D700034B14FF4167004490860012003490860BB
:108D80002046D7E7A800002028030020E8020020A2
:108D900070B504460D464FF480411848FDF7E7FAD8
:108DA00024B980211648FDF7E0FA03E08021144839
:108DB000FDF7DDFA25B140211248FDF7D8FA04E0AD
:108DC0004FF400410D48FDF7D2FA20210B48FDF782
:108DD000CEFA0B48FDF7B8FA0646360A20210748B6
:108DE000FDF7C3FA40210748FDF7BFFA4FF40041F1
:108DF0000248FDF7BAFA304670BD0000000C014091
:108E000000180140000801402DE9F0470646002700
:108E1000B500C5F30749ADB24FF0030800BF002409
:108E20002946484605F0B8FBF0B105F087FAA121C4
:108E300001EB4901C8B205F031FC0746A7B105F0C6
:108E400019F8044605F03EF805F014F800EB042488
:108E500005F038F805F00EF800EB042405F032F8C0
:108E600005F008F800EB042405F078FA27B9A8F11A
:108E7000010000F0FF0801E04FF00008B8F1000F1A
:108E8000CDDC2046BDE8F08710B51848006820B159
:108E9000012807D0022817D109E01448006804F01F
:108EA000B9FC15E01148006804F0B4FC10E010496A
:108EB0000E4A126831F81200FDF73CFB0D490B4ACF
:108EC000126841F8220003E000200849086000BF52
:108ED00000BF06480068401C044908600846006856
:108EE000022801DD0020086010BD0000C000002045
:108EF0003C0D0020B00B0020F0B502460B460024CC
:108F00000FE0174901EB021516490E680968491C64
:108F1000144F3960A85DF8F731FC04EB840100EBD5
:108F200041040F4800EB02100E490968405C98426A
:108F300013D00B4800EB02100A490968405C302846
:108F40000BDB074800EB021006490968405C392832
:108F500003DC044800681328D3DB2046F0BD000082
:108F6000FC1F0020F400002070B505460E460024CA
:108F700004E0FF2000F09EFF2855641CB442F8D3A3
:108F8000012070BD10B580210148FDF7EEF910BD3C
:108F90000014014010B580210148FDF7E8F910BD2B
:108FA0000014014010B580210348FDF7E0F980214D
:108FB0000148FDF7DAF910BD0010014010B510218D
:108FC0000148FDF7D2F910BD0014014010B5102181
:108FD0000148FDF7CCF910BD0014014010B54FF465
:108FE00000610248FDF7C1F910BD0000000C01400E
:108FF00010B54FF400610248FDF7B9F910BD00004B
:10900000000C014010B540210148FDF7AEF910BD3C
:109010000010014010B540210148FDF7A8F910BD2E
:109020000010014010B54FF480710248FDF79DF922
:1090300010BD00000010014010B54FF480710248CF
:10904000FDF795F910BD00000010014010B54FF478
:1090500000610248FDF789F910BD000000140140CD
:1090600010B54FF400610248FDF781F910BD000012
:109070000014014010B54FF400710248FDF775F976
:1090800010BD00000010014010B54FF400710248FF
:10909000FDF76DF910BD00000010014010B54FF450
:1090A00080610248FDF761F910BD00000014014025
:1090B00010B54FF480610248FDF759F910BD00006A
:1090C0000014014010B54FF400610248FDF74DF95E
:1090D00010BD00000008014010B54FF400610248C7
:1090E000FDF745F910BD00000008014010B54FF430
:1090F00000510248FDF739F910BD0000000C014095
:1091000010B54FF400510248FDF731F910BD0000D1
:10911000000C014010B54FF480510248FDF725F9CD
:1091200010BD00000008014010B54FF48051024806
:10913000FDF71DF910BD00000008014010B54FF407
:1091400080510248FDF711F910BD0000000C0140EC
:1091500010B54FF480510248FDF709F910BD000029
:10916000000C0140F0B507460C461646B44201D14A
:109170002046F0BDA01900EBD0714D1005EB450065
:10918000084901EB80004068B84205DD3246691CA1
:109190003846FFF7E7FFECE72A4621463846FFF757
:1091A000E1FFE6E7900B020870B5024600200023BD
:1091B00017E000EB4004304D55F82440944206D1AE
:1091C00000EB400405EB840464688C4206D000EB9D
:1091D0004004294D05EB8404A4680CB9012300E088
:1091E000401C192801DA002BE3D0E3B300EB400464
:1091F000214D05EB8404A468022C3BD123E0441CE0
:1092000004EB44041C4D55F8244000EB40051A4E75
:1092100046F82540441C04EB4404354605EB840421
:10922000646800EB400506EB85056C60441C04EBAC
:109230004404354605EB8404A46800EB400506EBC6
:109240008505AC60401C1828D9DB002400EB4005E4
:10925000094E46F8254000EB400506EB85056C609D
:1092600000EB400500E005E006EB8505AC6001245D
:10927000024D2C7070BD0000100C00203F0100203A
:10928000002010E0002100EB4002084B03EB8202BB
:10929000916000EB400243F8221000EB400203EB28
:1092A00082025160401C1928ECDB7047100C002032
:1092B0000021074A1170002004E00021054A1154E2
:1092C000411CC8B20828F8DB0021034A117070471E
:1092D0003D0100204101002040010020002014E059
:1092E000002100EB40020A4B43F8221000EB400241
:1092F00003EB8202516000EB400203EB82029160BB
:10930000044A1160044A1160401C1428E8DB7047CD
:10931000E40D0020C8000020CC00002070B50E48ED
:109320000068FCF7B7FD04460B480068FCF794FDA5
:10933000054601222946204601F068FE06490968D3
:10934000491C054A08461160FDF7D4FC10B1002005
:109350000149086070BD00002000002070B539A1EF
:109360003948F7F7F0F839490860084600680028DE
:1093700067D04FF480613648FCF7F9FF012035498A
:10938000087000F0DDFF03220421084600F0F4FF1E
:1093900005220621042000F0EFFF2AE0002400252A
:1093A0002D48005D2A2822D008E02B48005D05EBFF
:1093B000850100EB4100A0F13005641C2648005DEA
:1093C0003D28F2D1641C002608E02348005D06EB2E
:1093D000860100EB4100A0F13006641C1E48005DD0
:1093E0000A28F2D100223146284601F00FFEFDF78F
:1093F000CBF816481E2102681748F7F72FF8002807
:10940000CCD1FDF7C1F811480068F7F7C3F8FDF7B4
:10941000BBF812490C4803F0ADFBFDF7B5F841F27B
:1094200088300F49086001E0FDF7AEF80C4800688D
:109430000028F9D107490870FDF720FD01200949EE
:10944000087070BD720000009C4D0308AC03002042
:10945000000C0140D8000020D04B0020B14D030883
:10946000180000203F01002070B5E5E000F0ACFBE3
:10947000044674480078062870D2DFE800F0031430
:10948000384C70B3012C0DD1C8206F490860012001
:109490006C49087000206D4908606D4908602046DD
:1094A00000F0DEFBC7E0204600F0DAFB2C2C16D1E2
:1094B00001266520FFF7D8FB064665480068B042E4
:1094C00002D06348006818B902205E49087002E0C3
:1094D00000205C49087000205E49086006E02146D3
:1094E0005B480068F8F734F959490860A3E0204662
:1094F00000F0B6FB2C2C06D1032052490870002046
:109500005549086006E0214652480068F8F720F9FE
:10951000504908608FE0204600F0A2FB022C15D1D4
:1095200004204849087000204C4908604C490860F4
:10953000002508E000214B48484A126800EB021061
:109540004155681CC5B2102DF4DB06E021464248A7
:109550000068F8F7FDF8404908606CE067E02046D5
:1095600000F07EFB032C06D1052036490870002050
:109570003D49086035E02C2C20D138480068401C5B
:109580003649086008460068642803DB084600681E
:10959000401E0860002032490860002508E00020D5
:1095A00030492E4A126801EB02114855681CC5B2B9
:1095B000102DF4DBC8202449086012E0294827490F
:1095C000096800EB011026490968445424480068E2
:1095D000401C2349086008460068122801DD12205B
:1095E000086028E0042C13D11F4800681749096857
:1095F000884209D14FF416701C49086000F038F811
:1096000000201049087011E000200E4908700DE09C
:10961000154800680001144908602046F9F7AEF8C3
:109620001149098889B208430F49086003E0002006
:109630000449087000BF00BF00F0DEFA00287FF484
:1096400015AF70BD0B010020FC00002000010020C0
:10965000E0000020E4000020E8000020EC000020F2
:10966000F0000020FC1F002004010020F800002072
:109670002DE9F047FC4800680E2878D009DC0C285A
:1096800049D2DFE800F048174849788BCC48484871
:10969000FEFD65286CD006DC0F286AD0102869D042
:1096A000642838D1B2E1662876D0672875D068285A
:1096B000F7D129E20222ED480168ED480068F9F788
:1096C00015FC002400BF0020EA4908600021204664
:1096D000FFF712FC80464046FCF702FC002806DB40
:1096E0004046FCF79FFE054600F0ECFA05E02D2011
:1096F00000F090FA312000F08DFADF4800688442D3
:1097000002DA2C2000F086FA641CDB4800688442F0
:10971000D9DDF9F70BFC16E20222D4480168D448DF
:109720000068F9F7E3FBD5480078D5490978884205
:1097300006D12D2000F06EFA312000F06BFA13E014
:10974000CF4805780CE0681CC5B2142D00DB00255D
:10975000CC4951F8250000F0B5FA2C2000F05AFA57
:10976000C6480078A842EED1F9F7E0FBEBE109E149
:1097700096E134E146E1C1480078C149087002220F
:10978000BA480168BA480068F9F7B0FB302000F029
:1097900041FAF9F7CBFBD6E192E195E100250222EF
:1097A000B2480168B2480068F9F7A0FBB6480078F3
:1097B00030B92D2000F02EFA312000F02BFA1BE0FA
:1097C00016E0B24951F8350000F07CFA2C2000F088
:1097D00021FAAE4901EBC501486800F073FA681C34
:1097E000C5B2A9480078854202DA2C2000F012FAAE
:1097F000A54800788542E4DBF9F798FB002508E0EE
:109800000020A24941F8350001EBC5014860681C01
:10981000C5B2782DF4DB00209B49087093E1002548
:1098200002229248016892480068F9F75FFB984865
:10983000007830B92D2000F0EDF9312000F0EAF980
:109840001BE016E0934951F8350000F03BFA2C205C
:1098500000F0E0F98F4901EBC501486800F032FAE9
:10986000681CC5B28A480078854202DA2C2000F0D4
:10987000D1F9874800788542E4DBF9F757FB01E02E
:109880007FE010E0002508E00020824941F8350023
:1098900001EBC5014860681CC5B2782DF4DB0020DF
:1098A0007B4908704FE10024A1467B4800780028DE
:1098B00054D100BF002600206E4908603D2120469B
:1098C000FFF71AFB80466B480068401C6949086036
:1098D0004046FCF705FB002839DB4046FCF700FB5F
:1098E00040B900212046FFF707FB0646304600F04E
:1098F00099FC2EE04046FCF7F3FA1B2829D0002102
:109900002046FFF7F9FA06464046FCF7E9FA054615
:10991000FDF7D6F9E8B14046FCF7E2FA0546FCF758
:10992000AFFAB04202DD49F0020912E04046FCF70E
:10993000D7FA0546FCF79AFAB04202DA49F0040970
:1099400007E000223146404601F060FB01E049F0AB
:109950000109641C484800688442ABDD4348006844
:1099600070B114224148016841480068F9F7BEFA15
:109970004949097809EBC10000F0A4F9F9F7D6FAD2
:10998000E1E0E0E00024002717E00020394908600A
:1099900000212046FFF7B0FA404941F83700641C27
:1099A00000203449086000212046FFF7A5FA3B4912
:1099B00001EBC7014860641C7F1C2F48006884428B
:1099C000E3DB09E00020354941F837000022384642
:1099D0007F1C01EBC0004260192FF3DBB3E00020D5
:1099E0002449086000210846FFF786FA8046404671
:1099F000FCF718FD012804D101220221404601F0A4
:109A000005FBA0E000201B4908609CE000201949EC
:109A1000086000210846FFF76FFA804600201549CC
:109A2000086000210120FFF767FA0646FA2E00DDE4
:109A3000FA2602220D4801680D480068F9F756FA27
:109A4000C24600250AE01AF8010B00F03BF9701E2F
:109A5000A84202DD2C2000F0DDF86D1CB542F2DBDF
:109A6000F9F764FA6FE00000E8000020E000002051
:109A7000E4000020F4000020EC000020250000207D
:109A800024000020E0030020090100203004002011
:109A90000A010020F00700200C010020240F002004
:109AA00000202A49086000210846FFF725FA2849C6
:109AB00008600846006810B101202649087042E09D
:109AC0000020244908703EE0002020490860002161
:109AD0000846FFF711FA18B1A0F2E73090B902E09A
:109AE000FFF7C8F80EE0F7F779FF02221A4801687D
:109AF0001A480068F9F7FAF9002000F0E3F8F9F7DE
:109B000015FA00BF00BF1EE0022213480168134887
:109B10000068F9F7EBF9122000F0D4F82C2000F0DF
:109B200079F86420FFF7A0F8054600F0CBF82C2068
:109B300000F070F86520FFF797F8054600F0C2F8CE
:109B4000F9F7F4F900BF00BFBDE8F087F40000208A
:109B5000D4000020D8000020E0000020E400002015
:109B600010B50020114908601149086011490860CA
:109B700011490860114908704FF4164010490860F7
:109B800000208880C880088188810C2048810D4889
:109B900001F07EF8012240F225510A4801F05FF8F9
:109BA0000121084801F032F810BD00001401002026
:109BB000100100201C010020180100200B010020D2
:109BC000EC0F00200044004000BF08480068084A2D
:109BD00012689042F9D005480068401CC0F30A01A1
:109BE000024801600348405C7047000014010020F7
:109BF00010010020FC0F0020044800680449096897
:109C0000884201D0012070470020FCE710010020AD
:109C10001401002070B505460D480068401CC0F3D3
:109C20000A0400BF0B4800688442FBD00A4805556F
:109C300007480460284600F013F8012240F227711B
:109C4000064801F00CF80121044800F0DFFF70BD68
:109C5000180100201C010020FC17002000440040D7
:109C600007490988C1F307214140064A32F821100B
:109C7000034A127881EA022189B2014A11607047D1
:109C8000000100207415020810B5044604F13000EC
:109C9000C4B2392C01DDE01DC4B22046FFF7BAFF83
:109CA00010BD000010B50446002C02DD012004495F
:109CB00008700348007810B12046FFF7E5FF10BD9B
:109CC0000801002070B5044600203E490870002CB1
:109CD00000DA00243C4894FBF0F00A2190FBF1F2FA
:109CE00001FB1200C5B22846FFF7DCFF374894FBA2
:109CF000F0F00A2190FBF1F201FB1200C5B22846F8
:109D0000FFF7D0FF324894FBF0F00A2190FBF1F20C
:109D100001FB1200C5B22846FFF7C4FF2D4894FB93
:109D2000F0F00A2190FBF1F201FB1200C5B22846C7
:109D3000FFF7B8FF284894FBF0F00A2190FBF1F2FE
:109D400001FB1200C5B22846FFF7ACFF42F21070CB
:109D500094FBF0F00A2190FBF1F201FB1200C5B276
:109D60002846FFF79FFF4FF47A7094FBF0F00A212A
:109D700090FBF1F201FB1200C5B22846FFF792FFFB
:109D8000642094FBF0F00A2190FBF1F201FB120039
:109D9000C5B22846FFF786FF0A2094FBF0F00A219F
:109DA00090FBF1F201FB1200C5B22846FFF77AFFE3
:109DB0000A2094FBF0F100FB1140C5B22846FFF7E2
:109DC00063FF70BD0801002000CA9A3B00E1F50561
:109DD0008096980040420F00A086010010B504460E
:109DE000C4F30330FFF750FFC4F30320FFF74CFF29
:109DF000C4F30310FFF748FF04F00F00FFF744FF20
:109E000010BD000010B540210248FCF7B0FA02F086
:109E100087F910BD000C014010B540210248FCF745
:109E2000A4FA02F07DF910BD000C014010B58021AC
:109E30000748FCF79CFA80200649088003208870B8
:109E40000420C8700248FCF70DFA02F069F910BD51
:109E5000000C01402C01002010B58020074908802B
:109E6000032088701420C8700548FCF7FBF9802196
:109E70000348FCF77AFA02F053F910BD2C010020D8
:109E8000000C01407047704770477047704710B52D
:109E90000446204600F00EF810BD70B505460E468B
:109EA000002403E0285D00F005F8641CB442F9D3F7
:109EB000012070BD2DE9F04105462E460024002703
:109EC00025E006F0800028B94FF480511248FCF7D5
:109ED0004CFA04E04FF480510F48FCF748FA700642
:109EE000060E4FF480610C48FCF741FA6006040E40
:109EF0004FF400610848FCF72AFA08B144F0010465
:109F00004FF480610448FCF730FA781CC7B2082F80
:109F1000D7DB2046BDE8F08100100140014609B1C1
:109F2000102001E04FF48010014A106001207047BA
:109F3000100801402DE9F04104460D46164605F192
:109F40008600FEF791FE80460C4850F8240098B930
:109F500016B9601CFEF782FB05F17000FEF784FE67
:109F6000C0EB001106FB08F0C0EB8107474500DAA3
:109F70004746024840F82470BDE8F081E80B002015
:109F80000021024A42F8201070470000E80B002030
:109F90002DE9F84F05460C46164604F18600FEF7FB
:109FA00063FE81466B20FEF75FFE009004F16D00BA
:109FB000FEF75AFE83461E480068584535DB1D48AB
:109FC00050F8250088BB04F17100FEF74DFE824673
:109FD00004F17000FEF748FE074600985844144903
:109FE0000968884206DC06FB09F0CAEB0A11C0EBDF
:109FF000810810E00E480068A0EB0B00AAEB0701F7
:10A000004843009990FBF1F03844C0EB001106FB87
:10A0100009F0C0EB8108C84500DAC84616B9681CCB
:10A02000FEF71CFB034840F82580BDE8F88F0000D0
:10A0300034000020E80B00202DE9FC5F05460E46A9
:10A04000174606F18600FEF70FFE82466B20FEF7EC
:10A050000BFE019006F16E00F7F726FE00900098C7
:10A0600000283DD006F16D00FEF7FEFD04461D48B8
:10A070000168A14234DB1C4850F8250080BB0099E0
:10A08000C81CFEF7F1FD83460099881CFEF7ECFD25
:10A0900081460198204413490968884206DC07FB81
:10A0A0000AF0CBEB0B11C0EB81080FE00D48006804
:10A0B000001BABEB09014843019990FBF1F04844C8
:10A0C000C0EB001107FB0AF0C0EB8108D04500DAB5
:10A0D000D04617B9681CFEF7C1FA034840F825803E
:10A0E000BDE8FC9F34000020E80B00202DE9F0477C
:10A0F00004460D46164605F18600FEF7B5FD80467E
:10A1000005F16E00F7F7D0FD8146B9F1000F17D0C9
:10A110000C4850F8240098B916B9601CFEF79EFA56
:10A1200009F10200FEF7A0FDC0EB001106FB08F0EC
:10A13000C0EB8107474500DA4746024840F82470E3
:10A14000BDE8F087E80B002070B502460020002330
:10A1500017E000EB40042F4D55F82440944206D1FF
:10A1600000EB400405EB840464688C4206D000EBED
:10A170004004284D05EB8404A4680CB9012300E0D9
:10A18000401C192801DA002BE3D00BB300EB40048C
:10A19000204D05EB8404A468022C1AD11E4C2468BF
:10A1A000B4B900EB400445F8242000EB400405EB73
:10A1B00084046160012400EB4005164E06EB850522
:10A1C000AC60164C2468112C22D10124144D2C7043
:10A1D0001EE000EB40040F4D05EB8404A468012C45
:10A1E00016D000EB400445F8242000EB400405EBBA
:10A1F00084046160012400EB4005064E06EB8505F2
:10A20000AC60064C2468112C02D10124044D2C7042
:10A2100070BD0000100C0020A4000020D00200201F
:10A220003F01002010B50446FEF7EEFBFEF708FDE7
:10A23000C4EB04118800FEF7E3FCFEF701FD4AF2CF
:10A24000A5510420F7F7AAFAFEF752FC3C21B0FB17
:10A25000F1F00149086010BD3000002070B50446DF
:10A260000D4600F03CFE04F03F0000F14002A11159
:10A27000002000F029FF00F032FE05F1B802A11124
:10A28000002000F021FF00F02AFEC0220021084635
:10A2900000F01AFFC0220121002000F015FF70BD60
:10A2A00070B50025202600216C20FCF74DF92148CF
:10A2B000006800283DD14FF496701E4908600024C4
:10A2C0001CE004EB44001C4901EB8000406898B19D
:10A2D00004EB440001EB80008068022802D1012DCC
:10A2E00000DA012504EB4400134901EB800080688B
:10A2F000012802D1022500E01924641C192CE0DB9E
:10A30000012D02D0022D0ED101E096260BE00B4864
:10A31000007820B9962601200849087002E0002044
:10A320000649087000BF00BF012231461046FEF703
:10A330008DF870BDC8020020100C0020F40200202F
:10A3400010B5FCF79BFDFCF7DDFD0020044908700B
:10A3500004490870012204A1104600F0A7FF10BDB7
:10A3600035010020360100202020204452414D4D6F
:10A37000202020200000000070B504460D4616463F
:10A3800005490D7005490C7006F1AD01002210461B
:10A3900000F038FF70BD00003601002035010020BC
:10A3A0002DE9F0412148006800283CD14FF4AF70FE
:10A3B0001E4908601E48007818B901201C49087021
:10A3C00002E000201A4908704FF4BD70FEF74CFC03
:10A3D0000446012C01DA3C2604E03C2090FBF4F01A
:10A3E000801EC6B200251CE012480068401EA8422C
:10A3F00004D10F48007808B9E32700E0DF27C5EB58
:10A400000510C00090FBF4F000EB06080721404661
:10A41000FCF79AF8002239461046FEF717F8681C38
:10A42000C5B2A542E0DBBDE8F081000038010020A4
:10A43000F60200203800002070B5FCF763FD002014
:10A440004249087042490870012242A1104600F0BA
:10A450002DFF10203D49087004203D49087000225E
:10A4600040A1104600F022FF062039490870222042
:10A47000364908706420FEF7F7FB04460022562197
:10A480001046FDF7E3FF3B4894FBF0F03030C5B2D7
:10A49000002229461046FDF7D9FF42F2107094FBC6
:10A4A000F0F00A2190FBF1F201FB12003030C5B24E
:10A4B000002229461046FDF7C9FF00222E21104632
:10A4C000FDF7C4FF4FF47A7094FBF0F00A2190FB83
:10A4D000F1F201FB12003030C5B2002229461046CD
:10A4E000FDF7B4FF642094FBF0F00A2190FBF1F239
:10A4F00001FB12003030C5B2002229461046FDF79C
:10A50000A5FF00222E211046FDF7A0FF0A2094FB94
:10A51000F0F00A2190FBF1F201FB12003030C5B2DD
:10A52000002229461046FDF791FF0A2094FBF0F126
:10A5300000FB11403030C5B2002229461046FDF71D
:10A5400085FF42F210700C49086070BD3501002093
:10A55000360100202020204452414D4D2020202053
:10A56000000000002020204D6973742D54696D6532
:10A5700020202000A08601001400002070B50446B1
:10A5800000256720FEF770FB06283FD2DFE800F0C9
:10A59000030C16202A3404EB44011E4A52F8310001
:10A5A000F6F71EF8054631E004EB4401194A02EBC8
:10A5B000C1014868F6F714F8054627E004EB4401AA
:10A5C000144A02EBC1018868F6F70AF805461DE057
:10A5D00004EB44010F4A02EBC101C868F6F700F82A
:10A5E000054613E004EB44010A4A02EBC101086985
:10A5F000F5F7F6FF054609E004EB4401054A02EBD6
:10A60000C1014869F5F7ECFF054600BF00BF2846C9
:10A6100070BD0000F446020810B500F035F810BD1A
:10A620004FF0E021012804D0801C06D00020886172
:10A630007047086940F0010002E0086920F001005D
:10A64000086170474FF0E0210028086902D040F00F
:10A65000020001E020F002000861704710B541F6E9
:10A660006A0000F00DF80120FFF7ECFF0120FFF772
:10A67000D7FF14200149086010BD0000140000201D
:10A680004FF0E0214861704710B54E48006820B196
:10A690004C480068401E4B4908604B48006828B190
:10A6A00049480068401E4849086003E04FF47A704A
:10A6B000454908604548007870B143480068C821A2
:10A6C00090FBF1F201FB1200642805DD4FF480716C
:10A6D0003F48FBF74CFE04E04FF480713C48FBF729
:10A6E00044FE3C48006820B13A480068401E3949A1
:10A6F00008603948006820B137480068401E364974
:10A7000008603648006820B134480068401E33496C
:10A7100008603348006820B131480068401E304965
:10A7200008603048006820B12E480068401E2D495E
:10A7300008602D48007820B12B480078401E2A4937
:10A7400008702A48007820B128480078401E274920
:10A7500008702748007820B125480078401E244919
:10A7600008702448007820B122480078401E214912
:10A7700008702148006828B11F480068401E1E4923
:10A78000086002E000201D4908701D48006828B1DB
:10A790001B480068401E1A49086002E00020194961
:10A7A00008701948006820B117480068401E164913
:10A7B00008601648006820B114480068401E13491C
:10A7C000086010BD2001002014000020D8000020E7
:10A7D00000080140180000209C030020A403002072
:10A7E000A8030020A003002000000020010000209A
:10A7F0000200002003000020FC0000200B010020CC
:10A80000900300205203002038010020C8020020DD
:10A810007047704770477047704770477047704780
:10A820007047704770477047704770477047000027
:10A830002DE9F0419948007808B1FCF71DFF002090
:10A840009649087000212820FBF77EFE0123002294
:10A85000934801681846FDF7B9FA4FF4C170FEF746
:10A8600003FA40B303210846FBF76EFE00221E21C7
:10A87000104600F0C7FC8B480068FBF7D4FA80460E
:10A8800000231A4641461846FDF7D0FB40F27B10E4
:10A89000FEF7EAF928B900221146104600F0B2FC92
:10A8A00004E000220F21104600F0ACFC0022202121
:10A8B0001046FDF7CBFD04210320FBF745FE7A4847
:10A8C0000068002875D00022B321104600F09AFCE1
:10A8D00076480078801E75490870734800680B2818
:10A8E0004DD2DFE800F04C060D141B222930373E14
:10A8F0004500002240F287111046FCF748FF3EE079
:10A9000000224FF4C4711046FCF741FF37E00022EB
:10A9100040F289111046FCF73AFF30E000224FF474
:10A92000C5711046FCF733FF29E0002240F28B117D
:10A930001046FCF72CFF22E000224FF4C6711046AF
:10A94000FCF725FF1BE0002240F28D111046FCF7BA
:10A950001EFF14E000224FF4C7711046FCF717FFEA
:10A960000DE0002240F28F111046FCF710FF06E0C8
:10A9700000224FF4C8711046FCF709FF00BF00BF6A
:10A98000002220211046FDF761FD48480078801E16
:10A990004649087046480068062823D2DFE800F0E0
:10A9A00022030A10161C0022B521104600F02AFCD2
:10A9B0001EE01EE00022B621104600F023FC17E046
:10A9C0000022B721104600F01DFC11E00022B82142
:10A9D000104600F017FC0BE00022B921104600F0F1
:10A9E00011FC05E00022B521104600F00BFC00BF71
:10A9F0000DE03048006828B10022BA21104600F06E
:10AA000001FC04E00022BB21104600F0FBFB04E047
:10AA1000002220211046FDF719FD244800787828EF
:10AA2000F6DD4FF4BD70FEF71FF90446092C01DD79
:10AA3000092600E0E6B2012C01DA3C2704E03C20C4
:10AA400090FBF4F0401EC7B2002513E0C5EB0510E3
:10AA5000C00090FBF4F000EB070806214046FBF72E
:10AA600073FD05F13100C1B200221046FDF7EEFC86
:10AA7000681CC5B2B542E9DB0A2C0DD106216E2057
:10AA8000FBF762FD002231211046FDF7DFFC0022BA
:10AA900030211046FDF7DAFCBDE8F0813F010020CF
:10AAA0003000002034000020380000203501002054
:10AAB0003C0000208C000020704770477047000069
:10AAC00070B540F227711E4800F0AAF8C8B11D48C1
:10AAD00000681D49096888420CD01B480068401C6A
:10AAE000C0F30A041948015D154800F01BF9164827
:10AAF000046005E0002240F22771114800F0AFF831
:10AB000000BF40F225510E4800F08AF8B8B10C4859
:10AB100000F004F9C5B20E480068401CC0F30A04F6
:10AB20000B4804600B480068844202D101200A49A6
:10AB300008700A48055564200949086000BF70BDC7
:10AB400000440040180100201C010020FC170020D8
:10AB500010010020140100200C010020FC0F002037
:10AB6000FC00002070B540F227711F4800F058F833
:10AB7000C8B11E4800681E49096888420CD01C48AC
:10AB80000068401C00F01F041A48015D164800F0E0
:10AB9000C9F81748046005E0002240F22771124806
:10ABA00000F05DF800BF40F225510F4800F038F882
:10ABB000C0B10D4800F0B2F8C5B20F480068401CA3
:10ABC000C0F308040C4804600C480068844202D1B9
:10ABD00001200B4908700B4805554FF47A700A495B
:10ABE000086000BF70BD000000480040480300201E
:10ABF0004C03002088310020400300204403002043
:10AC000053030020882F0020900300200029818911
:10AC100002D041F4005101E021F4005181817047DC
:10AC200070B501F01F0601220025C1F3421302FA9C
:10AC300006F4012B0FD0022B0FD0838A4FEA11218B
:10AC40000088234202FA01F200EA020001D000B1BA
:10AC50000125284670BD8389F0E7038AEEE710B529
:10AC6000C1F3421301F01F040121A140012B07D0C1
:10AC7000022B07D01430002A026805D00A4304E0F2
:10AC80000C30F8E71030F6E78A43026010BD000090
:10AC900030B50446008A85B00D464CF6FF71084079
:10ACA000E98801432182A1894EF6F3100140A8886A
:10ACB0002A8910436A890A431043A081A08A4FF66B
:10ACC000FF410840A9890143A1826846FDF79CFD28
:10ACD0001148844201D1039800E00298642200EBFD
:10ACE000C00101EB001029686FF018058900B0FB66
:10ACF000F1F0B0FBF2F109010B096B4300EB8300AB
:10AD0000322303EB0010B0FBF2F000F00F00084319
:10AD1000208105B030BD0000003801408088C0F3BC
:10AD200008007047C1F30801818070477047704781
:10AD300070470120704700002D2802D08D2842D195
:10AD40002EE022490968042914DA20490968491CBF
:10AD50001E4A11601E490968126811441D4A02EB1F
:10AD600001110968491CD1B918490968491E174AD7
:10AD7000116014E016490968491C154A1160114612
:10AD80000968124A12681144124A02EB011109685B
:10AD9000491C21B90E490968491E0D4A116012E08B
:10ADA0000A49096829B109490968491E074A116019
:10ADB00008E007490968002904DD05490968491EBA
:10ADC000034A116000BF00BF70470000300100203F
:10ADD000BC020020582C00204FF6FF72904216D083
:10ADE00042F21072904212DB520090420FDA084A8F
:10ADF0001278521CD1B2142900DB0021054A1278C6
:10AE0000914204D0044A42F82100014A117070476F
:10AE10002500002024000020E003002000BFFEE702
:10AE200070B502460020002317E000EB4004174DE8
:10AE300055F82440944206D100EB400405EB84040D
:10AE400064688C4206D000EB4004104D05EB84048E
:10AE5000A4680CB9012300E0401C192801DA002B7A
:10AE6000E3D093B100EB4004084D05EB8404A468E3
:10AE7000012C0AD1022400EB4005044E06EB8505A7
:10AE8000AC604FF49674024D2C6070BD100C002025
:10AE9000A400002010B50D4A12680D4B1B681A441F
:10AEA00002EB42020B4B03EB82025168074A126825
:10AEB000074B1B681A4402EB4202064B53F8220070
:10AEC000FFF7AEFF01200449087010BD0803002001
:10AED00030010020100C00203F010020704770B5A9
:10AEE00000BF00210846FDF753FFC5B20121002035
:10AEF000FDF74EFFC4B2802D02D00DB1FCF702F871
:10AF0000802C02D00CB1FBF7FDFF05F0800000287B
:10AF1000E7D104F080000028E3D170BD10B515E042
:10AF2000FBF732FB0D480068C82190FBF1F201FBF2
:10AF30001200642805DA4FF480610948FBF717FA1C
:10AF400004E04FF480610648FBF70FFA03480068FD
:10AF500018B1FDF7D5FE0028E2D010BD1400002086
:10AF6000000C01402DE9F04107460D4690461C4675
:10AF7000069E01201A490870E2B220210020FDF748
:10AF800065FA042016490870E2B220210020FDF77E
:10AF90005DFA012D02D0022D0CD105E0E2B2BC21F8
:10AFA000002000F02FF905E0E2B2BD21002000F002
:10AFB00029F900BF00BF04E0E2B220210020FDF724
:10AFC00045FA074800787828F6DB772004490870AE
:10AFD000E2B220210020FDF739FABDE8F08100003F
:10AFE0003501002070B505460C462846FDF73CFEAD
:10AFF000A04209D02946204600F0C0F82846FAF7BA
:10B0000053FF0646FFF7E8FE70BD00002DE9F04152
:10B0100005460C4616461548854225DA2846FAF7B5
:10B020005FFF0746FBF740FEA0B12846FBF7E4F9B7
:10B030000746FDF719FEA04216D02846FBF7DCF9BB
:10B0400007463946204600F099F86EB12846FFF7CA
:10B05000C3FE09E02846FAF743FFC0EBC0000449ED
:10B0600001EB800040680460BDE8F08178D4030003
:10B0700038E901082DE9F04105460F4616464FF420
:10B08000C970FDF7F1FD0446002C01DB322C00DD18
:10B09000002404F293102946FFF7A4FF04F2C51020
:10B0A0003946FFF79FFF04F2F7103146FFF79AFF8A
:10B0B000641C322C00DB002421464FF4C970FFF7DA
:10B0C00091FFBDE8F0810000F8B505460E46174631
:10B0D0004FF480412648FBF748F925B980212548DF
:10B0E000FBF743F903E080212248FBF740F926B142
:10B0F00040212148FBF73BF904E04FF400411C4894
:10B10000FBF735F920211A48FBF731F94FF47F405E
:10B11000ADF8000010208DF8030003208DF8020028
:10B1200069461448FBF79EF81248FBF70DF90446F0
:10B13000E4B244EA0724A1B20E48FBF71AF9202131
:10B140000B48FBF712F940210B48FBF70EF94FF4BF
:10B1500000410748FBF709F94FF47F40ADF80000C4
:10B1600028208DF8030069460248FBF77BF8F8BDFC
:10B17000000C014000180140000801402DE9F04793
:10B18000074688464FEA8806C6F3074AB6B23D46E8
:10B190004FF0030903F0BEF900BF002431465046CA
:10B1A00003F0FAF9A0B1280E03F078FA044624B1AE
:10B1B000C5F3074003F072FA044624B1C5F3072033
:10B1C00003F06CFA04461CB1E8B203F067FA0446D7
:10B1D00003F0C4F824B9A9F1010000F0FF0901E06F
:10B1E0004FF00009B9F1000FD7DC03F089F90448EA
:10B1F0000068401C024908602046BDE8F087000056
:10B200002401002070B505460C4616466720FDF760
:10B210002BFD062845D2DFE800F0030D18232E3958
:10B2200004EB4400204A52F830103246284600F021
:10B230003DF836E004EB44001B4A02EBC000324606
:10B240004168284600F032F82BE004EB4400164A2F
:10B2500002EBC00032468168284600F027F820E063
:10B2600004EB4400104A02EBC0003246C168284695
:10B2700000F01CF815E004EB44000B4A02EBC000A0
:10B2800032460169284600F011F80AE004EB440058
:10B29000054A02EBC00032464169284600F006F834
:10B2A00000BF00BF70BD0000F44602082DE9F04168
:10B2B00006460C46174666E0207823285DD1641CBC
:10B2C0002078A0F13005641C207805EB850100EBA7
:10B2D0004100A0F13005641C0B2D4DD2DFE805F0D4
:10B2E0004C060D141B222930373E45003A4640F2E9
:10B2F00087113046FCF74BFA3EE03A464FF4C471F2
:10B300003046FCF744FA37E03A4640F289113046BD
:10B31000FCF73DFA30E03A464FF4C5713046FCF791
:10B3200036FA29E03A4640F28B113046FCF72FFA04
:10B3300022E03A464FF4C6713046FCF728FA1BE08B
:10B340003A4640F28D113046FCF721FA14E03A46B5
:10B350004FF4C7713046FCF71AFA0DE03A4640F256
:10B360008F113046FCF713FA06E03A464FF4C871E5
:10B370003046FCF70CFA00BF05E014F8011B3A4612
:10B380003046FDF763F82078002895D1BDE8F081BC
:10B390002DE9F04107460C4615461E461148007837
:10B3A00038B104F13000C1B232463846FDF74EF8EC
:10B3B00016E07CB101200B49087032462D21384639
:10B3C000FDF744F804F13000C1B232463846FDF7CB
:10B3D0003DF805E025B1324620210020FDF736F882
:10B3E000BDE8F0813401002070B504461148AFF388
:10B3F0000080114904EBC40001EB80040026208882
:10B400004FF0FF358107002906D00ADA8006204672
:10B4100004D501F072F903E02C4604E000F0ECFEE4
:10B4200030B1268000240348AFF30080204670BD71
:10B430002680F1E7000000003C26002010B50446FD
:10B440000C48AFF300800C4904EBC40001EB80040E
:10B450002088810703D0800603D5A46805E0002476
:10B4600003E0204600F0C1FE64680248AFF30080AC
:10B47000204610BD000000003C2600202DE9F843C6
:10B4800006460F466648AFF30080684601F048FC68
:10B4900004004FF0FF3575D00146304601F08EFCB8
:10B4A000814620690028F6D017F00C0004D004284B
:10B4B0000AD0082866D103E0208840F0010006E0A9
:10B4C000208840F004002080208840F00200208086
:10B4D00017F0060F04D0484601F010FC002851D1A7
:10B4E0002088DFF8408180064FF000064BD52146CA
:10B4F000484600F015FF012803D02088C00772D10C
:10B5000033E000214848C4461BE000BFB0F800808B
:10B510005FEA887213D0026923699A420FD1A04270
:10B520000DD0C28AE38A9A4209D1026A236A9A42FA
:10B5300005D15FEA887270D4228892076DD4491CC5
:10B540002430BCF800209142E0DB208810F0050F89
:10B5500006D0B9075AD500BF40F00B00208055E057
:10B560002146484600F077FEE8B3208810F0060F29
:10B5700004D02146484600F043FEA0B3B80745D5A5
:10B580002088E9E743E0B80741D42146484600F067
:10B590002AFE012803D02088C0073ED130E00021D8
:10B5A0002148424617E000BFB0F800C05FEA8C7344
:10B5B0000FD003692769BB420BD1A04209D0838A0F
:10B5C000A78ABB4205D15FEA8C7326D423889B07E8
:10B5D00023D4491C243013889942E5DB2088410795
:10B5E00005D5204600E018E000F0FFFD0EE0C007A2
:10B5F00002D0E069206209E0204600F0F0FD60B171
:10B60000A6822146484600F0E8FD30B1009D04487E
:10B61000AFF300802846BDE8F8832680F7E70000F6
:10B62000000000009C4602083C2600202DE9F04165
:10B6300007460E4615461348AFF3008045F0004418
:10B64000CEB1114907EBC70001EB800001888A07E2
:10B6500011D001F00F02022A06D089062A4631468F
:10B6600005D500F06BFF04E04FF0FF3403E000F07D
:10B67000BDFD00B12C1A0348AFF300802046BDE8A1
:10B68000F0810000000000003C26002070B5044658
:10B690000D460E48AFF300800D4904EBC40001EBEA
:10B6A00080004FF0FF3401888A070AD089062946B6
:10B6B00002D500F0E5FF01E000F09CFD012800D17B
:10B6C00000240248AFF30080204670BD0000000057
:10B6D0003C2600202DE9F04107460D46164611484C
:10B6E000AFF300804FF0FF34B5B10F4907EBC7004F
:10B6F00001EB800001888A070ED001F00F02012AB9
:10B700000AD089063246294602D501F071F801E0D7
:10B7100000F074FD00B100240248AFF30080204621
:10B72000BDE8F081000000003C26002030380A28E7
:10B7300001D2012070470020704710B50446B4F5CF
:10B74000004F01DD002010BD2046FFF74DFEFAE757
:10B7500000BFFEE710B50446B4F5004F01DD002040
:10B7600010BD2046FFF76AFEFAE70146B1F5004F2B
:10B7700001DD012070470020FCE7000070B50446A1
:10B780000D460EA12046F5F717F810B948F2010052
:10B7900070BD0CA12046F5F70FF810B948F2020071
:10B7A000F6E70AA12046F5F707F810B948F20300BA
:10B7B000EEE729462046FFF761FEE9E75354444986
:10B7C0004E0000005354444F555400005354444518
:10B7D000525200002DE9F04104460D4616461F4620
:10B7E000B4F5004F03DD4FF0FF30BDE8F081324685
:10B7F00029462046FFF71AFFF7E770B504460D46C5
:10B80000B4F5004F02DD4FF0FF3070BD29462046F1
:10B81000FFF73CFFF9E72DE9F04104460D461646D7
:10B820001F46B4F5004F03DD4FF0FF30BDE8F08157
:10B83000324629462046FFF74DFFF7E770470000E4
:10B840000021094A1268094B1B68D01800E0491C06
:10B85000074A02EB01121268521C002AF7D18842F3
:10B8600000DB401A70470000BC02002030010020BD
:10B87000582C00202DE9F84F05464FF00009C86903
:10B8800000900C460127C8464E46284600F0E9F8CD
:10B89000012808D12846F4F7A3FE0C300D21B0FB97
:10B8A000F1F0401CC7B22069009901F052FB8246BA
:10B8B0000025206990F87B1019B1B5F5007F56D0AE
:10B8C0002AE0818FA94227D1016C009A002591427C
:10B8D00000D900916946009E02F0CCFC002847D0B8
:10B8E0002069009901F04AFE88B10096012269465C
:10B8F000206900F048F800283AD02069009900F04B
:10B9000043F9002834D04FF00008009E34E020694D
:10B91000009900F05BF982460AEB1511206902F0EC
:10B9200033FB002824D02069C16D05F00F0001EB26
:10B930004010007838B1FF2805D0E52803D04FF03B
:10B9400000096D1CB5E7B9F1000F02D1009E1FFA86
:10B9500085F809F10101C9B28946E5280AD02069B4
:10B9600090F87B0040B1C7F50070A84204D20020D7
:10B97000BDE8F88FB942E4D12169A1F87880206947
:10B9800046670120F4E72DE9F041154607460C46CD
:10B990000E6801F00DFB002818D0384601F059FA66
:10B9A00002463846216802F007FF00280ED035B164
:10B9B00031463846226802F0FFFE002806D00021FA
:10B9C000384600F005F8002800D00120BDE8F081DD
:10B9D00070B50446806C0D46A8423ED094F85010D5
:10B9E000012928D166697EB1216889060CD5617F5D
:10B9F000022906D0002201463046E36C01F027FA06
:10BA000014E0218C4218F6E76268E16CD3680122E9
:10BA10009847002820D0607F022809D16268218CD5
:10BA2000A06CD3680844E16C01229847002813D029
:10BA3000002084F8500085B194F85100218C626890
:10BA4000484328449368E16C01229847012806D0B6
:10BA50004FF0FF30A064002070BD012070BDA564D0
:10BA6000FBE72DE9F04100270446B8463D463E4637
:10BA700025E002F027FD38B32078202824D02E2896
:10BA800014D0A0F16101192902D92031192907D850
:10BA9000B8F1000F03D088EA0001890614D480466B
:10BAA0004FB13046761C02280ED806E067B9641CF8
:10BAB0000026012703E0082D06D26D1C641C2078A7
:10BAC0000028D6D10C2D02D30120BDE8F081002042
:10BAD000FBE7012302F0BEBAF8B5C1690446009144
:10BAE00000293DD0206900F071F807460025206943
:10BAF000818FA9420FD10025694602F0BBFB0028C7
:10BB00002FD02069009901F039FD58BB20690099B8
:10BB100000F05CF8074607EB1511206902F034FAD3
:10BB200000281ED0206905F00F01C06D00EB411602
:10BB300030782E2809D10CA13046F4F73DFE68B1CB
:10BB40000DA13046F4F738FE40B1307850B1E52809
:10BB500004D0F07A0F2803D0000701D56D1CC6E78A
:10BB60000020F8BD0120F8BD2E202020202020201C
:10BB700020202010000000002E2E20202020202039
:10BB8000202020100000000070B5054600F01EF8CF
:10BB900006464FF40071E86DF4F7C4FD002406E09A
:10BBA0003119284602F02CFD00280AD0641CA87F19
:10BBB000A042F5D80021284602F022FD002800D03E
:10BBC000012070BD10B5FBF759F910BD838E826955
:10BBD0001A44037F032B01D0C38E1A44807F891E31
:10BBE00000FB012070472DE9F0410446007F00254D
:10BBF000012806D0022838D0032857D00020BDE8FD
:10BC0000F08102262CE03146204601F0B8F980464A
:10BC100001462046FFF7DCFE002867D006EB460011
:10BC2000C0F34800B0F5FF7F04D8E16C084401F090
:10BC30002DFC0CE0E06C08F1010190F8FF7120464A
:10BC4000FFF7C6FE88B3E06C007847EA0020F107F2
:10BC500001D0000901E0C0F30B0000B96D1C761C97
:10BC6000206B801CB042CED840E00221204601F07B
:10BC700086F9074601462046FFF7AAFEA8B102262C
:10BC80000FE016F0FF0F05D17F1C39462046FFF765
:10BC90009FFE50B1E06CF1B230F8110000B96D1C9C
:10BCA000761C206B801CB042EBD81FE0022120469E
:10BCB00001F065F9074601462046FFF789FEA8B165
:10BCC00002260FE0700605D17F1C39462046FFF79B
:10BCD0007FFE58B1E06C06F07F0150F8210000B9FA
:10BCE0006D1C761C206B801CB042EBD8284686E782
:10BCF0002DE9F04389B00E46904699460546FFF778
:10BD0000B0FE88B301271B4C1CE04246314604A814
:10BD1000FFF7DFFE28B1A74214D9002009B0BDE823
:10BD2000F083694604A800F0ACF90028F6D0684614
:10BD300001F040FC02463146284600F01DF800287C
:10BD4000ECD007E03A467F1C04A9284601F0BEFA71
:10BD50000128DAD04B4642463146684600F0B0F83A
:10BD60000028DBD00120D9E7FFE76946284600F02C
:10BD700088F9E4E73E420F002DE9F74F086982B0E9
:10BD80000C46416F0091B0F878504FF0000B0298CC
:10BD9000F4F726FC81462069009901F0DAF8824622
:10BDA000D846464E7DE0206990F87B1031B1B5F55C
:10BDB000007F1DD1002005B0BDE8F08F818FA94222
:10BDC00016D1016C009A0025914200D90091012200
:10BDD0006946FFF7D8FD0028EDD020690099FFF7EC
:10BDE000D3FE0028E7D020690099FFF7EFFE8246D6
:10BDF0000AEB15110191206902F0C6F80028DAD08B
:10BE0000206905F00F010D22C06DBBF1000F00EBA2
:10BE1000411109F10C00B0FBF2F0C0B2087001D082
:10BE2000002200E0402210430870049A4A73A1F8EF
:10BE30001A800F2200F01F00CA72401E00EB800221
:10BE400002EBC000029A4FF0010B131800204A1CAD
:10BE50001F5C4FB116F800C001F80C70375C401C35
:10BE60000D2807F80280F3D3002305E0375CCB559B
:10BE7000375CBB54FF23401C0D28F7D3B9F10C0FDE
:10BE800002D9A9F10D0000E000208146E843000737
:10BE900006D101222069019902F036FD00288AD0DE
:10BEA0006D1CB9F1000F7FF47EAF216900984867DF
:10BEB0002069A0F8785001207DE70000764E030845
:10BEC0002DE9FC5F06460D469A46012A0DD000205A
:10BED00081462869416F0091B0F8787090F87B2016
:10BEE00042B1B7F5007F02D018E00120F0E7002052
:10BEF000BDE8FC9F828FBA4210D1026C00278A42B3
:10BF000000D9009201226946FFF73DFD0028EFD0DD
:10BF100028690099FFF738FE0028E9D028690099C0
:10BF200001F017F800EB17118B46286902F02CF886
:10BF30000028DDD0286907F00F01C06D00EB411427
:10BF40000020315C2154401C0B28FAD35FEA0A0020
:10BF50004FF0000837D00646C07AE07284F80C80B3
:10BF600084F80D80F089E081308A208200F0DBFFC8
:10BF7000014604F1120002F0C3F9B08AA08201F078
:10BF80006DFA014604F1160002F0BAF9608A2083C6
:10BF9000708B6083F069E061F0696860F069C5E901
:10BFA000020806F11A0001F071FA044606F11400C5
:10BFB00001F06CFA04EB0040E8610122594628695F
:10BFC00002F0A2FC56E084F80C8084F80D8001F0A9
:10BFD00045FA014604F10E0002F092F900F0A3FFC9
:10BFE000014604F1100002F08BF9208A6082E18999
:10BFF000E1822083C4F81C80C5F80C80C5F8048059
:10C00000C5F80880B9F1000F1ED01020E072009929
:10C0100001912869006C884200D90190002201A991
:10C020002869FFF7B0FC00283FF462AF0198E8618F
:10C03000010C04F1140002F063F9019881B204F1DB
:10C040001A0002F05DF907E02020E072A4F81480E5
:10C05000A4F81A80C5F81C8001225946286902F00C
:10C0600053FC0028E0D0B9F1000F05D028690199F0
:10C07000FFF78AFD0028D7D0EF82009828620120C0
:10C0800036E72DE9F041002704460D4638462021C9
:10C090002954401C0B28FBD30021295420786178B7
:10C0A000A2782E2806D111B12E2902D002E02870E4
:10C0B00031E0AAB10026207868B32E2813D02028BA
:10C0C0000AD002F0F6F9A0F16101A855192902D8A9
:10C0D00020F02000A855761C641C082EEBD304E049
:10C0E0002870687017E00127641C0826207890B13A
:10C0F0002E2813D020280BD057B102F0DAF9A0F186
:10C100006101A855192902D820F02000A855761CF5
:10C11000641C0B2EEAD30120BDE8F0810127F7E76C
:10C120000649096809B9052101E04FF4FA6108469A
:10C1300000BF011EA0F10100FBD1704728010020C3
:10C140002DE9F8430546006990F87A60416F009147
:10C15000B0F8784000F0FDFE07463AE0286990F814
:10C160007B1029B1B4F5007F15D10020BDE8F8831C
:10C17000818FA1420FD1016C009A0024914200D915
:10C180000091694602F076F80028EFD028690099FE
:10C19000FFF71CFD074607EB14118846286901F0DC
:10C1A000F3FE0028E2D0286904F00F01761EC06D6E
:10C1B000F6B200EB4110E5210170E043000700D02A
:10C1C00036B901224146286902F09EFB0028CDD0F5
:10C1D000641C002EC2D10120C8E700207047002057
:10C1E000704700207047002070477047002070475C
:10C1F00000207047002070470020704700207047E3
:10C2000070B505460C460869142100F049FD002868
:10C2100020D028785C2800D16D1C2878002819D0FF
:10C220000020E06101222146284600F09FF8002806
:10C2300010D0206921467C30FFF71CFB002809D074
:10C24000206900237C301A462146FFF751FD002863
:10C2500000D0012070BD70B505460C460869142158
:10C2600000F01EFD002838D028785C2800D16D1C15
:10C270002878002831D000200246E0612146284677
:10C2800000F074F8002828D0206990F87C1029B1BB
:10C290007C300022214600F01DFC02E02046FFF722
:10C2A0001BFC002819D02046FFF74AFF002814D0B5
:10C2B000E169206902F060F800280ED02069017F52
:10C2C000032909D102F0ECFA002806D000212069E8
:10C2D00002F096F9002800D0012070BD70B5044628
:10C2E0000E4615460421106900F0DAFC002816D02D
:10C2F00020785C2800D1641C207800280FD0002012
:10C300000246E8612946204600F030F8002806D0B1
:10C310002946304600F0FAFE002800D0012070BD0A
:10C3200070B505460C460869042100F0B9FC0028E8
:10C330001BD028785C2800D16D1C2878002814D0E8
:10C340000026324621462846E66100F00FF8002814
:10C350000BD0206900227C30214600F0BBFB002876
:10C3600003D06675E069A061012070BD2DE9F0473A
:10C37000002706460D469146B84620E0286901226E
:10C380007C30294600F0A6FBC0B95FEA09002DD039
:10C390000127286929467C30FFF76CFA002825D050
:10C3A000286900237C3001222946FFF7A1FC0028E0
:10C3B0001CD0284602F07EF9002817D026442969AF
:10C3C0007C3100242046325D5C2A06D0222A04D02B
:10C3D0004AB10A54401C641CF5E7641C01F8008053
:10C3E000002FD6D1CAE701F800800120BDE8F08710
:10C3F0002DE9F0414FF0FF3500F148048564806875
:10C4000060604FF000062672667200F5007100F55C
:10C410008060E560C4E90510267766774FF0020872
:10C42000C4F82480A4F148044FF0300104F118004E
:10C43000F4F79AF90021204601F0A6FD08B3E06D5B
:10C4400000F5FF7001F022F8A0F52A41553918D106
:10C45000E06D0178E9290AD0EB2902D18178902991
:10C4600005D000F5E37001F016F8A06100E0A661C8
:10C47000204600F000FD38B1E18DB1F5007F40D1DC
:10C4800004E00220BDE8F0810320FBE7A07F08283C
:10C490000DD006DC01280AD0022808D0042830D1AB
:10C4A00005E0102803D0202801D0402829D1B4F875
:10C4B00022C0BCF1000F24D0627F012A01D0022AE1
:10C4C0001FD1238C666AB3421BD8A78D02FB03C31E
:10C4D00005EB471505F5007595FBF1F15A18B21AF1
:10C4E000A262B2FBF0F22263A386E1864002A0635F
:10C4F0004009A08740F6F570824204D201202077DF
:10C5000016E00420BEE74FF6F570824202D284F8AE
:10C510001C800DE003202077204600F0B7FD38B9DD
:10C520002046FFF760FBA066204602F0B9F908B18B
:10C530000020A7E70520A5E7012070472DE9F04777
:10C540000446008889461746C00613D40421206992
:10C5500000F0A6FB50B1E068A168C2198A4201D977
:10C560000F1A07D0C0F3080600253AE0208840F0F3
:10C57000100020800020BDE8F087A1692069FFF746
:10C5800025FB627D81182069837F9A1A01F0A4FC43
:10C590000028F0D0A7EB050808EB0600B0F5007FF7
:10C5A00001D9C6F5007820694246C06D811909EBB2
:10C5B0000500F4F740F806EB0800C605F60D0FD1AC
:10C5C000607D401CC1B261752069827F914207D1B4
:10C5D0000021617504F1180101F04CFE0028CAD059
:10C5E0004544BD42C9D3E0682844E0602846C2E71C
:10C5F00070B506460C4615461421106900F050FB34
:10C60000002839D030785C2800D1761C20785C284E
:10C6100000D1641C307880B3207870B300200246CB
:10C62000E86129463046FFF7A1FE002824D028699A
:10C6300090F87C0080B10026324629462046FFF75C
:10C6400048FA01281AD0286900227C30294600F0D7
:10C6500041FA002810D007E001263246294620463C
:10C66000FFF737FA012809D032462946204601F063
:10C67000B4FC002800D0012070BDFFE70020FBE7DC
:10C680002DE9F041044600880D46C00602D5002081
:10C69000BDE8F0810421206900F002FB40B3A068EE
:10C6A000A84200D205462069690A827FB1FBF2F3F5
:10C6B00002FB13116175E769A761806BB5FBF0F6AA
:10C6C00056B104F118084146A769206901F0D2FD6E
:10C6D0000028DDD0761EF6D1A169206900F04EFF5A
:10C6E00018B12069807F6075A7610120E560CFE700
:10C6F000208840F010002080C9E7F0B5044600888B
:10C7000089B0C0065FD41421206900F0C9FA00285E
:10C7100055D0D4E9010181424CD9491E2046FFF78A
:10C72000AFFF002850D0206900F093FB0246A169BA
:10C73000206902F041F8002846D06946204601F001
:10C7400008FC002840D0E069000CADF81400E06956
:10C75000ADF81A00A068079000F080FE01460DF1C8
:10C76000160001F0CDFD00F0DEFB014606A801F049
:10C77000C7FDBDF81800ADF812006F46E58A216AC2
:10C78000206900F0E6FB00EB15110E46206901F070
:10C79000FBFBC0B1206905F00F012022C06D00EB4A
:10C7A00041103946F3F78CFF01223146206902F02F
:10C7B000ABF840B12069017F032907D00AE0208847
:10C7C00040F010002080002009B0F0BD02F068F8B1
:10C7D0000028F9D00021206901F012FF0028F3D0D1
:10C7E00000212069FFF7F4F80028EDD00120EBE7E5
:10C7F0002DE9F74F0446008882B01746C00603D5DE
:10C80000002005B0BDE8F08F1421206900F048FA3F
:10C8100060B121884FF4007909EA811B04F1180006
:10C82000E1694FF0000A009029B10EE0208840F045
:10C8300010002080E4E72069009900F0B9FB00288F
:10C84000DFD0A069E06184F815A0E0680025C0F39E
:10C8500008064CE02069617D827F914218D1E16831
:10C86000A2682944914203D2009901F003FD0BE034
:10C87000D4F81880009900F09BFB0028C1D04146F5
:10C88000A269206901F098FF0028BAD084F815A0A9
:10C89000A1692069FFF79AF9617D084401900EB9FA
:10C8A0005F4505D22069019901F06EFB0028A8D0F0
:10C8B000A7EB050808EB0600484501D9C6F5007846
:10C8C0000398424641192069C06D3044F3F7B3FE26
:10C8D0002069019901F094FE002892D006EB08002F
:10C8E000C605F60D02D1607D401C60754544BD4211
:10C8F000B0D3E0682844E060A168884200D9A06015
:10C9000001207EE72DE9F05F05460C466848AFF34D
:10C910000080002000F004FA060055D001462846A9
:10C9200000F04CFA8246306900284DD00020514674
:10C93000024604E0401C5C2B00D10246491C0B78E7
:10C94000002BF7D10AEB020083465AA1F3F734FF1C
:10C9500000B32A21584600F06DFA05465846F3F711
:10C960003FFE8046681C1AD04FF001090BEB050012
:10C9700051A1F3F721FF18B1A8EB0500A0F10100C8
:10C980008046308880060DD5324621465046FFF756
:10C99000A5FC0BE000254FF00109A846F1E74FF098
:10C9A0000009EEE731462046FFF71BFC60B100208E
:10C9B00084F8FF00B9F1000F08D055EA08001FD035
:10C9C000CDB35946002349E001242EE023465A46C0
:10C9D00010E05B1C12F8011BA0F16107192F01D8B0
:10C9E00020F02000A1F16107192F01D821F02001CA
:10C9F0008842C6D118780028EBD111780029E8D1F7
:10CA00003088800603D5307D84F8060109E00020D7
:10CA100084F80601F082B4F80401B0823046FFF7D2
:10CA2000E4FB7068C4F8000100242148AFF30080E3
:10CA30002046BDE8F09F13E011F8012BE05CA2F165
:10CA40006107192F01D822F02002A0F16107192FE8
:10CA500001D820F02000824293D15B1CAB42EBDB7B
:10CA6000B8F1000FCCD02046F3F7BAFD844605EBB1
:10CA70000801614585DC0BEB05035B1CACEB080290
:10CA800012E000BF13F8010BA15CA0F16107192FA0
:10CA900001D820F02000A1F16107192F01D821F061
:10CAA00020018842A5D1521C6245EBDBA8E70000BB
:10CAB000000000002A2E2A002E2A0000016800290A
:10CAC00001DCF4F70EB9491E016041684A1C42605E
:10CAD00008787047002301F0BDBA0000F0B50446A5
:10CAE00089B01A48AFF3008000F0AAF8BCB100206A
:10CAF000ADF8000004906946204600F05FF9049804
:10CB000008B3BDF8000000F02001049800F0CEFC4E
:10CB100004460E48AFF3008009B02046F0BD002463
:10CB20000B4D26460B4F0AE0E87900F00401286817
:10CB300000F0BCFCA04200DD0446761C08353888B5
:10CB40008642F1DBE5E70324E3E700000000000094
:10CB5000B84602089E4602088A68002A01DCF4F7FB
:10CB6000B3BA521E8A604A68C0B2531C4B60107040
:10CB700070470000F0B5044695B00F462F48AFF35C
:10CB80000080002000F0CCF805004ED00146204681
:10CB900000F014F90646286980B3288880062ED54F
:10CBA0003046F3F71DFD441E06D4305D5C2802D0EC
:10CBB000641EFAD500E06CB1621C31466846F3F79A
:10CBC0003AFD0DEB04010020487039466846F3F742
:10CBD00026FD07E03846F3F703FD0246394668466E
:10CBE000F3F729FD29466846FFF79AFB01281CD078
:10CBF0002A4639463046FFF7FBFC14E015E029468B
:10CC00003846FFF7F0FA01280FD029463046FFF7E3
:10CC1000EAFA50B1284600F0A7F8012805D02946C5
:10CC20003846FFF7E5FA012806D001240348AFF3A0
:10CC3000008015B02046F0BD0024F7E7000000009A
:10CC400070B5124C207800281ED100F041F8002267
:10CC50000F4811460F4B05E0C5796D0750F8085B8A
:10CC6000521C29601D88AA42F6D300200A4B0B4AA9
:10CC700005E000BF00EBC005401C23F82510158817
:10CC8000A842F7D30120207070BD0000C00300202F
:10CC9000B84602089E4602083C2600209C46020830
:10CCA00010B504460068814301D0002010BD000784
:10CCB00006D460680021426908469047C00701D049
:10CCC000012010BD206820F006002060EDE7000084
:10CCD00007480021A0F58062C0E90221054A4260B0
:10CCE00000F5C073044A9A604161018270470000F8
:10CCF000CC2A0020A0460208D446020860B1017880
:10CD000051B1012100E0491C425C002AFBD10844DA
:10CD100010F8010C5C2801D00020704701207047FA
:10CD200070B5064600240A4D0A4804E029888907A0
:10CD300006D02435641C01888C42F7DB002070BDCE
:10CD400024212846F3F710FD06B13460284670BD53
:10CD50003C2600209C460208004870470101DB0782
:10CD60004FF440207047000030B500221149124BAB
:10CD70001AE00C88A40715D0814213D00C6905690C
:10CD8000AC420FD10488A40609D5CC8AC58AAC422E
:10CD900008D10C6A056AAC4204D1012030BD8C8AEE
:10CDA000858AF8E7521C24311C88A242E1DB00206E
:10CDB00030BD00003C2600209C460208F0B51B4A0E
:10CDC0001B4CE8B10378DBB123F0200643783A2B03
:10CDD00003D085783A2D03D012E03023801C01E087
:10CDE00073B1C01C002507E01779B74202D157790B
:10CDF0009F420AD06D1C08322788BD42F4DBF0BD8B
:10CE000000230EE0D579ED0709D013680B61D279C4
:10CE10005207F4D50A8842F020020A80F0BD5B1C5C
:10CE200008322588AB42EDDBF0BD0000B8460208B1
:10CE30009E460208002205E08B4201D11046704751
:10CE4000401C521C0378002BF6D1581E704700205E
:10CE50007047007F012805D0022806D0032807D09C
:10CE60000020704740F6FF7070474FF6FF70704724
:10CE70006FF07040704710B50446816901F084F886
:10CE8000002809D0E06D00F5FF7000F0FFFAA0F572
:10CE90002A41553901D0002010BDE06D417BA177BA
:10CEA0000B3000F0F3FAE085E06D0E3000F0EEFAA2
:10CEB0006084E06D017C6177113000F0E7FAA085B5
:10CEC000E06D133000F0E2FA6062E06D163000F0C1
:10CED000DDFA2084616AE9B9B8B9E06D283000F064
:10CEE000D5FAE087E06D2C3000F0D5FA2064E06DD3
:10CEF000303000F0CBFAA4F84400E06D323000F09E
:10CF0000C5FAA4F84600606A20B9E06D203000F050
:10CF1000C2FA6062208C20B9E06D243000F0BBFAC8
:10CF20002084012010BD10B5FFF716FF10F01F017F
:10CF300000D10121C0F303220C2A00D802B901223A
:10CF400041EA4211442202EB104041EA402080B203
:10CF500010BD10B5002280F87B2059B90267017F0F
:10CF6000032906D0828E81691144012280F87B203A
:10CF700003E0016CFEF72AFE0146084610BD027F61
:10CF8000012A04D0022A06D0032A0AD105E001EBC7
:10CF90004101890A02E0090A00E0C909028C8A42BB
:10CFA00001D8002070478269408C104408447047C3
:10CFB0002DE9F04105460E46C46E5CE02146284648
:10CFC000FFF7DDFF804601462846FEF701FD0028F9
:10CFD00038D0287F012804D0022823D0032830D15C
:10CFE00027E004EB4400C0F34800B0F5FF7F04D80D
:10CFF000E96C084400F04AFA0DE0E86C08F1010120
:10D0000090F8FF712846FEF7E3FC00281AD0E86C80
:10D01000007847EA0020E10701D000090FE0C0F3E3
:10D020000B000CE0E96C200601EBD05000F02EFA6A
:10D0300005E0E96C600601EBD05000F02CFA18B165
:10D0400018E00020BDE8F0810E48002102880E485B
:10D0500009E003889F0604D59B0702D58369A34294
:10D0600008D02430491C9142F3D33460641C012061
:10D07000EC66E7E7641C286B801CA0429ED8EC6637
:10D08000DFE700009C4602083C26002010B504465D
:10D090008069B4F844100144204600F075FF002870
:10D0A00029D0E06D00F5FE7000F0F5F914498842D2
:10D0B00020D1E06D00F0EFF9124988421AD1E06DFD
:10D0C00000F5F27000F0E7F90F49884212D1E06DE7
:10D0D00000F5F47000F0DFF9216B81420AD3A066FD
:10D0E000E06D00F5F67000F0D6F9022802D3216B4E
:10D0F000814201D2002010BDE066012010BD000079
:10D10000000055AA52526141727241612DE9FF5FE0
:10D11000054600200E46029001900390C9698146A1
:10D1200000913069FFF715FFB5F8047182464FF0A2
:10D13000000B306990F87B00E0B1B7F5007F10D0AC
:10D140001CE07F1A016C009A914200D90091694657
:10D1500001F090F8002805D03069009900F00EFA2F
:10D1600018B1002004B0BDE8F09F30690099FEF7C7
:10D170002DFD82463069818FB942E2D909F101095A
:10D180000AEB1711306900F0FFFE0028EAD0306981
:10D1900007F00F01C06D00EB411420780028E1D0AA
:10D1A000E5285AD0E17A0F2902D0080755D407E0C4
:10D1B000400605D5012003900190607B029011E0AC
:10D1C000039878B30F290BD000200390204600F07D
:10D1D000F1F90199002975D00299884248D001E0FF
:10D1E0000198D0B3617B0298814202D00020019067
:10D1F00068E02078344B00F01F00401E00EB8001F7
:10D2000001EBC00805EB080100201A5CA25C0A547F
:10D21000401C0D28F9D3207808F10D08400601D5EF
:10D2200005F808B0E07A00F03F000F284AD0072147
:10D2300000E0491E605C2028FBD0491C002002E071
:10D24000225C2A54401C8842FAD3217A20290DD02E
:10D250002E212954401C082103E033E02A54491CA4
:10D26000401C625C202A01D00B29F7D305F800B0DE
:10D2700005F58275298801EB09002880E07A307570
:10D2800004F11C0000F007F97060B06004F11600B2
:10D2900000F0FCF8C10A2971C0F34511C00669719C
:10D2A000800EA87104F1180000F0F0F800F01F01E2
:10D2B000E971C0F34311400A297200F2BC70688121
:10D2C00001204FE77F1C34E7764E03082DE9F84F25
:10D2D000834660480E4615464FF0000A4FF6FF7829
:10D2E000824201DD062713E042F20F70854201DD24
:10D2F00005270DE0B5F57A7F01DB042708E0632DF3
:10D3000001DD032704E0092D01DD022700E00127EC
:10D31000002003E02E2900D18046401C1BF800109D
:10D320000029F7D105B94F1E4FF00009C7F10700DA
:10D330004C46009018E000BF1BF809A0BAF1200F7E
:10D3400010D0BAF12E0F0DD0BAF1000F11D0AAF102
:10D350006100192801D82AF0200A504601F0A9F8E6
:10D360003055641C09F10109C14502D20098A04260
:10D37000E2D8EDB37E203055641C072F46D2DFE89B
:10D3800007F04542352A1E12040032483249401C3B
:10D3900095FBF0F0414305EB4115092800D9092020
:10D3A00030303055641C42F2107095FBF0F06FF491
:10D3B0001C7141433030305505EB0115641C4FF4AE
:10D3C0007A7095FBF0F06FF07C01414330303055BE
:10D3D00005EBC105641C642095FBF0F06FF01801AB
:10D3E00041433030305505EB8105641C0A2000E0D4
:10D3F0000CE095FBF0F04142303001EB81013055FB
:10D4000005EB4105641C30353555641CBAF1000F3D
:10D410001AD02E203055641CA8F57F414046FF39B4
:10D4200012D0451C071D0DE01BF8050060B1A0F1EE
:10D430006101192901D820F0200001F03AF8305597
:10D44000641C6D1CBD42EFD3002030550120BDE8A7
:10D45000F88F00009F860100CBF3FFFF10B5FFF7A8
:10D460007FFCC0F344011D2900D90021C0F305222F
:10D470003B2A00D90022C0F3044041EA4211172898
:10D4800000D9172041EAC02080B210BD4178007851
:10D4900040EA01207047C1788278090641EA0241DA
:10D4A0004278007841EA02210843704710B50446EB
:10D4B00040680022B1B318B12068C00702D00BE069
:10D4C000032010BD2260606801680020884750B3C7
:10D4D000206840F001012160206820F01E012160D9
:10D4E00060680021426908469047010603D520681C
:10D4F00040F0180106E0C10738D0800703D4206847
:10D5000040F010012160606801680120884750B137
:10D51000206840F0020120462160FEF769FF18B143
:10D52000022010BD0AE021E0206840F004012046FE
:10D530002160FFF701F8F0B90420F2E768B1206834
:10D54000C0070AD12260D4E90120E169126890473E
:10D5500060B1206840F001002060206840F00400C5
:10D560002060616821B1896811B104E00120D8E729
:10D5700040F0100020600020D3E70000007F012869
:10D5800004D0022805D003280FD107E040F6F87038
:10D5900001E04FF6F870814205D206E021F07040BC
:10D5A0000349884201D301207047002070470000E2
:10D5B000F8FFFF0F024600200146C30700D080237A
:10D5C00003EB5000535C491C1844C0B20B29F4D340
:10D5D00070470000FBF7C2F8F9F7E8FCF8F794FC95
:10D5E000F5F7CEFCFCF7BCFAFDF738F8F3F74EFF81
:10D5F000F8F7BAFFFBF7B4FAF8F7E0FFF9F760FCC9
:10D60000F4F760FEF4F75EFE002063490860052031
:10D61000624908604FF41670614908600020614952
:10D62000087061490860012060490860F4F79AFEBB
:10D630006820FBF719FB044640F2E7325C480168BA
:10D640002046FDF717FD42F6A2016420FDF7CAFC53
:10D65000F4F78CFF4FF42F7056490860FCF7ECFE8E
:10D66000F4F7B8FAFDF75AFCF4F752FB00210A2050
:10D67000FDF7B8FC00210B20FDF7B4FC00210C20C5
:10D68000FDF7B0FCFBF72AFE01204B4908604FF480
:10D690002F704A49086048607CE0FBF7E5FEF3F72D
:10D6A000D1FF3E48006810B9012045490870FBF7DA
:10D6B000EBFB3D4800683C490968491C3A4A116047
:10D6C000062836D006DC062845D2DFE800F013161F
:10D6D0001924272F092835D004DC07282CD0082846
:10D6E00039D12CE00A2830D0A0F59850883800288D
:10D6F00031D12DE0F4F736FE31E0F4F7C9FA2EE02F
:10D70000F8F7EAFE27480078012803D141F2883073
:10D710002549086023E0F4F7A7FD20E01F480068D2
:10D7200018B142F210702049086018E0F4F78AFF3F
:10D7300015E0F4F7D3FB12E0F4F700FD0FE0F4F787
:10D7400033FB0CE0F4F772F909E0F4F7A3FA06E012
:10D75000F4F714FC03E000201349086000BF00BF89
:10D7600018480068B0F5FA7F05DA4FF48061164872
:10D77000F8F7FDFD04E04FF480611348F8F7F5FD7C
:10D78000F5F7E6FDF4F7F2FEF4F79CFDF4F7A2F9E5
:10D79000F8F7FAFE81E7000054000020B0000020F6
:10D7A000F80000203C0100200C00002004000020B4
:10D7B00030000020340000204C000020B00B00207E
:10D7C0001000002014000020000C0140014A00F06D
:10D7D0005FB800004C2C0020014900F066B8000042
:10D7E0004C2C0020014900F05DB900004C2C0020B9
:10D7F000014B00F067B900004C2C0020014900F0FB
:10D800008DB900004C2C0020014B00F093B90000B2
:10D810004C2C00202DE9F04107461849184A12689F
:10D8200031F81200F8F746FE0646F8F7A5FD054662
:10D8300014481349096850F821002C1A002C00DA0A
:10D8400064420A2C0EDB10480D490968405C401CFC
:10D85000C0B20D490A4A12688854642802DC0B4899
:10D86000006848B107480649096840F8215000207F
:10D870000549034A12688854BDE8F0813C0D002038
:10D88000C0000020B00B0020C4000020B000002029
:10D8900018B1022807D0002070479068C06900B115
:10D8A000004780207047506870472DE9F8430C46C8
:10D8B00010B101287DD104E0886800688047BDE888
:10D8C000F883A068816901208847A06841694FF406
:10D8D000C87088470025A0688168FF2088476D1CB4
:10D8E000102DF8D3A06881690020884700222346C4
:10D8F0001146104600F04CF905460026012D07D0D0
:10D90000A0688168FF208847761C0546642EF5D301
:10D91000A068816901208847012DCBD1A0684169A9
:10D9200044F62060884700202070A06881690020AC
:10D93000884704268DF8006023466A464FF4D57167
:10D94000082000F025F901280FD19DF8000060B9EA
:10D950009DF8010048B99DF80200012805D19DF805
:10D960000300AA2801D103202070A068816901204A
:10D97000884700254CF25038A0688169002088470C
:10D98000002223461146372000F002F90746A0681E
:10D9900081690120884778071AD4012F15D1A06822
:10D9A0008169002088472078032815D0002081074E
:10D9B00000E06EE023460022292000F0E9F8074647
:10D9C000A06881690120884747B16D1C4545D3D3C4
:10D9D0002078032807D01EE00120E8E720780328FC
:10D9E00001D0022033E0A0688169002088478DF8CB
:10D9F000006023466A4600213A2000F0C9F8054637
:10DA0000A0688169012088472DB99DF80000400673
:10DA100001D526701CE02078D0B900254746A068C3
:10DA2000816900208847002223461146012000F02A
:10DA3000AFF80646A068816901208847012E01D011
:10DA40003EBB03E06D1CBD42E9D322E00120207003
:10DA5000A068816900208847234600224FF40071A6
:10DA6000102000F095F80546A068816901208847DC
:10DA70007DB9A068816900208847002223461146AD
:10DA80003B2000F085F80546A068816901208847A1
:10DA90000DB1002013E7204600F002F90028F9D06C
:10DAA00001200CE770B505460C46084600F0F8F872
:10DAB000002806D02146284600F017F9002800D09B
:10DAC000012070BD2DE9F041064698680F461546C5
:10DAD00081691C460020884723462A46394630463D
:10DAE00000F0A6F80646012D0FD900222346114664
:10DAF0000C2000F04DF8084DA0688168FF20884791
:10DB0000FF2802D06D1EF7D10026A0688169012090
:10DB100088473046BDE8F08148E8010038B1012867
:10DB20004FF0000002D108704860012070478868FB
:10DB3000406800472DE9F041064698680F461546B3
:10DB400081691C460020884723462A4639463046CC
:10DB500000F046F90646012D11D9A0688168FD2024
:10DB60008847A0688168FF208847084DA0688168C1
:10DB7000FF208847FF2802D06D1EF7D10026A0683D
:10DB80008169012088473046BDE8F08148E80100FE
:10DB90002DE9FC4140F040008DF80000080E8DF8A2
:10DBA0000100080C8DF80200080A8DF8030000201F
:10DBB00014461D468DF804106A46014605234E079B
:10DBC00007D1B3EBD10F04D902EBD106367846EA80
:10DBD0000000060401D580F409404000491C3029AA
:10DBE000EDD3000A40F001008DF80500A8688168B7
:10DBF000FF208847A8680621C2686846904700272A
:10DC0000A8688168FF2088470646FF2802D17F1C4C
:10DC1000082FF5D34CB1277805E0A8688168FF206C
:10DC2000884704F8010B7F1EF7D2F0B2BDE8FC81F3
:10DC30002DE9F04111250F4616461C46012A00D950
:10DC400012252178042900D24002014600222846EC
:10DC5000FFF79EFF10BB1CE046F2A815A068816884
:10DC6000FF208847FE2802D06D1EF7D116E0ADB127
:10DC7000A0684FF40071026938469047A068816837
:10DC8000FF208847A0688168FF20884707F5007754
:10DC9000761E002EE0D10120BDE8F0810020FBE7D8
:10DCA0007FB504468068816900208847234610229A
:10DCB00069460A2000F06CF80546A06881690120D9
:10DCC000884775B12078012868460CD00930016872
:10DCD000C07809BA21F0FF0101430120616004B05E
:10DCE00070BD0020FBE70A30F1E77FB50446886885
:10DCF0000D468169002088472B461022694609207D
:10DD000000F046F80646A868816901208847B6B148
:10DD10009DF80500012100F00F0001FA00F0A0803D
:10DD2000BDF80C0040BAC0F383108140E1809DF83B
:10DD30000000800906D0012819D0022802D0002056
:10DD400004B070BD9DF806009DF80710000440EA7D
:10DD500001209DF808100843BDF80910C0F38B108E
:10DD600049BAC1F3C211401C891C88400DE09DF8DE
:10DD700007009DF80810000440EA01209DF80910F2
:10DD800008430004800900F5806020600120D7E787
:10DD90002DE9F04117460E4600221C461146FFF7BA
:10DDA000F7FED8B946F2A815A0688168FF20884719
:10DDB000FE2802D06D1EF7D110E07DB1A068394673
:10DDC000026930469047A0688168FF208847A068B4
:10DDD0008168FF2088470120BDE8F0810020FBE733
:10DDE0002DE9F0411826884615461C46012A00D91F
:10DDF00019262178042900D240020146002230462B
:10DE0000FFF7C6FE38BBFE27012D29D9FC2727E0E6
:10DE1000A068816838468847A0684FF40071C268DE
:10DE200040469047A0688168FF208847A0688168C5
:10DE3000FF208847A0688168FF20884700F00F0016
:10DE4000052812D10A4EA0688168FF208847FF2864
:10DE500002D0761EF7D108E03EB108F500786D1EBD
:10DE6000002DD5D10120BDE8F0810020FBE70000A6
:10DE700020A1070070B500248020104908800320ED
:10DE800088700420C8700E48F8F7ECF9002510E0FF
:10DE90006006040EFBF7B6FFFEF742F98021084842
:10DEA000F8F755FA08B144F00104FBF7B5FF681C18
:10DEB000C5B2082DECDB204670BD00002C0100200F
:10DEC000000C014010B5FBF7C7FFFBF79BFFFBF70A
:10DED000A3FFFBF7ABFF10BD70B50446C0680D464D
:10DEE000164610B194F8641029B129462046BDE8C1
:10DEF000704000F049B894F8652082B1A16DA94244
:10DF00000DD80A44AA420AD9206E691A00EB4121B1
:10DF10004FF40072E06DF2F78EFB656517E0B042DA
:10DF200000D206466068E16D32468368284698470D
:10DF3000012806D04FF0FF306065002084F86500AE
:10DF400070BD65656D1C761EA56584F86560012051
:10DF500070BD70B50E460446C58A016A0069FEF7B9
:10DF6000F8FF00EB1511206900F00EF800280AD028
:10DF7000206905F00F012022C06D00EB41113046F1
:10DF8000F2F79EFB012070BD70B50446406D0D4652
:10DF9000A84201D1012070BDA06DA8420ED894F80E
:10DFA00064100144A94209D9216E281A01EB4021CD
:10DFB0004FF40072E06DF2F73EFB0CE06068E16D3B
:10DFC0000122836828469847012804D04FF0FF308B
:10DFD0006065002070BD6565DCE72DE9F04107460E
:10DFE000086988B00C4690F87A609046002538465B
:10DFF000FDF737FD60B1012E09D03846F2F7F0FA8F
:10E000000C300D21B0FBF1F0401CB04200D90125CD
:10E0100069462046FFF79DFF002817D02046FEF7EF
:10E020008FF8002812D045B120692146406FE06189
:10E030003846FDF71FFC002808D06B4642462146B3
:10E040003846FDF755FE002800D0012008B0BDE895
:10E05000F08100002DE9FF4F97B00C46012A19D03E
:10E060000020129001204FF0000ACDE90E0A039023
:10E07000E06900901798F2F7B3FA0490002010902E
:10E0800021698346E06908671798FDF7EAFC0128D3
:10E0900002D009E00120E4E704980D210C30B0FB28
:10E0A000F1F0401CC0B20E9009A91798FDF7E9FFE6
:10E0B000129808B1092000E00D200790206900990E
:10E0C000FEF747FF81460026206990F87B1019B1C2
:10E0D000B6F5007F13D01BE0818FB14218D1016CDF
:10E0E000009A0026914200D90091694600F0C2F8DA
:10E0F000002805D020690099FFF740FA18B10020E8
:10E100001BB0BDE8F08F20690099FDF75FFD8146E7
:10E1100009EB16112069FFF737FF0028F0D02069BE
:10E1200006F00F01C06D00EB411528780028E7D0FC
:10E13000E5286FD095F80B80B8F10F0F03D05FEA98
:10E14000087067D431E0410609D500991091697BC8
:10E150000F9120F04001491CC9B2B34603916A7B7C
:10E160000F998A4256D100F01F00401E00EB80013B
:10E1700001EBC0001799DFF8F8C00A18002000BFB3
:10E180001CF80010135C695C81EA030737F0200774
:10E1900008D103B911B1401C0D28F1D30AF10100D7
:10E1A00000F0FF0AB8F10F0F34D0039801280ED009
:10E1B00029D9A0F1010050451BD12846FFF7FAF9F3
:10E1C0000F99884215D10AF10100C0B21AE00E98E9
:10E1D000012803D007990498884214D2009810901F
:10E1E000B34609A9284600F097F878B14FF0010A24
:10E1F00012E00E98012806D109A9284600F08CF8F3
:10E2000008B1039882460398504505D001204FF08D
:10E21000000A0390761C57E7E87AC0F300111298C1
:10E220008142F3D11A9808BBE87A207505F11A00EB
:10E23000FFF72CF9074605F11400FFF727F907EB64
:10E240000040E061E68200982062216910984867EA
:10E2500021690020A1F878B0216981F87AA0E060F6
:10E2600005F11C00FFF717F96060A060012047E787
:10E27000764E03082DE9F0410D680E460446294606
:10E28000FEF77DFE804601462046FDF7A1FB0028F3
:10E2900007D0207F012806D0022825D0032828D0C7
:10E2A0000020BDE8F08105EB4500C0F34800B0F563
:10E2B000FF7F04D8E16C0844FFF7E8F80DE0E06C5C
:10E2C00008F1010190F8FF712046FDF781FB00285D
:10E2D000E7D0E06C007847EA0020E90701D00009A8
:10E2E0000BE0C0F30B0008E0E16C2806C00D085AF3
:10E2F00003E06806E16CC00D085830600120D0E7EB
:10E300000A0A4270017070470A0EC2700A0C8270CD
:10E310000A0A42700170704730B50022835C8C5C41
:10E3200083EA040535F0200501D0002030BD04B992
:10E3300013B1521C0B2AF1D3012030BD10B5FBF7ED
:10E3400075FDFBF75FFDFDF7EBFEFBF785FDFDF7C8
:10E35000E7FEFBF761FDFDF7E3FE10BD10B5FBF72F
:10E360007BFDFDF7DDFEFBF74DFDFDF7D9FEFBF76D
:10E370005DFDFDF7D5FE10BD2DE9F0470026012714
:10E3800004460D4602297DD379E0E06EA84200D90B
:10E39000E56629462046FEF7F2FD81460146204605
:10E3A000FDF716FB00287AD0207F012804D0022830
:10E3B00046D0032872D14DE005EB4500C0F3480874
:10E3C000B8F5FF7F16D8E16C01EB0800FFF75EF8A7
:10E3D000E90703D000F00F01000903E000F47041E9
:10E3E000C0F30B00E26C814602EB080089B2FFF734
:10E3F00087FF3BE0E06CEA0790F8FF11884604D005
:10E4000001F00F0180F8FF1101E080F8FF6184F84E
:10E41000507009F101012046FDF7DAFA00283ED0DC
:10E42000E06CEB07017848EA012202D0067010097F
:10E4300004E001F0F0010170C2F30B00814615E029
:10E440002806C50DE06C2844FFF720F88146E06CF3
:10E4500046530BE06806C50DE06C2844FFF71BF837
:10E460008146E06C4651A06E401CA06684F8507056
:10E4700049462046FFF782F8012812D04D46206B0E
:10E48000801C02E013E00AE008E0A8423FF67DAFFE
:10E4900000212046FDF79CFA002800D00020BDE8AE
:10E4A000F08700212046FDF793FA0028F7D00120DD
:10E4B000F5E710B5044600F005F808B1204610BD98
:10E4C000582010BDA0F12001012917D9C91E062925
:10E4D00014D92D2812D02E2810D00D3909290DD984
:10E4E00040280BD01139192908D91D391D2905D902
:10E4F0007D2803D07E2801D000207047012070477E
:10E5000010B501210248F7F732FFFDF709FE10BDF3
:10E510000018014010B501210248F7F726FFFDF76A
:10E52000FFFD10BD0018014070B5044625460026C9
:10E530000FE005F0800010B1FBF778FC01E0FBF77D
:10E540008BFC6806050EFBF75DFCFBF765FC701C99
:10E55000C6B2082EEDDB70BD70B50125FBF766FC79
:10E56000FBF750FC80210A48F7F7F1FE00B10025C7
:10E57000FBF752FC07480068012806D1002402E09E
:10E58000FDF7CEFD641C0A2CFADB284670BD0000A6
:10E59000000C0140280100202DE9F04107460C46FF
:10E5A0000A201649086000BFFFF7C8FEA02101EB52
:10E5B0004701C8B200F072F805460DB9FFF7CEFE6C
:10E5C0001DB90E4800680028EED145B12646E11776
:10E5D00004EB1161C1F3072000F060F8054655B166
:10E5E0002646E11704EB11610912A4EB0121C8B220
:10E5F00000F054F805462846BDE8F08120010020CF
:10E600002DE9F0410D46C1680446E1B100261DB375
:10E61000656594F864204FF400779AB3A06D831871
:10E62000AB4227D18A4225D204F15C04606821689C
:10E6300000EB42203A46F1F7FEFF207A401C2072A0
:10E640000120BDE8F081002DFAD00022294600F01B
:10E650005BF90028F5D0F3E794F86420002AEFD0A6
:10E660006368216EA06DDB6898470028E9D084F8C4
:10E670006460E5E76368216EDB6898470028E0D0B6
:10E6800084F8646004F158043A46D4E90110F1F7C3
:10E69000D2FF0120256020736673D1E710B50446D0
:10E6A0002046FFF741FFFFF757FF08B1012010BDDB
:10E6B0000020FCE72DE9F0410446C769FEF7CEFED5
:10E6C0000646FEF730FC804620694FF40071C06DAD
:10E6D000F2F728F820690B2234A1C56D2846F1F71E
:10E6E000EFFF1020E872314605F10E00FFF708FE3B
:10E6F000414605F11000FFF703FE414605F1120007
:10E70000FFF7FEFD314605F11600FFF7F9FD414622
:10E7100005F11800FFF7F4FD05F12000202229463D
:10E720000646F1F7CDFFE069010C05F11400FFF793
:10E73000E7FDE06981B205F11A00FFF7E1FD2E2047
:10E7400070702069006F010C06F11400FFF7D8FD0E
:10E750002069006F81B206F11A00FFF7D1FD21692F
:10E76000E069086739462069FDF730FA064601225C
:10E770003146206900F0C8F8002814D020694021F3
:10E78000C06DF1F7CFFF012506E07119002200F0FE
:10E79000BBF8002807D06D1C2069817FA942F4D8FE
:10E7A0000220E0820120BDE8F08100002E20202020
:10E7B00020202020202020002DE9F0471546044687
:10E7C0000E46FEF7DCFB814601462046FDF700F9C8
:10E7D000002809D0207F4FF00108012806D0022828
:10E7E00044D0032848D00020BDE8F08706EB46005F
:10E7F000C0F34807C5F30B05B7F5FF7F13D8E06CEE
:10E800003844FEF743FEF10702D065F31F1002E023
:10E8100000F470402843E16CCA1981B24FEA02004B
:10E82000FFF76EFD38E0F007E06C06D090F8FF11BE
:10E8300065F31F1180F8FF1101E080F8FF5184F8A3
:10E84000508009F101012046FDF7C2F80028CBD025
:10E85000F00703D0E16C280908701DE0E06C017836
:10E8600001F0F00141EA1521017015E0E16C30067C
:10E8700001EBD050A9B2D3E77006C60DE06C30446E
:10E88000FEF709FE18B9A06E08B1401EA066E06C44
:10E8900029463044FFF738FD84F850800120A3E773
:10E8A00010B50446C06D4FF40071F1F73BFF1449F9
:10E8B000E06DFFF729FDE06D124900F5F270FFF7FA
:10E8C00023FDE06DA16E00F5F470FFF71DFDE06D16
:10E8D000E16E00F5F670FFF717FDE06D4AF6552181
:10E8E00000F5FF70FFF70CFDB4F84410A069014477
:10E8F0002046FFF785FE002800D0012010BD000053
:10E90000525261417272416170B504460D464069D0
:10E91000E16D08B1012A09D060680122C368284668
:10E920009847002801D00120656570BD0B46002284
:10E930002946FEF78CFAF4E70000000030000020C2
:10E9400000000000000000009F0500000000000023
:10E9500040480000010000001C000020670000008B
:10E9600000000000030000000000000002E00000C2
:10E97000020000001C00002068000000650000008C
:10E98000280C00006500000002A000000300000049
:10E990001C00002069000000D0070000B80B000038
:10E9A000DE07000002200000040000001C00002020
:10E9B0006A00000001000000E80300000100000000
:10E9C00002200000050000001C000020650000007F
:10E9D0000100000040420F00010000000220000082
:10E9E000640000001C0000206B0000000A00000012
:10E9F000640000002800000012880000650000008C
:10EA0000340000200000000000000000D0070000DB
:10EA1000BC02000011500000660000001C00002035
:10EA20007A010000010000000A0000000A00000056
:10EA300002200000670000003800002000000000F5
:10EA4000000000000A00000000000000012000009B
:10EA5000680000001C0000207B0100000000000096
:10EA600001000000000000000260000069000000DA
:10EA70001C0000207C0100000000000001000000DC
:10EA800000000000026000006A0000001C0000207E
:10EA90007D0100000000000078000000050000007B
:10EAA000C24800006B0000001C0000207E01000036
:10EAB00000000000D0070000D00700001350000045
:10EAC0006C0000001C0000207F010000000000001E
:10EAD0009F05000000000000434800006D0000009A
:10EAE0001C0000208001000000000000D007000092
:10EAF00000000000135000006E0000001C00002009
:10EB000081010000000000009F05000000000000DF
:10EB1000434800006F0000001C000020820100003C
:10EB20000000000001000000000000000260000082
:10EB3000700000001C0000208301000001000000A4
:10EB4000060000000100000002200000710000002B
:10EB50001C00002084010000000000009F05000050
:10EB60000000000042480000720000001C0000206D
:10EB7000850100000000000001000000010000000D
:10EB800002600000730000001C00002086010000ED
:10EB90000000000001000000000000000260000012
:10EBA000C80000005C000020000000000000000021
:10EBB000D00700000000000011500000C900000054
:10EBC000600000200000000000000000D0070000EE
:10EBD0000000000011500000CA0000006400002086
:10EBE0000000000000000000010000000000000024
:10EBF00001600000CB000000680000200000000061
:10EC000000000000010000000000000001600000A2
:10EC1000CC0000006C00002000000000000000009C
:10EC2000010000000000000001600000CD000000B5
:10EC30007000002000000000000000000100000043
:10EC40000000000001600000CE0000007400002001
:10EC500000000000000000000A00000000000000AA
:10EC600000200000CF00000078000020000000001D
:10EC70000000000001000000000000000060000033
:10EC8000D00000007C000020000000000000000018
:10EC9000D00700000000000021290000D100000082
:10ECA00080000020000000000000000001000000C3
:10ECB0000000000000600000D2000000840000207E
:10ECC0000000000000000000010000000000000043
:10ECD00000600000E80300001C0000206C00000041
:10ECE000000000000500000000000000020000001D
:10ECF000E90300001C0000206D000000BC020000C1
:10ED0000B00400008403000012500000EA03000079
:10ED10001C0000208600000001000000100E000012
:10ED20000A000000C2480000EB0300001C000020A5
:10ED30006E000000000000009F05000000000000C1
:10ED400042480000EC0300001C0000206F0000009F
:10ED5000000000009F050000000000004248000085
:10ED6000ED0300001C000020700000000100000006
:10ED7000D00200003C00000042480000EE0300000A
:10ED80001C0000207100000001000000D002000003
:10ED90001E00000042480000EF0300001C0000209D
:10EDA00072000000000000009F050000000000004D
:10EDB00042480000F00300001C0000207300000027
:10EDC000000000009F050000000000004248000015
:10EDD000F10300001C00002074000000010000008E
:10EDE000D00200003C00000042480000F203000096
:10EDF0001C0000207500000001000000D00200008F
:10EE00001E00000042480000F30300001C00002028
:10EE100076000000000000009F05000000000000D8
:10EE200042480000F40300001C00002077000000AE
:10EE3000000000009F0500000000000042480000A4
:10EE4000F50300001C000020780000000100000015
:10EE5000D00200003C00000042480000F603000021
:10EE60001C0000207900000001000000D00200001A
:10EE70001E00000042480000F70300001C000020B4
:10EE80007A000000000000009F0500000000000064
:10EE900042480000F80300001C0000207B00000036
:10EEA000000000009F050000000000004248000034
:10EEB000F90300001C0000207C000000010000009D
:10EEC000D00200003C00000042480000FA030000AD
:10EED0001C0000207D00000001000000D0020000A6
:10EEE0001E00000042480000FB0300001C00002040
:10EEF0007E000000000000009F05000000000000F0
:10EF000042480000FC0300001C0000207F000000BD
:10EF1000000000009F0500000000000042480000C3
:10EF2000FD0300001C000020800000000100000024
:10EF3000D00200003C00000042480000FE03000038
:10EF40001C0000208100000001000000D002000031
:10EF50001E00000042480000FF0300001C000020CB
:10EF600082000000000000009F050000000000007B
:10EF700042480000000400001C0000208300000044
:10EF8000000000009F050000000000004248000053
:10EF9000010400001C0000208400000001000000AB
:10EFA000D00200003C0000004248000002040000C3
:10EFB0001C0000208500000001000000D0020000BD
:10EFC0001E00000042480000030400001C00002056
:10EFD0008701000020202020FFFFFF7F31302D56C9
:10EFE00002480100D00700001C000020870000003C
:10EFF000000000000500000000000000020000000A
:10F00000D10700001C00002088000000BC020000A6
:10F01000B00400008403000012500000D20700007A
:10F020001C000020A100000001000000100E0000E4
:10F030000A000000C2480000D30700001C000020A6
:10F0400089000000000000009F0500000000000093
:10F0500042480000D40700001C0000208A00000085
:10F06000000000009F050000000000004248000072
:10F07000D50700001C0000208B00000001000000EC
:10F08000D00200003C00000042480000D60700000B
:10F090001C0000208C00000001000000D0020000D5
:10F0A0001E00000042480000D70700001C0000209E
:10F0B0008D000000000000009F050000000000001F
:10F0C00042480000D80700001C0000208E0000000D
:10F0D000000000009F050000000000004248000002
:10F0E000D90700001C0000208F0000000100000074
:10F0F000D00200003C00000042480000DA07000097
:10F100001C0000209000000001000000D002000060
:10F110001E00000042480000DB0700001C00002029
:10F1200091000000000000009F05000000000000AA
:10F1300042480000DC0700001C0000209200000094
:10F14000000000009F050000000000004248000091
:10F15000DD0700001C0000209300000001000000FB
:10F16000D00200003C00000042480000DE07000022
:10F170001C0000209400000001000000D0020000EC
:10F180001E00000042480000DF0700001C000020B5
:10F1900095000000000000009F0500000000000036
:10F1A00042480000E00700001C000020960000001C
:10F1B000000000009F050000000000004248000021
:10F1C000E10700001C000020970000000100000083
:10F1D000D00200003C00000042480000E2070000AE
:10F1E0001C0000209800000001000000D002000078
:10F1F0001E00000042480000E30700001C00002041
:10F2000099000000000000009F05000000000000C1
:10F2100042480000E40700001C0000209A000000A3
:10F22000000000009F0500000000000042480000B0
:10F23000E50700001C0000209B000000010000000A
:10F24000D00200003C00000042480000E607000039
:10F250001C0000209C00000001000000D002000003
:10F260001E00000042480000E70700001C000020CC
:10F270009D000000000000009F050000000000004D
:10F2800042480000E80700001C0000209E0000002B
:10F29000000000009F050000000000004248000040
:10F2A000E90700001C0000209F0000000100000092
:10F2B000D00200003C00000042480000EA070000C5
:10F2C0001C000020A000000001000000D00200008F
:10F2D0001E00000042480000EB0700001C00002058
:10F2E0008801000020202020FFFFFF7F32302D56B4
:10F2F00002480100B80B00001C000020A200000022
:10F3000000000000050000000000000002000000F6
:10F31000B90B00001C000020A3000000BC0200008C
:10F32000B00400008403000012500000BA0B00007B
:10F330001C000020BC00000001000000100E0000B6
:10F340000A000000C2480000BB0B00001C000020A7
:10F35000A4000000000000009F0500000000000065
:10F3600042480000BC0B00001C000020A50000006B
:10F37000000000009F05000000000000424800005F
:10F38000BD0B00001C000020A600000001000000D2
:10F39000D00200003C00000042480000BE0B00000C
:10F3A0001C000020A700000001000000D0020000A7
:10F3B0001E00000042480000BF0B00001C0000209F
:10F3C000A8000000000000009F05000000000000F1
:10F3D00042480000C00B00001C000020A9000000F3
:10F3E000000000009F0500000000000042480000EF
:10F3F000C10B00001C000020AA000000010000005A
:10F40000D00200003C00000042480000C20B000097
:10F410001C000020AB00000001000000D002000032
:10F420001E00000042480000C30B00001C0000202A
:10F43000AC000000000000009F050000000000007C
:10F4400042480000C40B00001C000020AD0000007A
:10F45000000000009F05000000000000424800007E
:10F46000C50B00001C000020AE00000001000000E1
:10F47000D00200003C00000042480000C60B000023
:10F480001C000020AF00000001000000D0020000BE
:10F490001E00000042480000C70B00001C000020B6
:10F4A000B0000000000000009F0500000000000008
:10F4B00042480000C80B00001C000020B100000002
:10F4C000000000009F05000000000000424800000E
:10F4D000C90B00001C000020B20000000100000069
:10F4E000D00200003C00000042480000CA0B0000AF
:10F4F0001C000020B300000001000000D00200004A
:10F500001E00000042480000CB0B00001C00002041
:10F51000B4000000000000009F0500000000000093
:10F5200042480000CC0B00001C000020B500000089
:10F53000000000009F05000000000000424800009D
:10F54000CD0B00001C000020B600000001000000F0
:10F55000D00200003C00000042480000CE0B00003A
:10F560001C000020B700000001000000D0020000D5
:10F570001E00000042480000CF0B00001C000020CD
:10F58000B8000000000000009F050000000000001F
:10F5900042480000D00B00001C000020B900000011
:10F5A000000000009F05000000000000424800002D
:10F5B000D10B00001C000020BA0000000100000078
:10F5C000D00200003C00000042480000D20B0000C6
:10F5D0001C000020BB00000001000000D002000061
:10F5E0001E00000042480000D30B00001C00002059
:10F5F0008901000020202020FFFFFF7F33302D569F
:10F6000002480100A00F00001C000020BD00000007
:10F6100000000000050000000000000002000000E3
:10F62000A10F00001C000020BE000000BC02000072
:10F63000B00400008403000012500000A20F00007C
:10F640001C000020D700000001000000100E000088
:10F650000A000000C2480000A30F00001C000020A8
:10F66000BF000000000000009F0500000000000037
:10F6700042480000A40F00001C000020C000000051
:10F68000000000009F05000000000000424800004C
:10F69000A50F00001C000020C100000001000000B8
:10F6A000D00200003C00000042480000A60F00000D
:10F6B0001C000020C200000001000000D002000079
:10F6C0001E00000042480000A70F00001C000020A0
:10F6D000C3000000000000009F05000000000000C3
:10F6E00042480000A80F00001C000020C4000000D9
:10F6F000000000009F0500000000000042480000DC
:10F70000A90F00001C000020C5000000010000003F
:10F71000D00200003C00000042480000AA0F000098
:10F720001C000020C600000001000000D002000004
:10F730001E00000042480000AB0F00001C0000202B
:10F74000C7000000000000009F050000000000004E
:10F7500042480000AC0F00001C000020C800000060
:10F76000000000009F05000000000000424800006B
:10F77000AD0F00001C000020C900000001000000C7
:10F78000D00200003C00000042480000AE0F000024
:10F790001C000020CA00000001000000D002000090
:10F7A0001E00000042480000AF0F00001C000020B7
:10F7B000CB000000000000009F05000000000000DA
:10F7C00042480000B00F00001C000020CC000000E8
:10F7D000000000009F0500000000000042480000FB
:10F7E000B10F00001C000020CD000000010000004F
:10F7F000D00200003C00000042480000B20F0000B0
:10F800001C000020CE00000001000000D00200001B
:10F810001E00000042480000B30F00001C00002042
:10F82000CF000000000000009F0500000000000065
:10F8300042480000B40F00001C000020D00000006F
:10F84000000000009F05000000000000424800008A
:10F85000B50F00001C000020D100000001000000D6
:10F86000D00200003C00000042480000B60F00003B
:10F870001C000020D200000001000000D0020000A7
:10F880001E00000042480000B70F00001C000020CE
:10F89000D3000000000000009F05000000000000F1
:10F8A00042480000B80F00001C000020D4000000F7
:10F8B000000000009F05000000000000424800001A
:10F8C000B90F00001C000020D5000000010000005E
:10F8D000D00200003C00000042480000BA0F0000C7
:10F8E0001C000020D600000001000000D002000033
:10F8F0001E00000042480000BB0F00001C0000205A
:10F900008A01000020202020FFFFFF7F34302D5689
:10F9100002480100881300001C000020D8000000ED
:10F9200000000000050000000000000002000000D0
:10F93000891300001C000020D9000000BC02000058
:10F94000B004000084030000125000008A1300007D
:10F950001C000020F200000001000000100E00005A
:10F960000A000000C24800008B1300001C000020A9
:10F97000DA000000000000009F0500000000000009
:10F98000424800008C1300001C000020DB00000037
:10F99000000000009F050000000000004248000039
:10F9A0008D1300001C000020DC000000010000009E
:10F9B000D00200003C000000424800008E1300000E
:10F9C0001C000020DD00000001000000D00200004B
:10F9D0001E000000424800008F1300001C000020A1
:10F9E000DE000000000000009F0500000000000095
:10F9F00042480000901300001C000020DF000000BF
:10FA0000000000009F0500000000000042480000C8
:10FA1000911300001C000020E00000000100000025
:10FA2000D00200003C000000424800009213000099
:10FA30001C000020E100000001000000D0020000D6
:10FA40001E00000042480000931300001C0000202C
:10FA5000E2000000000000009F0500000000000020
:10FA600042480000941300001C000020E300000046
:10FA7000000000009F050000000000004248000058
:10FA8000951300001C000020E400000001000000AD
:10FA9000D00200003C000000424800009613000025
:10FAA0001C000020E500000001000000D002000062
:10FAB0001E00000042480000971300001C000020B8
:10FAC000E6000000000000009F05000000000000AC
:10FAD00042480000981300001C000020E7000000CE
:10FAE000000000009F0500000000000042480000E8
:10FAF000991300001C000020E80000000100000035
:10FB0000D00200003C000000424800009A130000B0
:10FB10001C000020E900000001000000D0020000ED
:10FB20001E000000424800009B1300001C00002043
:10FB3000EA000000000000009F0500000000000037
:10FB4000424800009C1300001C000020EB00000055
:10FB5000000000009F050000000000004248000077
:10FB60009D1300001C000020EC00000001000000BC
:10FB7000D00200003C000000424800009E1300003C
:10FB80001C000020ED00000001000000D002000079
:10FB90001E000000424800009F1300001C000020CF
:10FBA000EE000000000000009F05000000000000C3
:10FBB00042480000A01300001C000020EF000000DD
:10FBC000000000009F050000000000004248000007
:10FBD000A11300001C000020F00000000100000044
:10FBE000D00200003C00000042480000A2130000C8
:10FBF0001C000020F100000001000000D002000005
:10FC00001E00000042480000A31300001C0000205A
:10FC10008B01000020202020FFFFFF7F35302D5674
:10FC200002480100701700001C000020F3000000D3
:10FC300000000000050000000000000002000000BD
:10FC4000711700001C000020F4000000BC0200003E
:10FC5000B00400008403000012500000721700007E
:10FC60001C0000200D01000001000000100E00002B
:10FC70000A000000C2480000731700001C000020AA
:10FC8000F5000000000000009F05000000000000DB
:10FC900042480000741700001C000020F60000001D
:10FCA000000000009F050000000000004248000026
:10FCB000751700001C000020F70000000100000084
:10FCC000D00200003C00000042480000761700000F
:10FCD0001C000020F800000001000000D00200001D
:10FCE0001E00000042480000771700001C000020A2
:10FCF000F9000000000000009F0500000000000067
:10FD000042480000781700001C000020FA000000A4
:10FD1000000000009F0500000000000042480000B5
:10FD2000791700001C000020FB000000010000000B
:10FD3000D00200003C000000424800007A1700009A
:10FD40001C000020FC00000001000000D0020000A8
:10FD50001E000000424800007B1700001C0000202D
:10FD6000FD000000000000009F05000000000000F2
:10FD7000424800007C1700001C000020FE0000002C
:10FD8000000000009F050000000000004248000045
:10FD90007D1700001C000020FF0000000100000093
:10FDA000D00200003C000000424800007E17000026
:10FDB0001C0000200001000001000000D002000033
:10FDC0001E000000424800007F1700001C000020B9
:10FDD00001010000000000009F050000000000007D
:10FDE00042480000801700001C00002002010000B3
:10FDF000000000009F0500000000000042480000D5
:10FE0000811700001C000020030100000100000019
:10FE1000D00200003C0000004248000082170000B1
:10FE20001C0000200401000001000000D0020000BE
:10FE30001E00000042480000831700001C00002044
:10FE400005010000000000009F0500000000000008
:10FE500042480000841700001C000020060100003A
:10FE6000000000009F050000000000004248000064
:10FE7000851700001C0000200701000001000000A1
:10FE8000D00200003C00000042480000861700003D
:10FE90001C0000200801000001000000D00200004A
:10FEA0001E00000042480000871700001C000020D0
:10FEB00009010000000000009F0500000000000094
:10FEC00042480000881700001C0000200A010000C2
:10FED000000000009F0500000000000042480000F4
:10FEE000891700001C0000200B0100000100000029
:10FEF000D00200003C000000424800008A170000C9
:10FF00001C0000200C01000001000000D0020000D5
:10FF10001E000000424800008B1700001C0000205B
:10FF20008C01000020202020FFFFFF7F36302D565F
:10FF300002480100581B00001C0000200E010000B8
:10FF400000000000050000000000000002000000AA
:10FF5000591B00001C0000200F010000BC02000023
:10FF6000B004000084030000125000005A1B00007F
:10FF70001C0000202801000001000000100E0000FD
:10FF80000A000000C24800005B1B00001C000020AB
:10FF900010010000000000009F05000000000000AC
:10FFA000424800005C1B00001C0000201101000002
:10FFB000000000009F050000000000004248000013
:10FFC0005D1B00001C000020120100000100000069
:10FFD000D00200003C000000424800005E1B000010
:10FFE0001C0000201301000001000000D0020000EE
:10FFF0001E000000424800005F1B00001C000020A3
:020000040802F0
:1000000014010000000000009F0500000000000037
:1000100042480000601B00001C0000201501000089
:10002000000000009F0500000000000042480000A2
:10003000611B00001C0000201601000001000000F0
:10004000D00200003C00000042480000621B00009B
:100050001C0000201701000001000000D002000079
:100060001E00000042480000631B00001C0000202E
:1000700018010000000000009F05000000000000C3
:1000800042480000641B00001C0000201901000011
:10009000000000009F050000000000004248000032
:1000A000651B00001C0000201A0100000100000078
:1000B000D00200003C00000042480000661B000027
:1000C0001C0000201B01000001000000D002000005
:1000D0001E00000042480000671B00001C000020BA
:1000E0001C010000000000009F050000000000004F
:1000F00042480000681B00001C0000201D01000099
:10010000000000009F0500000000000042480000C1
:10011000691B00001C0000201E01000001000000FF
:10012000D00200003C000000424800006A1B0000B2
:100130001C0000201F01000001000000D002000090
:100140001E000000424800006B1B00001C00002045
:1001500020010000000000009F05000000000000DA
:10016000424800006C1B00001C0000202101000020
:10017000000000009F050000000000004248000051
:100180006D1B00001C000020220100000100000087
:10019000D00200003C000000424800006E1B00003E
:1001A0001C0000202301000001000000D00200001C
:1001B0001E000000424800006F1B00001C000020D1
:1001C00024010000000000009F0500000000000066
:1001D00042480000701B00001C00002025010000A8
:1001E000000000009F0500000000000042480000E1
:1001F000711B00001C00002026010000010000000F
:10020000D00200003C00000042480000721B0000C9
:100210001C0000202701000001000000D0020000A7
:100220001E00000042480000731B00001C0000205C
:100230008D01000020202020FFFFFF7F37302D564A
:1002400002480100401F00001C000020290100009E
:100250000000000005000000000000000200000097
:10026000411F00001C0000202A010000BC02000009
:10027000B00400008403000012500000421F000080
:100280001C0000204301000001000000100E0000CF
:100290000A000000C2480000431F00001C000020AC
:1002A0002B010000000000009F050000000000007E
:1002B00042480000441F00001C0000202C010000E8
:1002C000000000009F050000000000004248000000
:1002D000451F00001C0000202D010000010000004F
:1002E000D00200003C00000042480000461F000011
:1002F0001C0000202E01000001000000D0020000C0
:100300001E00000042480000471F00001C000020A3
:100310002F010000000000009F0500000000000009
:1003200042480000481F00001C000020300100006F
:10033000000000009F05000000000000424800008F
:10034000491F00001C0000203101000001000000D6
:10035000D00200003C000000424800004A1F00009C
:100360001C0000203201000001000000D00200004B
:100370001E000000424800004B1F00001C0000202F
:1003800033010000000000009F0500000000000095
:10039000424800004C1F00001C00002034010000F7
:1003A000000000009F05000000000000424800001F
:1003B0004D1F00001C00002035010000010000005E
:1003C000D00200003C000000424800004E1F000028
:1003D0001C0000203601000001000000D0020000D7
:1003E0001E000000424800004F1F00001C000020BB
:1003F00037010000000000009F0500000000000021
:1004000042480000501F00001C000020380100007E
:10041000000000009F0500000000000042480000AE
:10042000511F00001C0000203901000001000000E5
:10043000D00200003C00000042480000521F0000B3
:100440001C0000203A01000001000000D002000062
:100450001E00000042480000531F00001C00002046
:100460003B010000000000009F05000000000000AC
:1004700042480000541F00001C0000203C01000006
:10048000000000009F05000000000000424800003E
:10049000551F00001C0000203D010000010000006D
:1004A000D00200003C00000042480000561F00003F
:1004B0001C0000203E01000001000000D0020000EE
:1004C0001E00000042480000571F00001C000020D2
:1004D0003F010000000000009F0500000000000038
:1004E00042480000581F00001C000020400100008E
:1004F000000000009F0500000000000042480000CE
:10050000591F00001C0000204101000001000000F4
:10051000D00200003C000000424800005A1F0000CA
:100520001C0000204201000001000000D002000079
:100530001E000000424800005B1F00001C0000205D
:100540008E01000020202020FFFFFF7F38302D5635
:1005500002480100282300001C0000204401000084
:100560000000000005000000000000000200000084
:10057000292300001C00002045010000BC020000EF
:10058000B004000084030000125000002A23000081
:100590001C0000205E01000001000000100E0000A1
:1005A0000A000000C24800002B2300001C000020AD
:1005B00046010000000000009F0500000000000050
:1005C000424800002C2300001C00002047010000CE
:1005D000000000009F0500000000000042480000ED
:1005E0002D2300001C000020480100000100000035
:1005F000D00200003C000000424800002E23000012
:100600001C0000204901000001000000D002000091
:100610001E000000424800002F2300001C000020A4
:100620004A010000000000009F05000000000000DB
:1006300042480000302300001C0000204B01000055
:10064000000000009F05000000000000424800007C
:10065000312300001C0000204C01000001000000BC
:10066000D00200003C00000042480000322300009D
:100670001C0000204D01000001000000D00200001D
:100680001E00000042480000332300001C00002030
:100690004E010000000000009F0500000000000067
:1006A00042480000342300001C0000204F010000DD
:1006B000000000009F05000000000000424800000C
:1006C000352300001C000020500100000100000044
:1006D000D00200003C000000424800003623000029
:1006E0001C0000205101000001000000D0020000A9
:1006F0001E00000042480000372300001C000020BC
:1007000052010000000000009F05000000000000F2
:1007100042480000382300001C0000205301000064
:10072000000000009F05000000000000424800009B
:10073000392300001C0000205401000001000000CB
:10074000D00200003C000000424800003A230000B4
:100750001C0000205501000001000000D002000034
:100760001E000000424800003B2300001C00002047
:1007700056010000000000009F050000000000007E
:10078000424800003C2300001C00002057010000EC
:10079000000000009F05000000000000424800002B
:1007A0003D2300001C000020580100000100000053
:1007B000D00200003C000000424800003E23000040
:1007C0001C0000205901000001000000D0020000C0
:1007D0001E000000424800003F2300001C000020D3
:1007E0005A010000000000009F050000000000000A
:1007F00042480000402300001C0000205B01000074
:10080000000000009F0500000000000042480000BA
:10081000412300001C0000205C01000001000000DA
:10082000D00200003C0000004248000042230000CB
:100830001C0000205D01000001000000D00200004B
:100840001E00000042480000432300001C0000205E
:100850008F01000020202020FFFFFF7F39302D5620
:1008600002480100102700001C0000205F0100006A
:100870000000000005000000000000000200000071
:10088000112700001C00002060010000BC020000D5
:10089000B004000084030000125000001227000082
:1008A0001C0000207901000001000000100E000073
:1008B0000A000000C2480000132700001C000020AE
:1008C00061010000000000009F0500000000000022
:1008D00042480000142700001C00002062010000B4
:1008E000000000009F0500000000000042480000DA
:1008F000152700001C00002063010000010000001B
:10090000D00200003C000000424800001627000012
:100910001C0000206401000001000000D002000063
:100920001E00000042480000172700001C000020A5
:1009300065010000000000009F05000000000000AD
:1009400042480000182700001C000020660100003B
:10095000000000009F050000000000004248000069
:10096000192700001C0000206701000001000000A2
:10097000D00200003C000000424800001A2700009E
:100980001C0000206801000001000000D0020000EF
:100990001E000000424800001B2700001C00002031
:1009A00069010000000000009F0500000000000039
:1009B000424800001C2700001C0000206A010000C3
:1009C000000000009F0500000000000042480000F9
:1009D0001D2700001C0000206B010000010000002A
:1009E000D00200003C000000424800001E2700002A
:1009F0001C0000206C01000001000000D00200007B
:100A00001E000000424800001F2700001C000020BC
:100A10006D010000000000009F05000000000000C4
:100A200042480000202700001C0000206E0100004A
:100A3000000000009F050000000000004248000088
:100A4000212700001C0000206F01000001000000B1
:100A5000D00200003C0000004248000022270000B5
:100A60001C0000207001000001000000D002000006
:100A70001E00000042480000232700001C00002048
:100A800071010000000000009F0500000000000050
:100A900042480000242700001C00002072010000D2
:100AA000000000009F050000000000004248000018
:100AB000252700001C000020730100000100000039
:100AC000D00200003C000000424800002627000041
:100AD0001C0000207401000001000000D002000092
:100AE0001E00000042480000272700001C000020D4
:100AF00075010000000000009F05000000000000DC
:100B000042480000282700001C0000207601000059
:100B1000000000009F0500000000000042480000A7
:100B2000292700001C0000207701000001000000C0
:100B3000D00200003C000000424800002A270000CC
:100B40001C0000207801000001000000D00200001D
:100B50001E000000424800002B2700001C0000205F
:100B60009001000020202020FFFFFF7F30312D5614
:100B700002480100FFFF000000000000000000002C
:100B80000000000000000000000000000000000065
:100B90000000000054220E00010000000A000000C6
:100BA0002A070D000200000014000000E7030C00FB
:100BB000030000001E00000064160B00040000008B
:100BC00028000000AF3C0A000500000032000000D1
:100BD00004750900070000003C000000CBBD0800C0
:100BE0000800000046000000911508000A000000FF
:100BF00050000000077B07000B0000005A000000B7
:100C0000FCEC06000D000000640000005A6A0600BB
:100C10000F0000006E00000028F205001100000027
:100C2000780000007F8305001300000082000000B0
:100C3000921D0500160000008C000000A2BF0400F9
:100C40001800000096000000046904001B0000006A
:100C5000A00000001B1904001D000000AA000000F5
:100C600058CF030021000000B40000003A8B0300BD
:100C700024000000BE000000494C030027000000D3
:100C8000C80000001A1203002B000000D200000070
:100C90004ADC02002F000000DC0000007DAA0200F8
:100CA00033000000E6000000637C02003700000013
:100CB000F0000000AE5102003C000000FA0000000D
:100CC0001A2A020041000000040100006905020028
:100CD000460000000E0100005FE301004C00000030
:100CE00018010000C8C301005200000022010000EA
:100CF00073A60100580000002C010000348B010095
:100D00005F00000036010000E17101006600000094
:100D100040010000565A01006E0000004A01000028
:100D20006F44010076000000540100000D30010006
:100D30007E0000005E010000131D0100870000001E
:100D400068010000660B01009000000072010000C5
:100D5000EDFA00009A0000007C01000091EB000019
:100D6000A4000000860100003EDD0000AF0000008E
:100D700090010000E0CF0000BA0000009A010000DE
:100D800066C30000C6000000A4010000BFB7000059
:100D9000D3000000AE010000DCAC0000E000000069
:100DA000B8010000AFA20000EE000000C201000088
:100DB0002B990000FC000000CC01000044900000D2
:100DC0000C010000D6010000EF8700001B010000AD
:100DD000E0010000228000002C010000EA01000078
:100DE000D47800003D010000F4010000FC71000017
:100DF0004F010000FE010000916B00006201000045
:100E0000080200008D65000076010000120200005B
:100E1000E85F00008B0100001C0200009C5A0000EB
:100E2000A001000026020000A3550000B60100004A
:100E300030020000F8500000CD0100003A0200002E
:100E4000944C0000E50100004402000075480000D9
:100E5000FE0100004E020000944400001702000052
:100E600058020000EE400000320200006202000062
:100E7000803D00004D0200006C020000453A000079
:100E800069020000760200003A3700008702000085
:100E9000800200005D340000A50200008A0200000C
:100EA000AA310000C4020000940200001E2F0000BE
:100EB000E40200009E020000B82C000005030000C0
:100EC000A8020000752A000026030000B2020000FC
:100ED0005228000049030000BC0200004E2600001A
:100EE0006C030000C60200006724000090030000AD
:100EF000D00200009B220000B5030000DA020000CF
:100F0000E8200000DB030000E40200004D1F0000A9
:100F100002040000EE020000C91D000029040000C8
:100F2000F8020000591C00005104000002030000F8
:100F3000FD1A00007A0400000C030000B419000040
:100F4000A4040000160300007D180000CD0400007A
:100F50002003000056170000F80400002A030000D8
:100F60003F16000023050000340300003615000082
:100F70004F0500003E0300003B1400007B0500000D
:100F8000480300004D130000A805000052030000B4
:100F90006B120000D50500005C03000095110000F5
:100FA0000206000066030000CA1000002F060000C1
:100FB00070030000091000005D0600007A030000C5
:100FC000520F00008B06000084030000A40E0000F6
:100FD000B90600008E030000FF0D0000E8060000C7
:100FE00098030000620D000016070000A203000035
:100FF000CD0C000044070000AC0300003F0C0000D3
:1010000072070000B6030000B80B0000A007000044
:10101000C0030000380B0000CE070000CA03000028
:10102000BD0A0000FC070000D4030000490A0000CC
:101030002A080000DE030000DA090000570800005B
:10104000E80300007109000084080000F2030000BA
:101050000C090000B1080000FC030000AC0800000F
:10106000DD08000006040000510800000909000026
:1010700010040000FA070000350900001A040000FF
:10108000A7070000600900002404000058070000C2
:101090008A0900002E0400000C070000B4090000BB
:1010A00038040000C4060000DE090000420400000D
:1010B0007F060000070A00004C0400003D06000007
:1010C0002F0A000056040000FF050000560A000029
:1010D00060040000C30500007D0A00006A040000EF
:1010E00089050000A40A00007404000053050000F4
:1010F000CA0A00007E0400001E050000EF0A00007E
:1011000088040000EC040000130B000092040000AF
:10111000BC040000370B00009C0400008E0400009B
:101120005A0B0000A6040000630400007C0B0000C2
:10113000B0040000390400009E0B0000BA04000057
:1011400010040000BE0B0000C4040000EA0300000D
:10115000DF0B0000CE040000C5030000FE0B000002
:10116000D8040000A20300001D0C0000E2040000EF
:10117000800300003B0C0000EC0400005F03000053
:10118000580C0000F604000040030000750C00003D
:101190000005000023030000910C00000A05000078
:1011A00006030000AC0C000014050000EB02000078
:1011B000C70C00001E050000D0020000E00C00007B
:1011C00028050000B7020000FA0C000032050000FC
:1011D0009F020000120D00003C0500008802000084
:1011E0002A0D00004605000071020000420D0000BB
:1011F000500500005C020000580D00005A05000078
:10120000470200006E0D000064050000330200007C
:10121000840D00006E05000020020000990D000002
:10122000780500000E020000AD0D000082050000F0
:10123000FC010000C10D00008C050000EC01000065
:10124000D40D000096050000DB010000E70D000052
:10125000A0050000CC010000F90D0000AA05000067
:10126000BD0100000B0E0000B4050000AE0100003F
:101270001C0E0000BE050000A00100002D0E0000A5
:10128000C8050000930100003D0E0000D2050000DB
:10129000860100004D0E0000DC0500007901000011
:1012A0005C0E0000E60500006E0100006B0E000001
:1012B000F005000062010000790E0000FA05000050
:1012C00057010000870E0000040600004C010000DA
:1012D000950E00000E06000042010000A20E000064
:1012E0001806000038010000AF0E000022060000C2
:1012F0002E010000BB0E00002C060000250100009E
:10130000C70E0000360600001C010000D30E0000CE
:101310004006000013010000DE0E00004A06000037
:101320000B010000E90E000054060000030100005C
:10133000F40E00005E060000FB000000FE0E000040
:1013400068060000F4000000080F000072060000AC
:10135000ED000000120F00007C060000E600000017
:101360001C0F000086060000DF000000250F0000B3
:1013700090060000D90000002E0F00009A06000021
:10138000D2000000360F0000A4060000CC000000D0
:101390003F0F0000AE060000C6000000470F00002F
:1013A000B8060000C10000004F0F0000C206000098
:1013B000BB000000570F0000CC060000B600000084
:1013C0005E0F0000D6060000B1000000650F0000AF
:1013D000E0060000AC0000006D0F0000EA0600000F
:1013E000A7000000730F0000F4060000A200000038
:1013F0007A0F0000FE0600009E000000800F000033
:10140000080700009A000000860F00001207000085
:10141000950000008D0F00001C07000091000000E7
:10142000930F0000260700008D000000980F0000B9
:10143000300700008A0000009E0F00003A070000FD
:1014400086000000A30F0000440700008200000097
:10145000A80F00004E0700007F000000AE0F000044
:10146000580700007C000000B20F00006207000077
:1014700078000000B70F00006C0700007500000046
:10148000BC0F00007607000072000000C10F0000D2
:10149000800700006F000000C50F00008A070000F1
:1014A0006C000000C90F00009407000069000000F4
:1014B000CD0F00009E07000067000000D10F000064
:1014C000A807000064000000D50F0000B20700006C
:1014D00062000000D90F0000BC0700005F000000A0
:1014E000DD0F0000C60700005D000000E00F0000F7
:1014F000D00700005A000000E40F0000DA070000E7
:1015000058000000E70F0000E4070000560000004C
:10151000EB0F0000EE07000054000000EE0F00008B
:10152000F807000052000000F10F00000208000060
:1015300050000000F40F00000C0800004E000000F6
:10154000F70F0000160800004C000000FA0F000022
:10155000200800004A000000FD0F00002A080000DB
:1015600048000000FF0F00003408000047000000A2
:1015700002100000000000002110000042200000C6
:101580006330000084400000A5500000C6600000E9
:10159000E770000008810000299100004AA10000C6
:1015A0006BB100008CC10000ADD10000CEE10000A5
:1015B000EFF1000031120000100200007332000051
:1015C00052220000B552000094420000F772000061
:1015D000D662000039930000188300007BB300003E
:1015E0005AA30000BDD300009CC30000FFF300001D
:1015F000DEE3000062240000433400002004000009
:1016000001140000E6640000C7740000A444000058
:10161000855400006AA500004BB500002885000035
:1016200009950000EEE50000CFF50000ACC5000014
:101630008DD5000053360000722600001116000000
:1016400030060000D7760000F666000095560000D0
:10165000B44600005BB700007AA7000019970000AD
:1016600038870000DFF70000FEE700009DD700008C
:10167000BCC70000C4480000E558000086680000B0
:10168000A778000040080000611800000228000050
:1016900023380000CCC90000EDD900008EE900001D
:1016A000AFF9000048890000699900000AA900000C
:1016B0002BB90000F55A0000D44A0000B77A0000A8
:1016C000966A0000711A0000500A0000333A0000C8
:1016D000122A0000FDDB0000DCCB0000BFFB000095
:1016E0009EEB0000799B0000588B00003BBB000084
:1016F0001AAB0000A66C0000877C0000E44C0000E0
:10170000C55C0000222C0000033C0000600C0000BF
:10171000411C0000AEED00008FFD0000ECCD00008C
:10172000CDDD00002AAD00000BBD0000688D00007B
:10173000499D0000977E0000B66E0000D55E000057
:10174000F44E0000133E0000322E0000511E000037
:10175000700E00009FFF0000BEEF0000DDDF000004
:10176000FCCF00001BBF00003AAF0000599F0000F3
:10177000788F000088910000A9810000CAB10000A4
:10178000EBA100000CD100002DC100004EF10000C3
:101790006FE1000080100000A1000000C2300000D6
:1017A000E3200000045000002540000046700000C7
:1017B00067600000B983000098930000FBA300005D
:1017C000DAB300003DC300001CD300007FE300003B
:1017D0005EF30000B102000090120000F32200004E
:1017E000D23200003542000014520000776200003F
:1017F00056720000EAB50000CBA50000A8950000D5
:10180000898500006EF500004FE500002CD5000032
:101810000DC50000E2340000C3240000A014000045
:101820008104000066740000476400002454000036
:1018300005440000DBA70000FAB70000998700000C
:10184000B89700005FE700007EF700001DC70000AA
:101850003CD70000D3260000F236000091060000BD
:10186000B0160000576600007676000015460000AE
:10187000345600004CD900006DC900000EF900007C
:101880002FE90000C8990000E98900008AB900002A
:10189000ABA900004458000065480000067800002D
:1018A00027680000C0180000E1080000823800002E
:1018B000A32800007DCB00005CDB00003FEB0000B4
:1018C0001EFB0000F98B0000D89B0000BBAB0000A2
:1018D0009ABB0000754A0000545A0000376A0000A5
:1018E000167A0000F10A0000D01A0000B32A0000A6
:1018F000923A00002EFD00000FED00006CDD0000AC
:101900004DCD0000AABD00008BAD0000E89D000099
:10191000C98D0000267C0000076C0000645C00009C
:10192000454C0000A23C0000832C0000E01C00009D
:10193000C10C00001FEF00003EFF00005DCF000063
:101940007CDF00009BAF0000BABF0000D98F000011
:10195000F89F0000176E0000367E0000554E000014
:10196000745E0000932E0000B23E0000D10E000015
:10197000F01E0000000000000000000000005F00FA
:10198000000000000007000700000000147F147F23
:1019900014000000242A7F2A120000002313086488
:1019A0006200000036495522400000000005030097
:1019B00000000000001C2241000000000041221C29
:1019C0000000000014083E081400000008083E084B
:1019D000080000000050300000000000080808085F
:1019E00008000000006060000000000020100804F3
:1019F000020000003E4141413E00000000427F40A5
:101A00000000000042615149460000002141454B61
:101A1000310000001814127F1000000027454545D2
:101A2000390000003C4A49493000000001710905B5
:101A3000030000003649494936000000064949299B
:101A40001E00000000003636000000000056360080
:101A500000000000081C3E7F000000001414141455
:101A600014000000007F3E1C080000000201510924
:101A700006000000324979413E0000007E1111113C
:101A80007E0000007F494949360000003E41414147
:101A9000220000007F4141221C0000007F4949498B
:101AA000410000007F090909010000003E41494949
:101AB0003A0000007F0808087F00000000417F41D5
:101AC000000000002040413F010000007F08142278
:101AD000410000007F404040400000007F020C02B7
:101AE0007F0000007F0408107F0000003E4141415C
:101AF0003E0000007F090909060000003E41512117
:101B00005E0000007F091929460000004649494946
:101B10003100000001017F01010000003F40404012
:101B20003F0000001F2040201F0000003F40704089
:101B30003F000000631408146300000007087008E9
:101B4000070000006151494543000000007F41410A
:101B50000000000002040810200000000041417F46
:101B60000000000004020102040000004040404068
:101B70004000000000010200000000002054545406
:101B8000780000007F444444380000003844444456
:101B900020000000384444487F000000385454546A
:101BA00018000000087E09010200000018A4A4A487
:101BB0007C0000007F0804047800000000447D40A1
:101BC000000000002040443D000000007F10284439
:101BD0000000000000417F40000000007C04180469
:101BE000780000007C080404780000003844444475
:101BF00038000000FC2424241800000008141414E9
